:0200000460009A
:100400004643464200040156000000000103030079
:1004100001010000010400000200000000000000D3
:1004200000000000000000000000000000000000CC
:1004300000000000000000000000000000000000BC
:10044000000000000104080000000000000000009F
:10045000000040000000000000000000000000005C
:10046000000000000000000000000000000000008C
:10047000000000000000000000000000000000007C
:10048000EB04180A063204260000000000000000F9
:10049000050402240000000000000000000000002D
:1004A000000000000000000000000000000000004C
:1004B0000604000000000000000000000000000032
:1004C00031040120000000000000000000000000D6
:1004D00020041808000000000000000000000000D8
:1004E000000000000000000000000000000000000C
:1004F00000000000000000000000000000000000FC
:10050000D8041808000000000000000000000000EF
:100510000204180804200000000000000000000091
:1005200000000000000000000000000000000000CB
:100530006004000000000000000000000000000057
:1005400000000000000000000000000000000000AB
:10055000000000000000000000000000000000009B
:10056000000000000000000000000000000000008B
:10057000000000000000000000000000000000007B
:10058000000000000000000000000000000000006B
:10059000000000000000000000000000000000005B
:1005A000000000000000000000000000000000004B
:1005B000000000000000000000000000000000003B
:1005C0000001000000100000010000000000000019
:1005D000000001000000000000000000000000001A
:1005E000000000000000000000000000000000000B
:1005F00000000000000000000000000000000000FB
:10100000D100204100C0006000000000000000008E
:1010100020100060001000600000000000000000D0
:10102000000000600000400000000000FFFFFFFF24
:10C00000008000200D6B026035D90460657002600D
:10C010004D700260557002605D70026000000000AB
:10C020000000000000000000000000003DD9046096
:10C0300031D904600000000041D9046045D9046092
:10C0400049D904604DD9046051D9046055D90460C0
:10C0500059D904605DD9046061D9046065D9046070
:10C0600069D904606DD9046071D9046075D9046020
:10C0700079D904607DD9046081D9046085D90460D0
:10C0800089D9046031D9046031D9046031D90460A0
:10C090008DD9046091D9046095D9046099D9046060
:10C0A00031D9046051D602609DD9046031D9046051
:10C0B000A1D90460A5D9046031D9046031D90460E4
:10C0C000A9D90460ADD9046031D9046031D90460C4
:10C0D00031D9046031D9046031D9046031D90460A8
:10C0E00031D9046031D9046031D9046031D9046098
:10C0F00031D9046031D90460596F026031D90460CC
:10C1000031D9046031D9046031D9046031D9046077
:10C1100031D9046031D9046031D9046031D9046067
:10C12000B1D9046031D90460B5D90460B9D90460CB
:10C13000BDD9046031D9046031D9046031D90460BB
:10C1400031D9046031D9046031D9046031D9046037
:10C15000C1D9046031D9046031D9046031D9046097
:10C1600031D9046031D9046031D9046031D9046017
:10C1700031D9046031D9046031D9046031D9046007
:10C1800031D9046031D9046031D9046031D90460F7
:10C1900031D9046031D9046031D9046031D90460E7
:10C3F00031D9046031D9046031D90460FFFFFFFFF7
:10C40000044A03460020D16919601169D361996417
:10C41000704700BF00040020024BDA691268DA613D
:10C42000704700BF00040020C46005614661876159
:10C43000C0F81C80C0F82090C0F824A0C0F828B034
:10C44000C0F82CD080ED0C8B80ED0E9B80ED10ABF6
:10C45000C0F808E0FFF7D4BF114A08B5D3690BB99B
:10C460001AF050FB996C586011611968D161184637
:10C47000C468056946698769D0F81C80D0F82090A7
:10C48000D0F824A0D0F828B0D0F82CD090ED0C8BA8
:10C4900090ED0E9B90ED10ABD0F808E001207047B6
:10C4A0000004002010B50A460021044600F06CFB91
:10C4B00000B904B910BD204609F064FC0A46002109
:10C4C00000F062BB10B50A460121044600F05CFB97
:10C4D00000B904B910BD204609F054FCFFF7E2BFD3
:10C4E00010B501220C4600F0B3FC00B904B910BD30
:10C4F000204609F047FC00BF00F0AABC00F06ABC6F
:10C500002DE9F0434FF0030C00252A4CD4F8EC60E1
:10C510000021013143189A0803F00303B25C5B0069
:10C5200042FA03F303F00303022BF2D0D4F8F830FD
:10C53000090103EB00108A0811B300EB82020368C3
:10C5400019071AD1D4F8F810994216D8D4F8FC601B
:10C550009E4212D95B1AD4F8EC7048BF0F331B11FE
:10C560004FEA930E03F0030117F80E80490048FAD2
:10C5700001F606F00306012E09D004309042DED108
:10C58000B5B1013D04EB8503D3F80801BEE70CFA11
:10C5900001F13F2D04EB850941EA080107F80E106F
:10C5A00003D80135C9F80831E7E7C4F80461E4E7C6
:10C5B000BDE8F08300040020144B10B4D3F8F82039
:10C5C000824215D8D3F8FC10884211D2801AD3F8D1
:10C5D000EC4048BF0F300011810800F0030314F84D
:10C5E00001C05B004CFA03F202F00302012A02D000
:10C5F0005DF8044B7047032202FA03F343EA0C0C84
:10C6000004F801C05DF8044BFFF77ABF0004002076
:10C61000F8B5284DD5F8F820002A47D0821A4FF0F7
:10C620000103D5F8F4004FF0030748BF0F324FEA7B
:10C63000221E4FEADE010EF007024FEA9E0603FAC1
:10C6400002F2435CB44623EA0203724643540EF0FE
:10C650000301D5F8EC40A05D4900013207FA01F36F
:10C6600002F0030120EA03004B0004F80C004FEA3B
:10C67000920CD5F8EC4014F80C0040FA03F303F0E8
:10C680000303022BE8D0A2EB0E02082A28BF0822DF
:10C69000813205EB82025368B342D5F82C3288BF51
:10C6A0005660B34238BFC5F82C62F8BD08201BF0B5
:10C6B0001BFB00BF00040020164A10B4D2F8F8306B
:10C6C000834203D8D2F8FC10884203D300205DF8DF
:10C6D000044B7047C01AD2F8EC4048BF0F3003112A
:10C6E00000209A0803F00301A25C49000A4102F00D
:10C6F0000302012AEBD101301A18910802F003025B
:10C70000615C520041FA02F202F00302022AF2D006
:10C710000001DCE7000400200F4BD3F8F820824230
:10C7200003D8D3F8FC10884201D300207047801A48
:10C73000D3F8F43000280246B8BF00F17F02002889
:10C740004FEAE212B8BF0F309B5CC0F3021043FA0D
:10C7500000F000F0010070470004002021F00F01FC
:10C760001D4A38B50D1A1D4C0346ED00C4F8FC10E7
:10C77000C4F8EC00A2FB05256D0AA1EB85112B4442
:10C780002A46C4F8F8100021C4E93C5350F0CCF913
:10C790000021AA00D4F8F4000732D20850F0C4F9FE
:10C7A000D4F8F010D4F8F8200023481E02EB8112D0
:10C7B0000121C4F82C02C4F80021A4F8083284F83E
:10C7C0000A12C4F83032C4E98333C4E98533C4E9BA
:10C7D0008733C4E9893338BDF32C23FA00040020E1
:10C7E000034AB2F808320133A2F80832704700BF9A
:10C7F00000040020034AB2F80832013BA2F80832D4
:10C80000704700BF00040020034BB3F80802003853
:10C8100018BF0120704700BF00040020030701D1AA
:10C82000FFF7CABE704700BF70B50E4651B1051F75
:10C83000002455F8040F0134030701D1FFF7BCFEB3
:10C84000A642F6D170BD00BF70B5114E0022B6F8F9
:10C85000083206F1100406F1D805C6F804210133A8
:10C86000A6F8083254F8040F020701D1FFF7A4FE1E
:10C87000A542F7D1D6F83002030701D1FFF79CFE9D
:10C88000B0683169091ABDE870408908FFF7CCBF6C
:10C89000000400202DE9F04F614E83B0D6F804313A
:10C8A000D6F8F0C0002B00F0B88000254FEA8C07C6
:10C8B000C6F80451002F43D0002404F00303A0085D
:10C8C000D6F8EC105A000B5C134103F00303032B62
:10C8D0004BD00134BC42F0D3D6F80431002BE7D161
:10C8E00077B34FF0000E4FF003094FF0020A754680
:10C8F00004E0012B57D00135BD4221D2D6F8EC001F
:10C900004FEA950805F0030410F8082000EB9501A4
:10C91000640042FA04F303F00303022B35D0032B27
:10C92000E7D10AFA04F401354FF0000E22EA0402BE
:10C9300000F80820D6F8F0C04FEA8C07BD42DDD3DE
:10C94000B6F8081200220CF1FF330139C6F82C3278
:10C95000A6F80812C6E98322C6E98522C6E987221D
:10C96000C6E9892203B0BDE8F08F20460134FFF705
:10C97000C7FDD6F8F0C0B4EB8C0F4FEA8C079CD300
:10C98000D6F80431002B93D1AAE7BEF1000FB2D044
:10C9900009FA04F422EA040200F80820D6F8F0C0EC
:10C9A0004FEA8C07A7E7D6F8F400EF0805F0070B6D
:10C9B000C35D00EBD50C43FA0BF0C00721D5D6F8C8
:10C9C000F8002901415800EB051069B16A461121B0
:10C9D00009F0CAFB009810B101990AF007F9D6F8DE
:10C9E000F43003EB070CDB5D012202FA0BFB23EAB8
:10C9F0000B038CF80030D6F8EC3003EB080113F889
:10CA0000082009FA04F44FF0010E22EA04020A7029
:10CA1000D6F8F0C04FEA8C076DE74FEA8C075FE766
:10CA20000004002038B5074C0025B4F80832C4F8DB
:10CA300004510133A4F80832FFF72CFFC4F8F85072
:10CA400038BD00BF000400202DE9F04F484C002302
:10CA5000D4E93E129C46521AE64665460260674695
:10CA6000664661466246C0E90133C0E90333C0E966
:10CA70000533D4F8EC3093F800B063464FEA42082F
:10CA80004BFA08F808F00308B8F1010F64D0B8F1C8
:10CA9000020F5DD0B8F1000F55D0D4F8F02001336B
:10CAA00092009A420CBF4FF001094FF000093ED0AE
:10CAB0004FEA9308D4F8EC2012F808B003F0030210
:10CAC0004FEA420A4BFA0AFA1AF0030A14BFC846A0
:10CAD00049F00108B8F1000F42D1BAF1010FCDD1F0
:10CAE000C146D34601292AD0022902D14269013226
:10CAF0004261714501D98E468161BBF1000F0DD0B5
:10CB0000664501D9B446C660B9F1000F05D02D01C4
:10CB10003F01C0E90157BDE8F08F4E46D4F8EC2044
:10CB20004FEA930812F808B003F00302A6E7B8F141
:10CB3000010F14BFCB4649F0010B0129D4D1026982
:10CB400001320261D5E70137013641468760A4E72B
:10CB5000013501314560A0E70135414645609CE75C
:10CB6000BAF1010F14BFCB4649F0010BBAE700BF81
:10CB700000040020034BD3F8F800003818BF012050
:10CB8000704700BF000400200F302DE9F04F050969
:10CB900087B00591039258D08D4BD3F8F820002A26
:10CBA00000F013818A49B1F80832002B4DD191F879
:10CBB0000A324FF0FF3883F001030093D1F80031BF
:10CBC0009B1A039A48BF0F33002A15BF444601241D
:10CBD0004FF0030B4FF0000B082D4FEA23192B46A3
:10CBE00028BF082381330493794A049B039902EBFD
:10CBF00083035B68029369BBD2F82CA29C46744BFA
:10CC000000220327D3F8EC300193D44514D8019BBC
:10CC10004FEA8C0E13F80C00009B002B40D10BEB5D
:10CC20000E065B46590007FA01F101421AD04E4543
:10CC30002AD3012C28D10022954249D9009B23B93F
:10CC400019F040FF01230093CEE70025284607B0E6
:10CC5000BDE8F08F5E4BD3F82CC2029B6345EDD844
:10CC6000E246CCE7013295420BD901211B1928D4A9
:10CC700039B3042B2644D5D1A444029B6345C4D9BF
:10CC8000DAE703EB0E08D7E74E452CBF0021012160
:10CC9000621C4FF0000218BF002181F00101E5E79E
:10CCA0005B4606E001329542EBD91B1908D4042BF0
:10CCB000E2D0590007FA01F10142F3D00022F4E773
:10CCC0000099A444029B6345B6D800299DD1B3E7DF
:10CCD000039B53BB08F10104072DA4EB02042FD8DA
:10CCE00005EB08033A484FEA930300EB8501C1E9DD
:10CCF000823325D0062DC1F8103221D0052DC1F880
:10CD000014321DD0042DC1F8183219D0032DC1F8EA
:10CD10001C3205F1050113D000EB85050629C5F885
:10CD200020320DD1C0F828320AE008F1FF3328493B
:10CD300044469B08C1F82C3202EB080303F1FF388C
:10CD400004F00303A108019D580001238340685C9F
:10CD500003436B54611C884510D3022601F0030382
:10CD60001B4D88080131D5F8EC505B0088452F5CDD
:10CD700006FA03F343EA07032B54EFD2144B2701BF
:10CD8000D3F8F860039B06EB041533B11049D1F8D2
:10CD90000031AB4288BFC1F8005112010021284682
:10CDA0004FF0C2FE059B002B3FF450AF0023E2087A
:10CDB00004F00704F351064BD3F8F410012303FAEF
:10CDC00004F48B5C23438B5440E708201AF08CFF5B
:10CDD00000040020034BB3F8082212B908B1FFF792
:10CDE00017BC704700040020030701D1FFF764BCA3
:10CDF00000207047F8B5154E0446D6F8003183423E
:10CE000001D9030702D025462846F8BDFFF754FC98
:10CE100007460028F7D02046FFF77EFC0122014696
:10CE20003846FFF7B1FE05460028ECD0844207D90A
:10CE3000B6F80832002BE6D12546FFF7E9FBE3E719
:10CE40003A4621464FF048FEDEE700BF00040020CE
:10CE50002DE9F04788460646002800F0BD800029ED
:10CE600055D0624DB5F80832002B55D1D5F8F830C1
:10CE700001F10F0CD5F8F010C31A4FEA1C1C4FEA51
:10CE8000810948BF0F331B1103F1010EBEEB810F67
:10CE900080F0A980D5F8EC00012700214FEA9E041C
:10CEA0000EF0030A045D4FEA4A0A44FA0AF404F059
:10CEB0000304022C34D01CB90131CC19644530D3A1
:10CEC000BC4520D032D33944614563D222B3DA085D
:10CED000D5F8F41003F007034046895C002219419D
:10CEE00001F00101FFF750FE0446A8B13A013146B6
:10CEF0004FF0F2FDB5F8083233B93046FFF788FB42
:10CF00002046BDE8F08734462046BDE8F087374B21
:10CF1000B3F80842002CF1D000242046BDE8F08789
:10CF200001370EF1010EF145B8D8C9E703EB0C0E3D
:10CF3000A7EB0C083B444FF00309724602F0030CC8
:10CF40009408D5F8EC1001324FEA4C0C085D9A4277
:10CF500009FA0CFC20EA0C0C01F804C0EED1B8F17F
:10CF6000080FC4464FEA9E0328BF4FF0080C0CF18F
:10CF7000810C05EB8C0CDCF80420B2EB9E0FD5F88D
:10CF80002C2288BFCCF804309A42BCD23446C5F873
:10CF90002C32B9E7D8196344834211D94FF0020803
:10CFA00000F003028408D5F8EC100130520011F8AB
:10CFB00004E0834208FA02F242EA0E020A55EFD177
:10CFC000ACEB07023446002106EB071012014FF0CC
:10CFD000ABFD2046BDE8F087024601464046BDE86D
:10CFE000F047FFF7D1BD0127002169E700040020C9
:10CFF00038B50307044614D1FFF75EFB88B1154D21
:10D00000D5F8303233B90EE09A68D2B1DA68D2B1CD
:10D010001B6843B15A68002AF6D1043301201C6012
:10D0200038BD002038BD012200211020FFF7ACFDE3
:10D0300003460028F5D0D5F8302232B10022106026
:10D04000FFDE0833EAE70C33E8E7C5F830020120D9
:10D050005C6038BD0004002010B58AB00B4C03A8FA
:10D06000FFF7F2FC039A0A49DDE9043000902046FC
:10D0700001F02CF82046069C079ADDE90831CDE93D
:10D080000014044901F022F80AB010BD041406602F
:10D0900048CC05606CCC056010B50446C068FFF74D
:10D0A000A9FE03462046E360BDE81040FFF7A2BE9C
:10D0B000034610B408B304071FD1184AD2F8F84049
:10D0C00084421AD8D2F8FC20824216D982070FD1A6
:10D0D0000268134CA24219D0124CA2421AD0124933
:10D0E0008A420ED011498A420BD011498A4204D09B
:10D0F00018465DF8044BFFF77DBE18465DF8044BFB
:10D10000704718465DF8044BFFF7C6BF5DF8044B47
:10D1100000F068B85DF8044B00F00CB80004002083
:10D120001838066064410660984D0660044B06603E
:10D130009453066010B5044682B009B902B010BD20
:10D1400001394068C9B20191FFF7B2FF0346019966
:10D15000A0686360FFF7ACFF03460199A360E06835
:10D16000FFF7A6FF03462046E36002B0BDE810408B
:10D17000FFF740BEF8B504460E4638B131B1184B42
:10D18000984203D0037913F00A0501D02046F8BD78
:10D1900043F00803C0682371FFF72CFEA268E0602B
:10D1A0009AB1711ECFB200E0E06850F8353000EB64
:10D1B000C50601353BB1042B394604D07068FFF732
:10D1C00077FF7060A2689542EED32046FFF712FE0B
:10D1D000037904466FF3C30303712046F8BD00BF13
:10D1E000680400202DE9F84304460E4618B1354B7B
:10D1F000984200D011B92046BDE8F883013E80680E
:10D20000FFF7F8FD0346F6B26068A36000253146DB
:10D21000FFF7B0FF606007E031463846FFF748FF90
:10D22000E36843F808000135E0684FEA8508FFF736
:10D23000DBFDB5EB900F1AD2E36853F82500FFF73A
:10D24000D3FD0028EFD0E36853F825703B7803F056
:10D250000703022BE0D17868FFF7CCFD7860B8684F
:10D26000FFF7C8FDB860E36853F80870D4E7E068DA
:10D27000FFF7C0FD03462046E360FFF7B5FD8008D9
:10D28000B0F1040814D004F10C070025DFF8389041
:10D2900057F8043F314618463BB19A0702D11A6845
:10D2A0004A450AD0FFF704FF386001354545EFD104
:10D2B0002046BDE8F843FFF79DBDFFF75BFF3860F0
:10D2C000F3E700BFE84106601C2F0660024BC3E98C
:10D2D00002011861704700BF0004002008B5084A29
:10D2E000C31DD2E9031023F0070303448B4201D886
:10D2F000136108BD40F21631024808F023FD00BF5B
:10D300000004002030350660014488420ED241F20C
:10D31000055310F8012B03EB4313814283EA020308
:10D32000F7D1D8B2012838BF0120704705207047D7
:10D33000034B00220349C3F8DC201962704700BF89
:10D3400000040020B8F506602DE9F84F8846411822
:10D350008346884241D2034641F2055513F8012B1A
:10D3600005EB4515994285EA0205F7D1EDB2012D8D
:10D3700038BF01251A4BD3F82090B9F1000F29D0FE
:10D3800009F1100AD9F80C600AEB8606B2451CD2E6
:10D39000544601E0A64218D9274654F8040B90F8E9
:10D3A00000C0AC45F6D142784245F3D142465946D9
:10D3B00002304FF081FB0028ECD1A7EB0A07D9F827
:10D3C000040000EBA700BDE8F88FD9F80090B9F190
:10D3D000000FD5D10020BDE8F88F0525CAE700BFB2
:10D3E000000400202DE9F84306460C46FFF7ACFF89
:10D3F00000283AD14A4F04F10308D7F8DC50002D39
:10D400003ED0D7E9381208EB02038B4260D81544AE
:10D410003119C7F8E4308E4270D2B44641F2055358
:10D420001CF8012B03EB4313614583EA0203F7D198
:10D43000DBB2012B38BF0123314622466C70002637
:10D440002C442B70A81C4FF047FBA670386AD0E91B
:10D450000243A34227D25A1C0433C26040F823502F
:10D460003B6A5868DA6810440138BDE8F883024620
:10D47000D7F8E410D7F8DC00FFF73EF8C7F8DC5027
:10D48000B8F1800FC1464FF0010138BF4FF080095D
:10D490004846FFF713F80546C7F8DC0080B343465B
:10D4A000C7F8E090B4E764000121402C28BF402475
:10D4B000201D8000FFF702F860B33A6A02605368EB
:10D4C000D2681344C0E9024643603862C368C2E7C9
:10D4D000024641442846FFF70FF805460028C6D00B
:10D4E000D7F8E030D7F8DC504344C7F8E030002DDF
:10D4F000C6D0D7F8E4301D44434489E705239BE7B1
:10D5000001214046FEF7DAFF0546C7F8DC0020B1EE
:10D51000C146C4E7204608F035FC404608F032FC1E
:10D520000004002010B504464FF02FFB01462046B2
:10D53000BDE81040FFF756BF074B1B6A5A6882428E
:10D5400003D91B685A689042FBD3801A043053F801
:10D5500020305878704700BF00040020074B1B6A3A
:10D560005A68904203D21B685A689042FBD3801AD3
:10D57000043053F820000230704700BF0004002040
:10D58000084B1B6A5A68824203D91B685A6890424A
:10D59000FBD3801A043053F82000437802300B602C
:10D5A000704700BF000400202DE9F84300251E4607
:10D5B00080468946056014460D6015601D601C4B51
:10D5C0001D6A75B31B4FBD422BD0D8F8003005F152
:10D5D000100E0133C8F80030D9F80020EB6813446E
:10D5E000C9F80030E9680EEB81018E450AD2236844
:10D5F0005EF8042B92F801C071450CF1030C6344F2
:10D600002360F5D82846FFF7EFFB336818443060F5
:10D610002D680DB1BD42D8D1236818443060BDE8F3
:10D62000F8832368002018443060BDE8F88300BF09
:10D6300000040020B8F5066038B5D0E90032054690
:10D64000114499420DD9037BDB070BD401F110047F
:10D65000806824F0070408342146FEF741FF2C605F
:10D66000A86038BD0021014808F072FB3035066023
:10D6700070B504460E4611461546FFF7DDFF3146EC
:10D680002A46D4E9013018444FF034FA62682A443B
:10D69000626070BD70B50D46466804460121B54212
:10D6A00028BF3546FFF7C8FFA168681C721B0844F5
:10D6B00029444FF01FFAD4E9013001332844636054
:10D6C00070BD00BF012938BF012138B504460025CF
:10D6D00008462946C4E90005FEF7E4FE237BA06066
:10D6E00065F30003237338BD38B54B1C0C46054663
:10D6F00004D00131FFF7E6FF6C6038BD084608F042
:10D7000041FB00BF037B826043F0010310B400249F
:10D710000373C0E900145DF8044B704738B5054643
:10D720001446FFF7CFFF024BC4E9005338BD00BFDA
:10D7300071D6006010B5037B0446DB0702D50023D9
:10D74000A36010BD8068FEF7D9FE0023A36010BD62
:10D7500010B5044600211020FEF7A4FE2146044621
:10D76000FFF7B0FF204610BD10B5044678B1037B2B
:10D77000DB0704D52046BDE81040FEF7BFBE806839
:10D78000FEF7BCFE2046BDE81040FEF7B7BE10BD58
:10D7900038B5037B04460D46DB070AD40168806870
:10D7A0002944FEF79DFE2368A0601D4418442560AF
:10D7B00038BD0021014808F0CBFA00BF30350660C3
:10D7C00038B504460D46FFF737FFD4E901301D4454
:10D7D0001844656038BD00BF10B5D0E90023044689
:10D7E0009A4204D0A2680021D154A06810BD012142
:10D7F000FFF7CEFF6368A2680021D154A06810BD76
:10D8000038B504460D460121FFF716FFD4E9013271
:10D81000591C6160D55438BD7F29F8B50C460546C2
:10D820002ED9B1F5006F19D3B1F5803F31D2032164
:10D83000FFF702FFC4F38513210B04F03F0463F0EC
:10D840007F0361F01F0164F07F04D5E90126B01861
:10D85000D71C6F60B15443708470F8BD0221FFF78C
:10D86000EBFEA20904F03F04D5E9013162F03F026A
:10D8700064F07F04C8189E1C6E60CA544470F8BDE2
:10D880000121FFF7D9FED5E90132591C6960D45452
:10D89000F8BD0421FFF7D0FEC4F305314FEA944CE4
:10D8A000C4F3851204F03F0461F07F016CF00F0CAB
:10D8B00062F07F0264F07F04D5E901063318071D8A
:10D8C0006F6006F800C059709A70DC70F8BD00BF38
:10D8D00010B5044682B0084601914FF056F90199FF
:10D8E0000246204602B0BDE81040FFF7C1BE00BFAF
:10D8F00010B51446FFF7CEFE047010BD10B51446E7
:10D90000FFF7C8FE047010BD43688B422CBF5B1A42
:10D9100000234360704700BF38B51546426804468F
:10D920000B468A4203D929448A4201D8436038BD54
:10D930008068521A014418444FF0DCF86268521BA8
:10D94000626038BD0846114626F004BB70B5054636
:10D9500008460E464FF019F9044620B102466B689E
:10D96000314628689847204670BD00BF2DE9F84F22
:10D970008A469DF8281091460B9A11F0DF0F054654
:10D98000A2EB09023DD030290AA9264E0EBF10276E
:10D990000E46012713F0800839D0002A9046B8BF00
:10D9A00002F10108A2EB68044FEA6808B8F1000F21
:10D9B00032DDC3465F453A466B683146A8BF5A46DA
:10D9C0002868ABEB020B9847BBF1000FF2DCB9F112
:10D9D000000F05D04A465146C844D5E90003984790
:10D9E000002C0BDDA044A7423A466B683146A8BF25
:10D9F00022462868A41A9847002CF4DC4046BDE86B
:10DA0000F88F13F08008084E4FF01007C5D113F0BF
:10DA1000010404D01446DAE74FF00008D7E7904637
:10DA2000C4E700BF201406600C1406602DE9F04F17
:10DA3000064689B000209C469DF85070139B159DAA
:10DA40008DF80F001AB3814249DB9A075AD413F0BC
:10DA500004021CD0202292468DF80F20D1B930222A
:10DA60000DF11F048DF81F2013F040082DD0BAF1DE
:10DA7000000F3AD1D04608AA304621460195121B24
:10DA80000097FFF773FF404409B0BDE8F08F92465E
:10DA90000029E4D0129A08AC0DF11009A2F10A0B8A
:10DAA0008846B1FBFCFE0CFB1E127146092A02F1EE
:10DAB000300088BF0BEB0200E04504F8010DD3D322
:10DAC0004C45EDD813F04008D1D1BAF1000FD2D0B7
:10DAD00004AA9442CFD904F801AC013CCBE72D2233
:10DAE000494292468DF80F20D4E701220DF10F0133
:10DAF000304600970192013D1393FFF737FF139BC8
:10DB00008046B8E72B2292468DF80F20A6E700BF8B
:10DB10002DE9F04F0F4691B080461C46F9071A9D3B
:10DB20009DF86CB00DD4BB0703D1A14B3968994265
:10DB300007D03846059209F077FC059A400040F07E
:10DB4000010715F0810F03D1BBF1300F00F0CD803C
:10DB5000384605920CF040FF0028059A77DBAE07A7
:10DB600073D52B23E9060DF121060DF1200A8DF85E
:10DB7000203071D4E3B2A6EB0A0115F0200F4FF06C
:10DB800000041D9805914FF0100134700CAE0A91FD
:10DB90000CBF21462C2101280B9409966DDD0092C3
:10DBA00009A80BAA01948DF81F40CDE902313B462C
:10DBB0000AA90CF0C9FC037807462D2B72D18DF809
:10DBC0001F3001370B9B1D9A013B93420B93B8BF4B
:10DBD0001346059A013313441C9A9A4270DC25F0CF
:10DBE00001054FF0000945F040054C464FF0300B61
:10DBF0009DF81F30002B40F0A180059B002B40F0CA
:10DC0000AE801D9B012B4ADD1D9B39460B9A404679
:10DC1000CDE900B32B46FFF7A9FE0444B9F1000F8C
:10DC20000AD0002320224046624900921A46CDF8CD
:10DC30000490FFF79BFE04440998B04201D0FEF720
:10DC40005DFC204611B0BDE8F08F680756D40DF199
:10DC5000200A5646E9068DD5022A3DD0082A00F052
:10DC60008C80102AE3B286D13146302001F8020BB5
:10DC700003F1170070700E467DE715F040098DF82E
:10DC80001F40CDE9023140F085803B460AA909A832
:10DC90004C46CDE9002A0BAA0CF056FC07461C9B0B
:10DCA0001D93B1E71D9A0B9B9342B8BF13469DF895
:10DCB0001F20002A8DD1059A13441C9A9A428EDDAA
:10DCC00015F0010922D025F001051C9A0024A2EBD1
:10DCD000030945F0400589E731463020E3B201F8F9
:10DCE000020B581C70700E4645E7DDE91C318B4273
:10DCF000B8BF0B461C9300231D9329E720230DF189
:10DD000021060DEB030A8DF82030A3E71C9A25F0BD
:10DD1000010528494046D31A4A4645F0400501937B
:10DD2000202300934B46FFF721FE04465EE78DF863
:10DD30001F3001370B9BA146013B0B931C9B01221B
:10DD40000DF11F014046013B1C930023CDE9003239
:10DD5000FFF70CFE059B0444002B3FF452AF1C9BC5
:10DD60000120059A51469B1A1C930023CDE90030EF
:10DD70004046FFF7FBFD044443E730233370AB0517
:10DD800001D40136F6E6E3B2023603F10E0106F8DD
:10DD9000011CF0E63B4600920AA90BAA09A80194CF
:10DDA0000CF0D2FB037807462D2BC0D0A1461FE70D
:10DDB000703C0660387007602DE9F04314468BB064
:10DDC0000A460746A1079846129E1BD414F0040F7A
:10DDD0000CBF0023202300932021139B02A806F0F0
:10DDE000A5FFE305054602D5431C1F2B18D914F0E7
:10DDF000400909D09DF8083002A92F2B1CD94FF0FB
:10DE0000000902E02B23E6E702A923462A4638460A
:10DE1000CDE90086FFF7AAFD48440BB0BDE8F083CA
:10DE20000AAA1544252205F8202C0AAA1D461A44E0
:10DE3000002302F8203CDAE7002301223846013EA5
:10DE4000013DCDE90032FFF791FD0DF10901814659
:10DE5000DBE700BF2DE9F04F4FF0000A89B08346A1
:10DE600090460B78252B12D0002B00F085800C46B5
:10DE7000254614F8013F0BB1252BF9D1A14208D258
:10DE8000621ADBE90003924498476B782146002B25
:10DE900072D04B784C1C002B00F007814FF020090A
:10DEA00000260DE02B2B15D0202B16D0212B17D0C0
:10DEB000302B18D146F04006994614F8013F3BB18B
:10DEC0002D2BEFD114F8013F46F00106002BF7D1BE
:10DED00000251CE046F00206EFE746F00406ECE7FA
:10DEE00046F00806E9E723780025A3F13002092A65
:10DEF0000AD805EB850503EB450514F8013FA3F1AE
:10DF00003002303D092AF4D92E2B00F0A980277861
:10DF10004FF0FF326C2F2BD077B3A7F14503332B93
:10DF20001BD8DFE803F02D2D2D1A1A1A1A1A1A1A07
:10DF30001A431A1A1A1A1A1A1A511A1A1A1A1A1AE1
:10DF40001A1A1A618F8B2D2D2D1A1A1A1A1A1A1ACB
:10DF50001A437F1A731A6F1A1A51DBF80430012220
:10DF60002146DBF800000AF1010A9847611C78E7B6
:10DF700067780134002FD0D1504609B0BDE8F08F4A
:10DF800008F10708059228F00708F8E802014EF0AA
:10DF9000BDFB059A00EE100A4B4639465846CDE9BE
:10DFA00000523246FFF708FF8244DFE7612010236A
:10DFB000002258F8041BCDE90006CDE90295584629
:10DFC000FFF734FD8244D1E7A7F1170358F8041B8B
:10DFD00000225846DBB2CDE90295CDE90036102388
:10DFE000FFF724FD8244C1E758F8043BCDE90095D2
:10DFF000002B52D03346042232495846FFF7B6FC74
:10E000008244B3E761200A230022D2E7531C58F868
:10E01000041B4FD033465846CDE90095FFF7A6FCC8
:10E020008244A3E707A958F8040B0592FFF7A8FA62
:10E03000059A0146501CEDD1079AEBE761200A23AF
:10E040000122B6E758F8040B3346012207A98DF8E0
:10E050001C005846CDE90095FFF788FC824485E70F
:10E0600067782A2F06D158F8042B0234277822EA41
:10E07000E2724FE7A7F1300301340022092B3FF68B
:10E0800049AF02EB820207EB420214F8017FA7F1CD
:10E090003003303A092BF4D93CE7334605220A49CC
:10E0A0005846FFF763FC824460E71E464FF02009A4
:10E0B00000252CE7084605914EF067FD05990246BC
:10E0C000A8E700BFF4130660FC1306600EB400B5A9
:10E0D00082B003AA52F8041B0192FFF7BBFE02B004
:10E0E0005DF804EB03B0704790F900100246037826
:10E0F00000291ADA03F07F005B0605D5402320EAE9
:10E1000003005B081842FAD1517801F0C003802B5C
:10E110000CD1531C01F03F0C13F8011F01F0C00299
:10E120004CEA8010802AF5D070471846704700BF2F
:10E130004378013003F0C003802B05D110F8013F74
:10E1400003F0C003802BF9D0704700BF02460020C7
:10E15000914209D911F8013D03F0C003802B18BF8B
:10E1600001308A42F6D17047704700BF01448842AF
:10E170000CD2421E0139002012F8013F03F0C00307
:10E18000802B18BF01308A42F6D1704700207047BB
:10E190007F2804D8034B185CC0F340007047002070
:10E1A000704700BF341406607F2804D8034B185C06
:10E1B000C0F3C00070470020704700BF34140660F1
:10E1C0007F2804D8034B185CC0F380007047002000
:10E1D000704700BF341406607F2804D8034B185CD6
:10E1E000C0F3801070470020704700BF34140660F1
:10E1F0007F2803460BD8074A125C12F00C0F14BF9D
:10E20000012000205F2B08BF40F001007047002074
:10E21000704700BF341406607F2804D8034B185C95
:10E22000C0F3001070470020704700BF3414066030
:10E230007F2804D8034B185CC0F3401070470020BF
:10E24000704700BF341406607F2804D8024B1B5C63
:10E25000DB0648BF20307047341406607F2804D89E
:10E26000024B1B5C9B0648BF203870473414066085
:10E270003038092802D920F020000738704700BF45
:10E28000014488421DD200224FF0E50C06E01B0637
:10E2900029D50130531E8142DAB220D90378002AF1
:10E2A000F5D1BF2B0FD81A061DD4421C914208D9B4
:10E2B000104612F8013BBF2B05D81B0613D4914220
:10E2C000F6D101207047F72B0DD8DB08013003F0A1
:10E2D000060381424CFA03F303F00302DED8B2FADC
:10E2E00082F0400970470020704700BFB2EB131F57
:10E2F00070B506464FEA131420D901EB4405141BF0
:10E3000003F00F0184462346AE46012B03F1FF3391
:10E3100009D05EF8022B012B03F1FF3322FA01F240
:10E320002CF8022BF5D1601E35F8103023FA01F1DC
:10E3300026F81010002918BF204670BD002070BDBF
:10E340002DE9F041069FD21BAFB3A3F1020E8E1E42
:10E35000BC460546002436F8023FBCF1010C3EF8ED
:10E36000028F434423444FEA134425F8023BF2D181
:10E3700001EB470100EB470772B1A1F1020CBE4669
:10E3800011463CF8023F013923444FEA13442EF86A
:10E39000023BF6D107EB420744B1012327F8023BC9
:10E3A0003F1A47FA03F21046BDE8F0813F1A7A108F
:10E3B0001046BDE8F081002AF5D03C460746DCE770
:10E3C0002DE9F041069FD21BEFB39C1E8E1EBE4668
:10E3D00005464FF0000C36F8023FBEF1010E34F84E
:10E3E000028F6344A3EB08034FEA234C25F8023B5A
:10E3F000F1D101EB470100EB47050AB3A1F1020E91
:10E400002C4611463EF8023F013963444FEA234C43
:10E4100024F8023BF6D1531E05EB420205EB430301
:10E4200003E01A4633F8021929B99842F9D9101AAB
:10E430004010BDE8F0810232101A4010BDE8F081B2
:10E44000AB1E2A46F1E70546BC46D6E7022938B599
:10E4500038BF0221044680680D4618B12368B1EB2D
:10E46000930F07D96900FEF73BF82368A06065F3B6
:10E470009F03236038BD00BF38B5054600210C203E
:10E48000FEF710F82B780446002103F00102037810
:10E4900023F003031343037028682368C0F39D002F
:10E4A00060F39F03400023606B686360FDF7FAFF31
:10E4B000A0602A68A968C2F39D0252004EF00CFBCE
:10E4C000204638BD00EB410302EB410219B910E0D0
:10E4D0000CD101390CD033F8020D32F802CDA0EB8B
:10E4E0000C000028F4DA4FF0FF307047012070472D
:10E4F00070470846704700BF10B504468068FDF7B6
:10E50000FDFF2046BDE81040FDF7F8BF38B50C46CA
:10E5100002210546FFF79AFF002C10DB2146002060
:10E520002A78002360F300022A7000E06B68581C10
:10E53000AA68686022F81310090CF7D138BD61424F
:10E540000120EDE70023C0E900338360704700BF7E
:10E550000022C0E90022826001B97047FFF7D6BFF0
:10E560009200816042F0020202600022426003B920
:10E5700070471946FFF7CABF10B103789B0700D553
:10E5800070478068FDF7BABF38B504460D46496844
:10E59000FFF75CFF2A782378A06862F300032370FA
:10E5A0006A6862605200A968BDE838404EF094BACB
:10E5B000F8B51D46042106469DF818701446FFF76D
:10E5C00045FF002D317816DAAFB1624241F001010A
:10E5D00065EB45033170002100E071684D1CB468A3
:10E5E000100C756024F8112040EA03421B0C52EA1B
:10E5F0000301F2D1F8BD6FF30001002022462B4643
:10E60000317054EA05017060E5D1F8BD2DE9F041A3
:10E6100082B0027805468DED010A019CE30F63F399
:10E620000002C4F30F4313F4FF4302702BD0B3F581
:10E63000FF4F28D0C4F3C752A2F17F03002B22DB87
:10E6400047D0B2F16F01C4F3160448BFA2F16001D4
:10E65000162B44F400044FEA211719DCC3F1170309
:10E660003946DC40FFF7F2FE00236F609F420CD07A
:10E670005B007900AA68D4520233240C9942F9D184
:10E6800002B0BDE8F08100236B6002B0BDE8F0810C
:10E690000933394603F00F08B2F1960348BFA2F1DF
:10E6A00087031E11FFF7D2FE6F6026B172000021B2
:10E6B000A8684EF039FAB8F1000F10D004FA08F249
:10E6C000AB68C8F1100823F81620731C24FA08F46C
:10E6D000CCE7012102B0BDE8F041FFF717BF334698
:10E6E000C4E700BF2DE9F8438846C2F35B01054645
:10E6F0001C46013108EB0206089FFFF7A7FE2B78A6
:10E700000020B04564F3000368602B702ED2C6462B
:10E71000B9B272460EF1010E1378A3F13000092848
:10E7200005D9A3F14100192822D8A3F13700B84236
:10E7300026D2D5E901493CB3A4464A461388BCF128
:10E74000010C01FB03034FEA134022F8023BF5D111
:10E7500009EB440408B124F8020BA4EB0904764544
:10E760004FEA64046C60D4D1A6EB0800BDE8F883DE
:10E77000A3F16100192803D8A3F15700B842D8D3F8
:10E78000A2EB0800BDE8F8834C46E3E72DE9F04131
:10E79000074614461D4600294DD0531E4FF0FF3644
:10E7A0001D44E10038460F310909FFF74FFE3B7861
:10E7B00000206FF3000378603B70002C3DD00146D1
:10E7C00080460F291CDC4FF0000C95F800E0013C5E
:10E7D0000B4635440EFA01FE01F108014EEA0C0C1D
:10E7E0001FFA8CFC01D00F29EFDD421CA3F10801B8
:10E7F000BB687A6023F810C04CB10F297868E2DD5D
:10E80000BB68421C10397A6023F81080F5E77B68FA
:10E810005B00023BB868C31802D311E0984205D8E8
:10E820001A4633F802190029F8D00232131A5B1085
:10E830007B60BDE8F0810126B3E76FF00103E9E7F3
:10E840009A1CF3E738B5446884460CB94868A8B107
:10E850000B789CF8005003F0010305F00100181A32
:10E860000CD14B689C420AD30CD88A682146DCF84C
:10E870000800FFF727FEEB0748BF404238BD4FF0C6
:10E88000FF30F8E70120F6E7884210B5044601D0D2
:10E89000FFF77AFE23786FF30003237010BD00BFEB
:10E8A000884210B5044601D0FFF76EFE2378C3F30B
:10E8B0000002C2F1010262F30003237010BD00BF29
:10E8C000884210B5044684B001D0FFF75DFE62684F
:10E8D0004AB32378D90715D4511C2046FFF7B6FD5B
:10E8E000A16801200DF10E036268ADF80E000090E2
:10E8F0000846FFF725FD2378606043F0010323708D
:10E9000004B010BD18460123A1686FF30000009306
:10E91000ADF80E300DF10E0320700846FFF750FDE4
:10E92000606004B010BD01212046FFF78FFD012279
:10E93000A3681A80237862601343237004B010BD6B
:10E940002DE9F0470E4607464968144602B129B939
:10E9500031463846BDE8F047FFF716BE02F10F0911
:10E960006FF0004801EB1911FFF770FD14F00F0272
:10E970004FEA1919BB6818BFC2F11002D6E901C0ED
:10E9800009EB0C05A84403EB48044FEA4808BCF126
:10E99000000F35D000EB4C006146A646002330F84E
:10E9A00002AD01394AEA030323FA02FA4FEA0343AC
:10E9B0002EF802A9F3D1D340CCEBCC7C9BB204EB74
:10E9C0004C042380C9F1010309F1FF32002104EB5B
:10E9D0004304520020464EF0A7F84DB108F102035F
:10E9E000234401E0013D03D033F8022D002AF9D081
:10E9F0003B787D60327862F300033B70BDE8F087BE
:10EA00006346DEE72DE9F0410C4684B006464968CE
:10EA100017461AB1B1FA81F56D0931B92146304670
:10EA200004B0BDE8F041FFF7AFBDFFF70FFD3B4677
:10EA3000B068D4E90121FFF759FC3378706022787F
:10EA400062F300033370DB0717D55FEA171E6268B5
:10EA5000ADF80E500FD072B1D4F808809645F44648
:10EA6000294628BF9446A8F1020333F8025F01311A
:10EA7000CDB96145F9D3964502D304B0BDE8F08124
:10EA8000A36807F00F0733F81E100123BB40013BBA
:10EA90001942F2D00123ADF80E3098B90123B268C3
:10EAA00013807360E9E701239645ADF80E30F4D288
:10EAB00007F00F0738F81E2003FA07F7013F3A4224
:10EAC000EBD0E7E7B168012402460DF10E030846DA
:10EAD0000094FFF735FC7060CFE700BF2DE9F041EF
:10EAE0004F6882B0D2F804800C461546064647456A
:10EAF00021D306D892683946A068FFF7E3FC0028C6
:10EB000019DB23782A785340DB0719D4791C304667
:10EB1000FFF79CFC6868AB686268A1680090B06809
:10EB2000FFF70EFC70602278337862F300033370D5
:10EB300002B0BDE8F081234647462C461D46E0E77B
:10EB400039463046FFF782FC6868AB686268A168A6
:10EB50000090B068FFF734FC7060E4E72DE9F04105
:10EB60004F6882B0D2F804800C46154606464745E9
:10EB70000AD306D892683946A068FFF7A3FC00289C
:10EB800002DB4FF0000805E0234647462C464FF0D5
:10EB900001081D4623782A785340DB071AD5791CD3
:10EBA0003046FFF753FCD5E90103D4E90121009079
:10EBB000B068FFF7C5FB70602378B8F1000F1AD07A
:10EBC000DB4303F00103327863F30002327002B0DA
:10EBD000BDE8F08139463046FFF738FCD5E901033E
:10EBE000D4E901210090B068FFF7EAFB7060237858
:10EBF000B8F1000FE4D103F00103E4E72DE9F04F91
:10EC000087B00B46039111460292049018465A6849
:10EC10004B689A4202D31346CDE90201029A127858
:10EC2000D20700F18B80039A117801F00101049C56
:10EC300019442046FFF70AFC029B039A93F800C090
:10EC400011789D6858685368D2F808A01A468CEA73
:10EC50000103D4F80890DB075FD50CF0010C01F03C
:10EC60000101CCF1000BC1F100081FFA8BFB1FFA68
:10EC700088F800284DD0002601964F46CDF8149014
:10EC8000023D0446914635F8023F013CD6464246D5
:10EC900083EA0B03634409EB040CACEB000C644502
:10ECA00004D33EF8022B82EA0802F24611444FEAEE
:10ECB000134C019A0B40090C534016FA83F31E0CB7
:10ECC00027F8023B002CDED1DDF8149009EB400060
:10ECD00006B30346012223F8022B03E0034630F873
:10ECE00002296ABB8145F9D9A3EB09030498039A69
:10ECF0005B1001784360029B12781B78C2F300021C
:10ED0000C3F30003134063F30001017007B0BDE8D3
:10ED1000F08F484603460238E4E71CF0010C01F08E
:10ED200001019ED0C1F100081FFA88F850B14FF6DA
:10ED3000FF7B0126CDF804B0B4469EE7012176E7BB
:10ED40000233D1E74846C4E72DE9F04F87B00B46C0
:10ED5000039111460292049018465A684B689A42F1
:10ED600002D31346CDE90201029A1278D2077FD46A
:10ED7000039A117801F00101049C19442046FFF721
:10ED800065FB029BD4F8089093F800C09D685C680E
:10ED90001CF0010F039B0CF0010CD3E9012A019236
:10EDA0005ED1197841F3000301F001069BB23146B0
:10EDB000CCF1000BC1F100081FFA8BFB1FFA88F899
:10EDC000002C59D0023D4F46CDF81490204699466C
:10EDD0000095009A0138019DD64632F8023F83EA39
:10EDE0000B0300924246634405EB000CACEB040CB1
:10EDF000604504D33EF8022B82EA0802F246114431
:10EE00004FEA134C0B43090C83EA090316FA83F308
:10EE10001E0C27F8023B0028DBD1DDF81490631E9E
:10EE200009EB440409EB430303E01C4633F80229D1
:10EE300002BB9945F9D9A4EB09040498029B64101C
:10EE4000039A017844601B781278C3F30003C2F37D
:10EE50000002134363F30001017007B0BDE8F08FB7
:10EE6000039B012619784FF6FF7301F001019FE71C
:10EE7000012181E70234DEE7A9F102034C46D8E71D
:10EE80002DE9F04F85B00B4601911146009202909A
:10EE900018465A684B689A4202D31346CDE90001DE
:10EEA000009A1278D2076AD4019A117801F0010110
:10EEB000029C19442046FFF7C9FA009B019A1D786D
:10EEC0001178EE43D4F808904D405C68C9439F68C0
:10EED00006F0010605F0010501F00101D2F808A0D5
:10EEE0005368002C4FD0C846CDF80C90023F204606
:10EEF0004FF6FF7B9946013837F8023FD6464FF66A
:10EF0000FF7209EB000C5B44ACEB040C334460452E
:10EF100003D33EF8022B5A44F24611441E0C4B40D8
:10EF2000090C15FA83F31D0C28F8023B0028E2D1E6
:10EF3000DDF80C9009EB4404E5B9A31E03E01C4680
:10EF400033F80229EAB99945F9D9A4EB09040298E2
:10EF5000009B6410019A017844601B781278C3F317
:10EF60000003C2F30002534063F30001017005B0D7
:10EF7000BDE8F08F0122234624F8022BE3E70121AC
:10EF800096E70234E1E74C46D6E700BF2DE9F04FA3
:10EF900087B04B680F4606460192002B66D0516839
:10EFA000002963D087426BD0019A824273D000223D
:10EFB000029219443046FFF749FA33680021B068DD
:10EFC000C3F39D035A004DF0AFFD019AB368D2F828
:10EFD0000490D2F808800393D7E901B1B9F1000F8A
:10EFE00032D003EB4B00CA46C1468846CDE90467E0
:10EFF0005F469B46002F40D0ABF1020439464546A0
:10F00000002335F8026B0139B9F800C034F8022F3B
:10F010000CFB0622134423804FEA1343F1D104462C
:10F020004BB3851C03802C464DF006FEBAF1010A55
:10F030000BF1020B09F102092846DBD1039BE41A0C
:10F04000DDE904674FEA6409019AC6F80490117873
:10F050003B7832784B4063F30002029B32703BB145
:10F06000184607B0BDE8F04FFFF746BA00237360BB
:10F0700007B0BDE8F08F851CD6E7851C5C46D3E75A
:10F08000FFF7FAF9019B0746B34243680AD0019A99
:10F09000029051688DE7FFF7EFF97B6841680190B6
:10F0A000029086E71946CDE9010082E770B54B680A
:10F0B000064614466BB31378DA072AD46368A3B301
:10F0C0000846FFF7D9F905462046FFF7D5F904466B
:10F0D00001213046FFF71AFA626872B91CE0012379
:10F0E0000846FFF703F903462A4629462846636087
:10F0F00093B1FFF74BFF626872B1A1680B88DB0721
:10F10000EDD52A4631463046FFF740FFD4E90121CC
:10F11000E5E70023736070BD15B12846FFF7ECF9F1
:10F120002046BDE87040FFF7E7B90121BDE8704017
:10F13000FFF7ECB92DE9F04F8FB00E4614461F468D
:10F140000191054651680992013107930590FFF737
:10F150007DF963680021A86801335A004DF0E4FC92
:10F16000002330466B6061680131FFF76FF921467B
:10F170003046FFF709FA7B683A4677680293BB424C
:10F1800000F23681B0689268AB68069003920893EB
:10F1900008D33946FFF796F9002800F02D81013099
:10F1A00000F02681029B6FF00046039A00241E4463
:10F1B00032F91630750032F81620002B05DB5300AB
:10F1C00001341904A4B29AB2F9D506990023019822
:10F1D00021F81730426801324260084601EB4201D3
:10F1E000884213D2C4F1100701468446DDF804E0DA
:10F1F0000A8802FA04F0FA40034321F8023B93B272
:10F20000DEF804200CEB42008142F1D3039931F87F
:10F21000163003FA04F0029B012B049007D94B1916
:10F22000C4F1100133F8023CCB4018430490029E15
:10F230006FF000410598931B0A4443600B44069904
:10F2400001EB4200089A02EB43030093019B5B68C9
:10F250009E4270D2451B039B0230A5F10208A3F128
:10F26000020B30F802CD0021049B30F8027C80456F
:10F2700047EA0C47B7FBF3F733D2039B46468C466D
:10F28000A3F102090BE05B1A8A45A3EB05031AD927
:10F290009AB2B0424FF0000126F8022C1FD939F87B
:10F2A000022F36F8023BA24042EA1C4C1FFA8CF5B2
:10F2B00007FB05F56A189D42A3EB050AA2EB030EB6
:10F2C000A3EB0202DFD31FFA8EF192B2003926F8C7
:10F2D000022C18BF0121B04201EB1E41DFD8B0F86B
:10F2E00000C0B1EB0C0C19D0804569D200235E46FA
:10F2F00041461D4636F8022FA24042EA15450A88CB
:10F3000012FA85F2134421F8023B81424FEA13437B
:10F31000F0D3BCEB030C07F1FF37E5D1009BA8F15C
:10F320000208019A23F8027900935368013B536065
:10F33000029A9A4295D36FF000421A44069B03EB5F
:10F34000420293420DD8C4F110050020069E138896
:10F3500043FA04F1AB40014398B222F802199642F5
:10F36000F5D9059B5B685BB1089A059802EB4302EF
:10F3700001E0436023B132F8021D013B0029F8D0BF
:10F380000198436853B1069A02EB430201E04360DF
:10F3900023B132F8021D013B0029F8D0099B079ADE
:10F3A0001B7812785340DB0707D5059A137843F092
:10F3B00001031370019B5B6823B90FB0BDE8F08FA8
:10F3C000013F91E700230BA84FF0FF310D93CDE9EA
:10F3D0000B33FFF79BF805990BAA0846FFF77EFB56
:10F3E0000199079A0846FFF779FB0FB0BDE8F08F47
:10F3F0000023059A5360D1E7019B089A58600123C6
:10F400001380059A5360C9E72DE9F04398464B688D
:10F4100085B00C4607461546002B49D01378DA070D
:10F4200046D4D8F80430012B04D1D8F808301B8812
:10F43000012B3DD001213846FFF768F86B68002B9F
:10F4400038D020460DF10409FFF716F80446284687
:10F45000FFF712F8002306460193CDE90233426814
:10F46000A2B92AE008460123FEF740FF05462246DE
:10F4700021462046756005B3FFF788FD22464346C6
:10F4800021464846FFF756FE7268B2B1B1680B8854
:10F49000DB07E7D5224639463846FFF777FD3A467F
:10F4A000394643464846FFF745FED6E90121D9E7EC
:10F4B00000237B6005B0BDE8F0834846FFF75CF8A9
:10F4C00014B12046FFF718F83046FFF715F805B0DD
:10F4D000BDE8F083D0E901318446002001EB43030D
:10F4E000994205D233F8022D994242EA0040F9D3FD
:10F4F0009CF80030DB0748BF4042704710B4D0E9A9
:10F500000134002204EB43039C4203D308E0B2F52C
:10F51000004F0ED233F802CD9C424CEA0242F6D3A1
:10F52000037801205DF8044BDB0748BF52420A60B4
:10F53000704700205DF8044B704700BF2DE9F04F85
:10F54000C9B303EB020CD0E9019AB9F1000F29D03D
:10F550004FF0000E03EB02084FF0010B74463AF82F
:10F56000022B103442EA0E4E06781FFA8EF20CF18E
:10F57000FF37654616F0010F6FEA020604D05BFA0A
:10F5800086F6B2B2C6F3072B71B1BB420CF8012C60
:10F59000BC4607D0083C4FEA1E2E072CE4DCB9F12C
:10F5A0000109DCD1BDE8F08F05F8012B4545AC46DB
:10F5B000F0D1BDE8F08F9C46C5E700BFD0E901322D
:10F5C0009FED0C0A02EB43039A420DD29FED0A7A9B
:10F5D00033F8021D07EE901A9A42F8EEE77AE0EE51
:10F5E000077AB0EE670AF3D30378DB0748BFB1EEC2
:10F5F000400A704700000000000080472DE9F84FE6
:10F600001646426880460C469A469DF82890AAB94C
:10F61000002E00F09E8033780B992BB101F8013B4E
:10F6200016F8013F002BF9D10846302200230A705A
:10F6300000F8013F0B9BC01ABDE8F88F4FEA420B60
:10F6400000215846FCF72EFF05465A46D8F8081008
:10F650004DF042FA05EB0B01DDF82CC0AAF13A0E91
:10F66000881E6246A84225D382460023BAF800B01D
:10F670004BEA0343B3FBF4FB2AF802B9554504FBFC
:10F680001B33F3D930339246392B88BF7344A942D8
:10F69000DBB20AF8013B13D92B4601E099420FD99E
:10F6A00033F8027B002FF9D0B9F1000F41D1524657
:10F6B000A842D9D230239246A9420AF8013BEBD89E
:10F6C000B9F1000F08D0AAEB0C0CBCF1030F03D169
:10F6D00002F1020A82F801902846FCF70FFF76B18A
:10F6E00030464DF052FA33189E4208D20AF1FF32EA
:10F6F00013F8011D9E4202F8011FF9D1824498F8C7
:10F700000030DB0720D40AF1FF330B9A9A4208D26B
:10F710000B9A1178187802F8010B03F801199A4234
:10F72000F7D300230B9A8AF80030AAEB0200BDE859
:10F73000F88FAAEB0C03032BB9D102F1020A82F86D
:10F740000190D4465246B3E72D2253460AF8012BC6
:10F75000DBE70B9968E700BFD0E90232934203D29E
:10F760005A1C8260187870474FF0FF30704700BF16
:10F7700010B50368044623B92046BDE81040FCF7E5
:10F78000BDBE4068FCF7BAFE2046BDE81040FCF75D
:10F79000B5BE00BFF8B50E46154604460021102040
:10F7A0001F463544FCF77EFE044A054B0760C560E2
:10F7B000C0E90166C4E90002A360F8BD59F7006022
:10F7C00071F7006010B40369272B18BF222B0CBF00
:10F7D0000122002203D110465DF8044B7047A3F1CB
:10F7E00062011329F7D8124C24FA01F1C907F2D5A6
:10F7F0004169272918BF22290CBF01220022EAD023
:10F80000722B10D0662B01D0622BE4D17229E2D189
:10F8100082695DF8044B272A18BF222A0CBF0122F7
:10F820000022104670476629F2D06229D3D1EFE753
:10F830001100090010B5036904460A2B49D0092BB1
:10F84000C36A04BF073323F007030133C36294F88C
:10F850007020D4E90513C4E904137AB1B4F8722016
:10F86000616E8A423BD0501CA16EA4F872008A5C83
:10F87000A2610D2B23D02369ABB110BDD4E90103E4
:10F8800098476369A0610D2B1AD001301CD16369C0
:10F890005A1C19D00A2B17D00A2294F87030A26192
:10F8A000002BE8D110BDD4E90701626A84F87030FA
:10F8B000A2616366A4F87230C4E9040110BDA069B6
:10F8C0000A23984263610DD094F87030002BE9D080
:10F8D000D1E7836A01221344C0E90A32B7E7002264
:10F8E000A261C6E7D4E901039847A061CDE700BF54
:10F8F00070B504460D4600690026431C0BD00A284B
:10F900000BD10DB1636B33B120460126FFF792FF97
:10F910002069431CF3D1304670BDFEF739FC50B965
:10F920002369232B0CD05C2BF5D163690A2BF2D110
:10F930002046FFF77FFF2046FFF77CFF2069DCE7CA
:10F940002046FFF777FF20690A28D6D00130F7D18B
:10F95000304670BD2DE9F04F2DED028B426E89B01F
:10F96000834622B190F87020002A00F0E880002140
:10F970005846CBF85410FFF7BBFFDBF83030DBE91B
:10F980000A12002B0793CBE91112C0F2CD800BD0E5
:10F99000079B0B215A1E8BF84C10CBF8302009B076
:10F9A000BDEC028BBDE8F08F30B3DBF8341019BB2F
:10F9B000DBF83C506FF00041DBF840000A2429449A
:10F9C0008BF84C40541E30F8112000EB410194425A
:10F9D000E5D000F25E830BD26A1E531BCBF83C20AD
:10F9E000013ACBF8303031F8023D9C42F5D3D6D005
:10F9F00002228BF84C20D2E7DBF81090B9F1FF3FE0
:10FA000000F0C7805846FFF7DDFE0290002800F0A6
:10FA100080824C460022DA46752C8BF84C20CDE9CA
:10FA2000052279D0622C00F0DB81722C00F0F58188
:10FA3000662C00F009820027029B10210593039792
:10FA4000DDE90625002AAAD19AF84C20002A40F0C8
:10FA500092818AF84C10002D40F09381222C504660
:10FA600018BF2724FFF7E6FEDAF81010A14200F0D5
:10FA700090810126481C00F0A782731E18BF012345
:10FA800001930025DDF808900AF15008AB460A29D9
:10FA900001D1019B43B3B3452BD2A14200F0888032
:10FAA00027B17B2900F08C817D2966D0002D74D090
:10FAB000232900F0F4815C2900F081803A290CBFF1
:10FAC0004FF0000909F00109B9F1000F40F0698118
:10FAD0004046FDF7A1FE4FF0000B5046FFF7AAFE8F
:10FAE000DAF81010481CD2D1B34502D203228AF8AA
:10FAF0004C2059460AF15000FDF706FF01215046FF
:10FB0000FFF7F6FE5046FFF75DFE00283FF447AFD3
:10FB1000DAF81040752C85D10027029B069A012542
:10FB20001021059303978DE70C2101338BF84C10BE
:10FB3000CBF8303009B0BDEC028BBDE8F08F292145
:10FB40006030FDF769FE0124DBF86820DBF818104F
:10FB50008BF87040DBE90450CBE90801CBF81C506E
:10FB600003211078CBF810005078CBF8140092786D
:10FB7000ABF87210CBF81820F9E64046FDF74CFEC2
:10FB8000002D40F0758100255046FFF753FEAB462F
:10FB9000A6E700228BF84C2001E75C2913D0AB4686
:10FBA000C9B24046FDF72CFE5046FFF743FE97E7EB
:10FBB000214640460BF1010BFDF72EFEF4E704222F
:10FBC0008AF84C209AE750460491FFF733FEDAF8A2
:10FBD0001030DDE90321002A40F00E81A3F10A0272
:10FBE0006E2A70D8DFE812F0AD006F006F006F0072
:10FBF0006F006F006F006F006F006F006F006F008D
:10FC00006F006F006F006F006F006F006F006F007C
:10FC10006F006F006F006F0012016F006F006F00C8
:10FC20006F0012016F006F006F006F006F006F00B8
:10FC30006F006F006F006F006F006F006F006F004C
:10FC40006F006F006F006F006F006F006F006F003C
:10FC50006F006F006F006F006F006F006F006F002C
:10FC60006F006F006F006F006F006F006F006F001C
:10FC70008A016F006F006F006F006F006F007C00E3
:10FC80006F006F006F006F006F006F0012016F0058
:10FC90006F006F006F00880186016F006F006F00BA
:10FCA000BF006F006F006F006F006F006F006F008C
:10FCB000B0006F006F006F00C5006F00C3007C00D4
:10FCC000C1006F008301A3F1300BBBF1070F40F2BD
:10FCD000EA805C2140460493FDF79EFD049B90E082
:10FCE0009AF84C20112A00F0FB80752B0CBF4FF0C6
:10FCF000030B4FF0070B002308EE108A0494A8466C
:10FD00005C469B4608E028464FEA0B1BFEF7B0FA1C
:10FD1000013C8344C0F0F7805046FFF78BFDDAF8D2
:10FD200010502846FEF758FA0028ECD14546049CAE
:10FD300018EE108A4FF001034FF0000B8AF84C3098
:10FD400032E74FF0000B2FE70A239AF84C20102AD5
:10FD500000F09E80112AEDD1D9B240464FF0000B41
:10FD6000FDF74EFD20E70C23EFE70B23EDE709231A
:10FD7000EBE70D23E9E78A427FF411AE002D3FF453
:10FD80006DAE5046FFF756FD022D77D0DAF81040E1
:10FD900064E6DAF81420A24208D000230126019379
:10FDA0006FE60AF16000FDF737FD94E65046032642
:10FDB000FFF740FD5046FFF73DFDDAF8101059E619
:10FDC000404685F00105FDF727FDDAF86430002B89
:10FDD00048D05046A9464FF0000BFFF72BFD7FE6B9
:10FDE000DAF81420722A27D00027029B069A0125F0
:10FDF00011210593039725E640460493FDF70CFD7A
:10FE0000049B5A1C9DD0B3F5881F93D29AF84C20BE
:10FE1000102A3DD0FF2B9DD98CE7DAF81420622AF6
:10FE20000AD0662A00F05A81029B0125069A102109
:10FE300000270393059305E6029B0225069A1121EC
:10FE4000002703930593FDE5DAF81420722A00F0E9
:10FE50004581029B0125059A10211F460693002328
:10FE60000393EFE5A5490AF16000FDF731FDB0E726
:10FE70002C210AF16000FDF7CFFC84E65046FFF725
:10FE8000D9FC83E79AF84C205B46102A7FF462AFD6
:10FE9000194640464FF0000BFDF7BEFC84E60522F4
:10FEA0008AF84C202AE6DAF81430303B072BE9D8E0
:10FEB0005046FFF7BFFCDAF81420DAF81030303A79
:10FEC000303B072A03EBCB039BD850460493FFF744
:10FED000B1FCDAF81020049B303A02EBC30390E740
:10FEE0005C2140460493FDF797FC049B8EE74FF09E
:10FEF000010B00E7082328E7072326E7804818F0CE
:10FF0000C9F906F04FFE45465B46049C18EE108A80
:10FF100077E74846FEF748F9002840F0B580DBF85F
:10FF20001000A0F15F04B4FA84F464097F2888BF4C
:10FF300044F00104002C4AD00BF150040D22C1B250
:10FF400020468BF84C20FDF75BFC5846FFF772FC0F
:10FF5000DBF81000431C0BD0FEF726F978BBDBF86A
:10FF600010007F282DD85F282BD0FEF729F930BB51
:10FF70002046644DFDF730FC00246349064607E047
:10FF8000FFF60DAD0134242C3FF409AD55F8041FE4
:10FF900030464CF0F0FD0028F2D104F11302D2B249
:10FFA000162A8BF84C207FF4FAAC584AD2F8E82095
:10FFB000002A0CBF152213228BF84C20EFE4DBF84B
:10FFC0001000C1B22046BEE74FF0000B8EE5FEF7F1
:10FFD000F7F800286CD0DBF810102E2900F0DA803A
:10FFE0000E2230298BF84C2000F0D8800BF1500500
:10FFF0002846FDF711FC5846FFF71CFCDBF8100003
:02000004600199
:10000000411C3FF4CCAC0F26ACB920F02003452BAB
:1000100011D1652128468BF84C60FDF7FDFB584651
:10002000FFF708FCDBF810002B2830D02D282ED04D
:10003000421CE9D1B3E4FEF7B7F890B1DBF8101039
:1000400021F020034A2B01D02E2901D18BF84C60DE
:100050002846FDF7E1FB5846FFF7ECFBDBF8100004
:10006000E6E7DBF81000FEF7ABF80028E6D1DBF896
:1000700010102E29EAD05F297FF491AC5846FFF783
:10008000D9FBDBF81000D3E7DBF8100054E701469A
:10009000DEE7DBF83820954224D26A1CCBF83C20FE
:1000A00020F81540DBF830200132CBF8302076E420
:1000B000DBF810102E297FD00026154D282407E0EC
:1000C000632C09D02B465C7801365D1C002C5AD07D
:1000D0008C421FD0652CF3D16B1CF4E709228AF8FF
:1000E0004C205CE408325100FCF7FAF9CBF84000F0
:1000F000DBE90E250832CBF83820CEE70015066084
:100100000C15066010160660B4140660000400208A
:10011000BC1406605846FFF78DFB212C5DD02E2CB9
:1001200067D06F786C1C632F01D0652F0FD13046DC
:1001300063780136DBF810209A421DD0632F05D07A
:1001400014F8027F632FF3D0652FF1D00646354AAD
:10015000925D4C2A02F0FB018BF84C2036D04A29E4
:1001600034D04D2A02D04B297FF419ACDBF834206F
:10017000013ACBF8342012E45846FFF75BFB652FB9
:10018000E5D03046DCE75846FFF754FB01228BF8F8
:100190004C2004E40F228BF84C2027E7DBF81420D6
:1001A00042F02002623A162A3FF620AF1E4C24FA93
:1001B00002F202F0010419E7DBF81400FEF700F880
:1001C00000287FF408AFDBF8101075E7DBF8342067
:1001D0000132CBF83420FFF7E2BBDBF810203D2AD8
:1001E000D4D15846FFF726FB49228BF84C20FFF765
:1001F000D6BBDBF810202E2A04D052228BF84C20DC
:10020000FFF7CDBBDBF814202E2AF6D15846FFF7B6
:1002100011FB5846FFF70EFB12228BF84C20FFF71C
:10022000BEBB00BFE41506600120400070B584B07D
:100230000646742001AD85E80E000021FCF732F976
:100240000446034695E8070043F8046B002583E85D
:1002500007000A2201236FF001011420E3632563E4
:10026000C4E90D52C4E90A312946FCF71BF90346DB
:10027000202104F150002364FDF724FA294604F1FB
:100280006000FDF71FFA236C20461D802561C4E93C
:100290000555FFF7CFFA2046FFF7CCFA2046FFF7C7
:1002A000C9FA2046FFF756FBA36C012B02D00B23A3
:1002B00084F84C30204604B070BD00BF30B585B026
:1002C000054601AC2046FFF765FA284694E80E0083
:1002D000FFF7ACFF05B030BD30B585B0054601ACC9
:1002E0002946204615F01AFB2846FDF71BF994E82D
:1002F0000E00FFF79BFF05B030BD00BF10B50446F0
:1003000070B1E3684068984704F15000FDF712FAB5
:10031000206CFCF7F3F82046BDE81040FCF7EEB87F
:1003200010BD00BF38B50D460446D0E903138B421B
:1003300005D240695A1C226140F8235038BD103163
:1003400040698900FCF7CCF86061D4E903231032DE
:10035000E2605A1C226140F8235038BD2DE9F0417B
:100360008846044617461E46D0E900158D420ED237
:1003700080686B1C636050F8353068F3170340F8F1
:10038000353000EBC500C7704660BDE8F081103124
:100390008068C900FCF7A4F8236865681033A06082
:1003A0002360E6E710B48469CAB20023616C5DF88B
:1003B000044BFFF7D3BF00BFF8B5446A06460D46AD
:1003C00034B363685A1821688A4204D804F10800DB
:1003D00062601844F8BD05F1080320460022194464
:1003E000FCF78AF848B104F10800D4E90023511958
:1003F000EA18184421606260F8BD61680246204630
:100400000831FCF779F863682360336A636034620B
:10041000102D2F464FF0000138BF102707F10800BC
:10042000FCF740F800230446C0E90073706243689B
:1004300004F10800EA1818446260F8BDF0B5866956
:1004400083B005460F4696F84C300D2B10D00E2B7E
:1004500049D00F2B1ED0A3F11002012A33D9190164
:1004600041F00E01284603B0BDE8F040FFF75ABF47
:10047000716DFF2966D8B06DFCF7B4FF8E2F04466E
:1004800052D02101284641F0020103B0BDE8F040FE
:10049000FFF748BFD6E9151000230122009605F0AA
:1004A00031F804460C212846766CFFF785FF40F2B0
:1004B000391301468460C0E90063284603B0BDE8F3
:1004C000F040FFF72FBFD6E915100A291CD8FCF71A
:1004D00089FFE0B196F84C30102B0CBF06220A229F
:1004E00042EA0011BEE733460022D6E9151004F0B7
:1004F00061FFC3070446D5D544F00101284603B087
:10050000BDE8F040FFF70EBFFCF71EFFE1E796F8ED
:100510004C00104A104B10280CBF10461846D6E964
:1005200015210CF0D5FCBCE7C100002205F1280024
:1005300041F006014CF060FB0028A2D04468E207BD
:10054000B0D5D9E7054817F0A5FE0146044805F0E7
:10055000FFFB00BF984D0660044B0660A0160660C6
:10056000E4350660B0F59F7F09D010F0010304D098
:1005700043080CBF01200020704718467047012037
:10058000704700BFB0F5AF7F09D010F0010304D071
:10059000430814BF0120002070471846704701200F
:1005A000704700BF10F0010308D130B110F0030212
:1005B00017D10379392B06D01046704740F001035C
:1005C00001200B607047836813F001000B60F4D1C9
:1005D0009A07F2D11868044BC01AB0FA80F04009AB
:1005E00070471846704700BF703C06602C2A2DE902
:1005F000F04F174687B0044688461E4640F0888074
:1006000003694269013B52F82330002B78D1A7F1EE
:100610002503022B40F2E080282F00F0D081052F27
:1006200040F07C81D4E90432013B52F823509B0016
:10063000002D46D0A90744D1696801F0FE00562874
:100640003FD0134453F8042C02F00F03022B38D18F
:10065000C9B22B2935D1AB6803F00F01022930D183
:100660001B09B3F5EA7F2CD1E96851B311F0030AF5
:1006700027D10B792F2B24D1D1F808B004A94FEA48
:1006800012195846FFF78EFF002800F0CD814FEA7F
:10069000C901012204F1280041F006014CF0ACFA36
:1006A000049B024648465360FCF758FF03785F2BD3
:1006B00000F0B081236959462046013B2361FFF7D2
:1006C00031FEB51C47EA06272046AD002946FFF754
:1006D00073FE0146C0E9008766B12A1F0244013E4D
:1006E000D4E9043503F1FF33236155F8233042F890
:1006F0000439F4D1204607B0BDE8F04FFFF712BE31
:10070000980702D11B79902B81D007B0BDE8F08FFC
:10071000A2F11D03012B1BD91F2A40F0B1800369F0
:100720004269013B52F82320B2F59F7F00F0A5807B
:10073000D00740F1DC80520814BF4FF49F714FF492
:10074000AF712046236107B0BDE8F04FFFF7EABD67
:10075000002E00F05C8103694269701EA3EB060362
:1007600052F82330D1D01D2F324629D0B3F59F7FC8
:1007700003D0DD0714D55B0816D1013AA1D0002AB9
:100780002369A6EB0206C2F1010203F1FF3308BFA1
:100790000022012E1A44226193D107B0BDE8F08FE8
:1007A000B3F5AF7F00D0013AD4E904512B1AAD1A4A
:1007B000013851F8233041F82530DED01D2FD5D136
:1007C000B3F5AF7FD9D0D90702D55B08D5D1EBE718
:1007D000B3F59F7FE7D1E7E7236903A962699B1B14
:1007E00052F82300FFF7DEFE00283FF46AAFB51E83
:1007F000002D40F30881A6F1030A0DF11009DFF87E
:100800005CB22AF00103A6F1040AAAEB03030193E8
:100810000DE00028FFF655AF5046023DDDE903121A
:100820004CF0DEF9019A03460390954266D02369A5
:10083000494662695B1B52F82300FFF7B3FE0028AC
:100840003FF43FAF23696269013B5B1B52F82330E1
:10085000C3F307135B4413F837ACBAF1FF0F3FF44F
:1008600030AF04980AF0B8F8BAF1190FD1D9BAF13B
:100870001C0FD1D90028CFD123E74FF4AF7160E727
:10088000A2F12203022B3FF6C2AE036903A942691B
:100890009B1B52F82300FFF785FE00283FF411AFA1
:1008A000222F00F0AC80232F0CBF16251725B6F1A0
:1008B000020A00F1A8800DF110090BE00AF1FF3ADD
:1008C0002846DDE903124CF08BF9BAF1FF3F0346ED
:1008D000039013D0236949466269013BA3EB0A03E5
:1008E00052F82300FFF75EFE0028E7D1E9E6B2F5F3
:1008F000AF7F7FF4E6AE4FF49F7122E703F0010172
:1009000016B12269921B226101F0FF05002946D031
:1009100043F001012046FFF705FDF6E62B2F7FF49B
:10092000D0AED4E90423023A53F8221003EB820339
:1009300001F00F025B68022A7FF4C3AE002B3FF484
:10094000C0AE13F003027FF4BCAE187931287FF4F7
:10095000B8AE09093D489D68C90041F006014CF058
:100960004BF900283FF4ADAE2909406804AA05F010
:10097000FBFB049B002B3FF4A4AED80703F001015E
:1009800007D49A077FF49DAE314A186890427FF4ED
:1009900098AE059A002A7FF494AE0393B0E70C2139
:1009A00020460193FFF708FD40F239120146019BF2
:1009B0002046C1E900528B60FFF7B4FCA5E623692D
:1009C00003A96269013B52F82300FFF7EBFD002801
:1009D0003FF477AED4E90432023B52F82330C3F33C
:1009E0000713372B0DD0382B0CBF012002200399A1
:1009F00005F02EFA034600F00101039080E715256B
:100A000055E70020F3E7039B03F0010178E74FF07F
:100A1000FF32B4E62069534608225146023820616D
:100A20002046FFF7E3FD70E601900A4817F032FC1C
:100A30000146094808F026FEA1690446019B2A6880
:100A4000096808F069FE2046FBF706FD50170660AE
:100A5000703C0660B0160660E4350660401C066017
:100A600010B4046803464CB1A00702D12079884233
:100A700009D001205DF8044B1360704720461460D4
:100A80005DF8044B704704F10803136060685DF87B
:100A9000044B000A704700BF2DE9F04F402393B08C
:100AA00000240F460390184602920593CDE90644B0
:100AB00004E0059840080128059006D90021C000EF
:100AC000FBF7FCFC07900028F3D0002320200A93BA
:100AD000CDE9080305E0089840080128089040F295
:100AE0003D8200218000FBF7E9FC0A900028F2D04B
:100AF000079B002B00F0328200210FA80B97CDE955
:100B00000D1106F085F9029B002B00F0F481022BF9
:100B10000CBF3C2200220023796C05A8FFF71EFCC5
:100B2000069B002B4FD04FF0000BDFF80C93013BDE
:100B3000079A069302EBC30152F8332091F803A001
:100B4000C2F317024C68BAF1650F0192B54A12F868
:100B50000A200092B44A12F80A50B44A88BF45F4F9
:100B6000807502EB4505009A02F0300102F00F0695
:100B7000102900F08280202954D0BBF1000F00F032
:100B80001A81022E00F01281012C00F0B28014F0C4
:100B9000010B03D0032E54D14FF0010B009A631EBA
:100BA000D20706D5698809EA0101B1F5805F08BF5F
:100BB0006308012B40F09380BBF1000F40F08F8061
:100BC000069B002BB3D10FA806F042F90E9860B136
:100BD000416800220831FBF78FFC0E9B5A681A60AF
:100BE000DDE90D235A600E9B0D9397F84C1051BB15
:100BF000099B002B00F0B9810A9B07981B680C9396
:100C0000FBF77CFC0A98FBF779FC3846FFF776FB8C
:100C10000CAB93E80300039B83E80300184613B072
:100C2000BDE8F08FBBF1000F6ED06FF000412144A2
:100C300035F8111009EA0101B1F5405F60D0012CCF
:100C4000BFD997F84C10092900F27B81032900F2E3
:100C50007C81022940F08981754817F01BFB014611
:100C6000744808F00FFD0446204600237A6C39686A
:100C700008F052FD2046FBF7EFFB14B1BBF1000F6B
:100C80009FD0B44236D205EB440509E0C1F30B0115
:100C900097F84C208A4200F0B6800134B44229D241
:100CA000A84635F8021B01EA0902B2F5805FEDD0D3
:100CB000631CB342C0F0E58005A84FF0000BFFF7BE
:100CC00071FB069B002B7FF432AF7CE7B8F1010F7C
:100CD00000F01381009B190600F100812346524663
:100CE000019905A84FF0000BFFF780FC68E7002C86
:100CF000A9D1069B4FF0010B002B7FF418AF62E7E0
:100D0000002105A8FFF70EFBA64222D905EB440BF4
:100D100005E001343846FEF71DFEB44219D0D8462E
:100D20003BF8023B03EA0902B2F5805F40F097808E
:100D3000DBB297F84C109942D9D10D29E9D151462F
:100D400005A80134FFF77AFB3846FEF703FEB442EC
:100D5000E5D1029B002B00F0C880BAF1050F40F0EE
:100D6000C480DDE909C00CF1FF3150F821308C005E
:100D7000002B40F094800444ACF1020354F8044C7E
:100D8000A20700F0868004F00F04022C00F0878098
:100D9000099308220023019905A84FF0000BFFF7E3
:100DA00025FC069B002B7FF4C2AE0CE7012CA0D0E3
:100DB0004FF0000BF2E606EA040303F0010335F8F6
:100DC000138008EA0901B1F5805F0FD036E00134E5
:100DD0003846FEF7BFFD04EA060303F0010335F8C9
:100DE000138008EA0902B2F5805F27D1C8F30B0827
:100DF00097F84C20424530D1002BE8D1514605A848
:100E0000FFF71CFBE3E7514605A8FFF717FB384641
:100E1000FEF7A0FD069B4FF0000B002B7FF487AE82
:100E2000D1E600BF64170660901B066014180660C8
:100E3000F81606606032066000F0FFFF631C524641
:100E4000019905A8FFF78AFA414605A8FFF7AAFA13
:100E5000069B002B7FF46BAEB5E6013491E6631C74
:100E60005246019905A8FFF779FAB8F8001005A8CD
:100E70004FF0000BFFF796FA069B002B7FF457AE5E
:100E8000A1E60199524605A8FFF768FAB8F80010E4
:100E900012E7002C50D02479392C3FF479AF002E82
:100EA0004DD0002405EB4606A04609E00B1B50F888
:100EB00023300BB108F101080134B5423FF406AF0D
:100EC00036F8023D03EA0902B2F5805FEED1DBB2EB
:100ED0000D2BF2D1013408F10108EEE701340021B5
:100EE00005A8FFF71FFA2346F9E646B3DDE909C076
:100EF0000CF1FF31D5E73A220DE6009B5D067FF548
:100F0000E9AE74B1ACEB040200EB8C00002400E00D
:100F10000139099150F8043D002B18BF1C468A4244
:100F2000F6D1214605A8FFF7FDF9069B4FF0000B0F
:100F3000002B7FF4FCAD46E6002EB2D1CAE6344663
:100F4000C8E60B2911D10A4887E60A4817F0A2F92A
:100F50000146094808F096FB044685E6074817F065
:100F600099F90146064804F0F3FE0648EEE700BF93
:100F7000E41606602C170660E4350660CC160660A1
:100F80008C3306604017066010B544682CB12046CB
:100F90006468FBF7B3FA002CF9D110BD2DE9F041DC
:100FA00005460E463020002190461F46FBF796FA74
:100FB000072D04460570C660A0F8108013D0012DDF
:100FC00011D00B4B5B5D638204F026FC042360614F
:100FD0000021E38420206776FBF764FA034620466D
:100FE000E362BDE8F081B368C3F30F13EBE700BF22
:100FF0004C1C066010B50446C06AFBF77FFA204619
:10100000BDE81040FBF77ABA2DE9F041058D07469F
:101010000E469046C06A95B14FF0000C034601E0C1
:10102000AC450CD05C6819460CF1010C0833A642A3
:10103000F6D10023084688F80030BDE8F081F98C2D
:10104000A9420DD96B1C00EBC5013B85002340F87C
:10105000353001234E60084688F80030BDE8F08145
:101060000631C900FBF73CFAFB8C3D8D0633F86274
:10107000FB84E7E730B4058D7DB1C36A002201E04F
:10108000AA4207D05C681846013208338C42F7D177
:1010900030BC7047002030BC70472846F8E700BFDE
:1010A00030B4034640680028FBD11C8D5CB1DB6A7C
:1010B000024603E0A24203F1080304D05D68013256
:1010C000A942F7D1184630BC704700BFF0B543685D
:1010D00083B0164693B15A6882B11D8D95B1DC6A12
:1010E000002303E09D4204F108040BD0676801333C
:1010F000BE42F7D12378023B022B09D900230B70A3
:1011000003B0F0BD54681346002CF7D02246E4E744
:1011100004250D70446801E0057064680DF1070254
:1011200031462046FFF770FF9DF80730002BF3D1C2
:101130000378022BE4D103230370E1E7F0B51D46E9
:1011400083B0B1B111F0030603D14F68FBB29342F3
:1011500004D02B4603B0BDE8F04018473F0A08D042
:101160000C1D0136019054F8041FA847B74201989E
:10117000F7D103B0F0BD00BF024B9B228968FFF797
:10118000DDBF00BFE91D0160024B6A228968FFF7DD
:10119000D5BF00BF6519016010B504460846114669
:1011A0002268FFF7FBFE0023626AC0E90123236A7D
:1011B0002BB11A469B68002BFBD1906010BD2062BA
:1011C00010BD00BF10B504460021806A03F04CFC3E
:1011D000A06A142103F074FAA06A0121BDE810404E
:1011E00003F08CBD89680022806A090903F05ABBAC
:1011F000806A896803F0EEBA2DE9F04F804683B02B
:101200000F46924699461BB10B7E43F008030B76BE
:10121000A7F81EA0D8F824201378002B38D0138DFF
:10122000002B35D00025AB4603E00135138DAB42D2
:101230002BDDD66A16F8353006EBC506033B012BCD
:10124000F3D8388D0028F0D0002401E0A04216DD4C
:10125000FB6A13F8342003EBC4030134042AF5D1EC
:1012600071685B689942F1D1D8F828000023728830
:101270000BF1010B03F016F9388DA042E8DCD8F829
:1012800024200135138DAB42D3DCBBF1000F09D113
:101290004B4652463946D8F8280003B0BDE8F04F17
:1012A00003F0C4BCD8F8280053465A463946CDF856
:1012B000009003F0D3FC03B0BDE8F08FF8B50D4605
:1012C00011461A46002304468679476983714361B3
:1012D0000F4BFFF733FFA36803B1F8BDE18AA38A80
:1012E00001B153B10A4620462946FFF785FF003E6B
:1012F000676118BF0126A671F8BD1A46A06A03F0FF
:1013000041FCA06A03F07CFAE18AA38AEAE700BF05
:101310003926016070B5437904460D46012B07D08C
:101320000969AA6820464B23BDE87040FFF7C6BF95
:10133000436A0A4602215B7EFFF72EFF01462861C1
:10134000EFE700BF70B5437905460C46012B08D086
:101350008E6928464323E2683146FFF7AFFF708A63
:1013600070BD13460A460721FFF716FF0646A06127
:10137000EFE700BF10B500220446806A03F04AFA86
:101380000023A06A1A46194603F092FC2046BDE8E5
:101390001040FFF717BF00BF2DE9F04F134687B08D
:1013A0008146002965D08A076DD10A790191672AA3
:1013B00079D001F00F02022A6BD08A68002112094D
:1013C00003911A60019A53684FEA132808F1FF3617
:1013D000B8F1000F77D0171D0024BA465AF8040F51
:1013E000254601340009FCF7A7F8A0450644F5D1CD
:1013F00030464FF0000BFBF771FF4FF02E0A04460A
:10140000029001E004F801AB57F8040F05A90009A8
:10141000FCF7B6F8059A014620464BF05DFB059BAC
:101420000BF10102AB451C449346EBD1029C3146C3
:101430002046FBF7D7FF2B4B01460022D9F82800A6
:101440001C6103F01FF9039B83B1B8F1010F0DD0AC
:10145000019D0124083555F8041F01340022D9F8F4
:101460002800090903F01EFAA045F4D107B0BDE831
:10147000F08F012100221960D9F8280007B0BDE8DB
:10148000F04F03F0FFB801F00F02022A01D00191E2
:1014900093E7090919600022D9F8280007B0BDE8D0
:1014A000F04F03F0EFB8CA6812091A608968002982
:1014B000DFD001F00F03022B03D00123019103932E
:1014C00080E70909E7E73046FBF708FF31460446A5
:1014D000FBF788FF034B01464246D9F828001C6100
:1014E000CCE700BF0004002001B9704701F00303FE
:1014F000C2681343F9D10B68C360704738B504461E
:101500000D460648114608F0BDF803462946204618
:10151000A360BDE83840FFF7E7BF00BFE4350660D1
:1015200038B5044606480D4616F0B4FEA36803B16C
:1015300038BD024629462046BDE83840FFF7DEBFE9
:10154000541C066070B50B790D460446092B10D06B
:101550001048668B16F09EFE4FF6FF739E4210D029
:10156000A28B3146E38BA06AD21ABDE8704003F02B
:1015700025BA0948268B16F08DFE4FF6FF739E4262
:10158000EED1A368002BEBD1024629462046FFF797
:10159000B5FFE5E78C1C0660741C0660F8B5436A6D
:1015A00005460E461B7E13F0100401D00120F8BD45
:1015B000064816F06FFEAF680FB12046F8BD024630
:1015C00031462846FFF79AFF3846F8BDA41C06604E
:1015D0002DE9F04F437985B005460E46012B02D028
:1015E00005B0BDE8F08F91F80480B8F1100F03D07A
:1015F000436A1B78002B56D003AA6C2106F1080021
:10160000FFF72EFA071EEBDD4FF0000BDFF8C0905E
:101610000DE06ABB0278042A05D0484616F03AFE6F
:10162000AA68002A32D00BF1010B5F45D8D0039A8B
:10163000686A52F82B100DF10B0209090191FFF7AE
:10164000E3FCB8F1100F04469DF80B200199E0D19E
:1016500012B90278012A1FD14FF0010A84F800A0C4
:10166000686AFFF71DFD0028DDD080F800A0DAE7EA
:101670000A460146686AFFF729FD2278002AD2D17E
:10168000104816F007FEAA68002ACCD1024631465F
:101690002846FFF733FFC6E70B4816F0FBFDAA68A4
:1016A000002AC0D1F2E7094816F0F4FDAB68002B20
:1016B00096D102463146284605B0BDE8F04FFFF707
:1016C0001DBF00BF281D0660081D0660E01C0660E7
:1016D000481D066070B50446406A82B00D4690F819
:1016E00018C01CF0020F33D101F00F0102290ED0F7
:1016F0002979914222D0994238D0A9684CF0020C45
:101700000526090980F818C051B902B070BDA37947
:101710002909C3B1838B0126013383830029F4D0C7
:101720000DF10702606AFFF76FFC9DF80730002B90
:1017300031D002234670037002B070BDA968A3794E
:101740000909002BE6D1438B012601334383DBE7F4
:10175000184816F09FFDA368002BD6D102462946F3
:10176000204602B0BDE87040FFF7C8BEA379002B49
:10177000EED10123A371AB68002BC6D003F00F0399
:101780000326022B037E43F0010303760FD0AB68E0
:1017900099680909B8E7084816F07CFDA368002B92
:1017A000B3D1024629462046FFF7A8FEADE7A96857
:1017B0000909A9E7401706606C1D0660462345220B
:1017C000FFF788BF4E234D22FFF784BF42790B46B7
:1017D000012A04D0426A0349806A02F069BC406A67
:1017E00002F048BCB820066042790B46012A04D0BA
:1017F000426A0349806A02F05BBC406A02F03ABC6C
:10180000C820066010B5436A04465A7EFFF79AFD69
:1018100001462046BDE81040FFF7E6BF2DE9F04342
:101820008F6885B00D46044607F00F030E2B53D08A
:10183000002F46D100210DF10C08EA6840F29E33DA
:10184000A06A9A4269D002F069FF02AA05F10C0071
:101850006921FFF705F9B0F1000976DD0025029B4B
:101860002E46A06A53F8253001359968090902F01F
:10187000A3FFA945F3D149460022A06A002503F041
:1018800081F9424639462046FFF786FD029B012238
:10189000A06A53F82570B9680909019102F0F2FEB7
:1018A000FB682046019903B11909FFF79DFF6B1CE6
:1018B000B5421D46EAD1A06A02F0DEFF05B0BDE8E0
:1018C000F083BB07B6D13B79642B05D0612BB1D136
:1018D000BB680293FF6801E0029700270DF10C0836
:1018E000642102A84246FFF7BBF8002838DD039BBD
:1018F000002240F22E56043B03EB800153F8040F04
:10190000B0420CBF013203329942F7D1114640F286
:101910009E33EA68A06A9A4295D102F0FFFEA06A5F
:10192000502102F049FFA06A0022012103F02AF9A8
:10193000424639462046FFF72FFD02220021A06AC9
:1019400002F0A0FE05B0BDE8F0834946A06A00227F
:1019500003F018F9424639462046FFF71DFDAAE775
:1019600000216AE730B5044683B00D46806A002145
:1019700002F0D4FEA06A142102F0A2FE29462046FD
:1019800001AAFFF709FD01992046FFF72DFF03B0DB
:1019900030BD00BF42790B46012A04D0426A034998
:1019A000806A02F085BB406A02F050BBC02006602E
:1019B00030B5054683B00C4671B1CA070ED48B070B
:1019C0002AD001F00F030C09062B1ED00A2B0CD0D5
:1019D000022B14D00A2C2DD103B030BD4910806ADF
:1019E00003B0BDE8304002F099BE4379042B28D003
:1019F0001A49806A03B0BDE8304002F0EBBE2146D0
:101A000003B0BDE83040FFF7C5BF2146806A03B090
:101A1000BDE8304002F0D0BE0968806A02F0C6FD21
:101A200022790F4B2146284653F8223003B0BDE8F7
:101A300030401847E1B2806A03B0BDE8304002F0A0
:101A40003FBE01A92046FBF79BFDAC6A01990BF054
:101A5000C5FA0146204602F0BDFEBDE7E84106603A
:101A6000D01F06602DE9F04F074683B00C4616469E
:101A7000984611E0FEF786FD50BBD4B1A30718D1FC
:101A80006168CBB2090A1D2B2BD01E2B59D01F2BFE
:101A90000DD1A46886F001062046FEF763FD0346DB
:101AA0002046002BE6D0AEB103B0BDE8F08F2C2B62
:101AB0000BD038462146FFF77BFF42463146B86AD5
:101AC00003B0BDE8F04F02F04DBFA368002BEAD091
:101AD000002EE9D04146B86A03B0BDE8F04F02F0ED
:101AE00033BF86BBD7F8109001F1FF3A09F101032B
:101AF000BAF1000F3B6114DD04EB810586F00102B1
:101B000004F1040B019626462C4615465BF8041F8B
:101B10004B462A463846FFF7A5FFA345F6D1344683
:101B2000019E0AF1020A38464346324654F82A100A
:101B3000FFF798FF4946B86A03B0BDE8F04F02F0DE
:101B400091BD002ECED10029AED0251D05EB81041C
:101B500055F8041F434632463846FFF783FFAC4230
:101B6000F6D103B0BDE8F08F38B5426A04460D46A1
:101B70001378072B01D0022B10D1AD68A5B1A907AE
:101B800002D12B79AE2B19D029462046FFF710FF42
:101B9000A06A0021BDE8384003F0B0B8144816F040
:101BA00079FBA368E3B138BDA06A142102F088FD77
:101BB0002946A06ABDE8384003F0A0B8137EDB06D2
:101BC00008D42046A968FFF7F3FE2046BDE8384058
:101BD000FFF7F8BA074816F05DFBA368002BE2D1C7
:101BE000024629462046BDE83840FFF787BC00BFC3
:101BF000881D0660A41D066038B50C460546C968F8
:101C0000FFF7D6FEA1682846BDE83840FFF7D0BEF2
:101C100038B50B790C460546332B17D01421806A52
:101C200002F04EFDA468C4B1A30704D12379982B18
:101C30002AD0992B16D021462846FFF7B9FEA86A6C
:101C400008220221BDE8384002F09CBF8968FFF7F6
:101C5000AFFEE468A468002CE6D11421A86A02F063
:101C60002FFDECE7A1682846FFF7A2FEE36899681C
:101C70000029E4D02846FFF79BFEA86A082203212A
:101C8000BDE8384002F07EBF1421A86A02F018FDBA
:101C9000A1680029EED1D2E710B504468968FFF7A4
:101CA00087FE0021A06ABDE8104002F02DBE00BFF3
:101CB0002DE9F041064615468846A9B96DB16F6811
:101CC0003F0A09D004350024013455F8041F30467A
:101CD000FFF76EFEA742F7D1B8444146B06A002232
:101CE000BDE8F04102F04EBF4FF00108FFF760FE83
:101CF000E4E700BF0A460021FFF7DABF2DE9F0470D
:101D000006690446838B0D46B0F81E80771CC3839A
:101D1000B31CD0F818900361068347838868FEF7E8
:101D200021FC68B12046C4F81890A4F81E802969E7
:101D3000FFF73EFE3146A06ABDE8F04702F092BCD4
:101D4000D4F810A00AF101032361A868FEF71AFC79
:101D500090B15146A06A02F085FC2046E968FFF781
:101D600027FE3946A06A02F07DFC53460122A9688D
:101D70002046FFF777FED5E73946A06A02F0E4FD7A
:101D8000E7E700BF10B504468968FFF711FEA06AB7
:101D9000BDE8104002F070BD38B5436A04460D46F8
:101DA0001B78072B11D1896831B1FFF701FEA06ABA
:101DB000BDE8384002F08ABF806A142102F080FC3E
:101DC000A06ABDE8384002F081BF064816F062FA0A
:101DD000A36803B138BD024629462046BDE8384015
:101DE000FFF78CBBC81D06602DE9F84301F00F0317
:101DF0000C460646022B35D044B1A30714D0444804
:101E000016F048FAB36843B1BDE8F88340480024AF
:101E100016F040FAB368002BF6D102462146304650
:101E2000BDE8F843FFF76ABB23792B2B22D02C2B7C
:101E3000E5D1A468002CE9D0E56855B115F0030799
:101E400007D16A68D3B2932B12D0942B2DD0AB2B31
:101E5000D5D0A1683046FFF7C7FFE46804F00F0350
:101E6000022BC9D121093046BDE8F843FFF7AEBCCB
:101E7000A468F3E7A1683046FFF79AFDE768002FF2
:101E8000BDD017F00305BAD17B683946DAB28C2A87
:101E90001ED0302A32D0312AB1D189680222B06AEC
:101EA0000909BDE8F84302F0FDBC4FEA1228A16819
:101EB0003046FFF799FFB8F1000FA5D00435013780
:101EC00055F8041F3046FFF78FFFB845F7D19BE761
:101ED0001B0A03F1FF38B8F1000F09DD07F104090F
:101EE000013559F8041F3046FFF762FD4545F7D12B
:101EF00008F1020857F828100A79CAE730468968BD
:101F0000FFF756FDB06A0221BDE8F84302F0FCBCC1
:101F1000E41D06602DE9F0414F68884605463F0AFA
:101F200015D00E1D002402E00134A7420FD056F850
:101F3000041F2846FFF73CFDAB68002BF4D00234A9
:101F4000284658F82410BDE8F041FFF7CDBABDE8A7
:101F5000F08100BF10B50446FFF7DCFF2021A06A26
:101F6000BDE8104002F0E6BD2DE9F047D0F8109032
:101F700082B00646884609F1010303618868FEF7CE
:101F8000F1FA18BB346902463046631C33612346BC
:101F9000D8F80810FFF766FD3046D8F80C10FFF7A8
:101FA00007FDD8F80800FEF7EDFA002845D1D8F86B
:101FB000103013B9D8F8143023B1B06A02F05EFAC9
:101FC000002846D02146B06A02F04CFB01AA7021DD
:101FD00008F11000FEF744FD071E29DD002401E092
:101FE000A74225D0019B53F824500134A868FEF77E
:101FF000B9FA02460028F3D1D6F810A030460AF10B
:10200000010153463161A968FFF72CFD3046E968AC
:10201000FFF7CEFCA868FEF7B5FA70B9B06A02F017
:102020002DFA88B15146B06A02F01CFBA742D9D103
:10203000D8F814103046FFF7BBFC4946B06A02F0EE
:1020400011FB02B0BDE8F0874946B06A02F07CFCA3
:10205000E8E74946B06A02F077FCB3E770B5437928
:1020600004461546CE68012B13D071690023204623
:102070001A46FFF7C1F8F1682046FFF799FC062DD4
:1020800010D00023A06A01211A46BDE8704002F07A
:1020900001BE436A0A4629465B7EFFF77DF801468A
:1020A0007061E3E70021A06A02F0DEFCE9E700BF0F
:1020B00010B489680346B1B1CC686CB114F0030266
:1020C0000AD194F804C0BCF1930F13D0BCF1940F63
:1020D0000FD0BCF1AB0F12D00A46184600215DF8B4
:1020E000044BFFF7E5BD0A46806A5DF8044B02F039
:1020F00049BD224689685DF8044BFFF7D9BD062229
:102100005DF8044BFFF7AABF70B58D6804467DB13A
:10211000AA0702D12B79902B11D029462046FFF730
:1021200047FC0122A06A1146BDE8704002F02ABDBA
:1021300029460122806ABDE8704002F023BDEE68A6
:1021400076B1B3070CD13379932B18D0942B18D0D8
:10215000AB2B05D129460322BDE87040FFF77EBFB7
:10216000A9682046FFF724FCE9682046FFF720FC19
:10217000A06A01220221BDE8704002F003BDA968F7
:10218000CDE7A968FFF714FC31462046FFF7C2FEF1
:1021900071680122A06A090ABDE87040114402F08A
:1021A000F1BC00BF2DE9F04F87B0144680461D46B4
:1021B000039105AAA32103A80294FEF751FC071E70
:1021C00040F3A7800024A346A2462646A146059BCD
:1021D00053F82430002B3FD099073DD11A79A52A16
:1021E00044D0A62A48D0A72A36D1DA68002A49D195
:1021F0009968019301F00F02022A40F091800909C9
:10220000D8F8280002F0D8FA019B404609F10109EC
:10221000D968FFF7CDFB0134A742D8D17EB1BAF11E
:10222000000F61D0DAF808104046FFF7C1FBBBF1A0
:10223000000F5ED0DBF808104046FFF7B9FB029BA9
:10224000002B47D033464A462946D8F8280002F0EA
:102250002FFD07B0BDE8F08F06BBB9F1000F28D104
:10226000194640460135FFF7A3FBD4E7F20745D4F2
:1022700046F001069A46CEE7B0074ED446F0020675
:102280009B46C8E79107B3D11279AB2AB0D1194662
:10229000062240460135FFF7E1FEBCE721480193E5
:1022A00015F0F8FFD8F80820019B5AB107B0BDE837
:1022B000F08F1D48019315F0EDFFD8F80820019B21
:1022C000002AF3D1024619464046FFF717F907B036
:1022D000BDE8F08F33464A462946D8F8280002F078
:1022E000D9FC07B0BDE8F08FD8F8280002F088FAD2
:1022F0009DE7D8F8280002F083FAA0E70B48019385
:1023000015F0C8FFD8F808100246019B0029CDD16E
:10231000D9E74FF000094E4691E705480193EFE7F2
:102320000448EDE7501E06606C1E0660FC1D06604A
:10233000141E06602C1E066070B50D4641790446D9
:1023400001291CD0A06A02F079FA6E6900232046A8
:1023500031461A46FEF750FF718AA06A02F02CFA45
:10236000E96829B18B0703D10B79A22B08BF0021A3
:10237000204602230022FFF715FF708A70BD134626
:102380002A46FEF709FF6861DCE700BF10B5436A23
:1023900004465A7EFFF7D0FF01462046BDE81040B4
:1023A000FFF722BA002389681A46FFF7FBBE00BF79
:1023B0000B463F212DE9F04F85B0064603F108009A
:1023C00002AA0193FEF74CFB736A071E5B7E009323
:1023D00031DD0025DFF804A1B346A946029B03AA1C
:1023E0006B2153F8256006F10800FEF739FB039BCB
:1023F00080461C682209B2F5357F3BD021465846FD
:10240000FFF7D6FAB8F1010F0CDD0124039B00227F
:10241000DBF8280053F824100134090902F042FACD
:10242000A045F3D1F168002941D10135AF42D5D1A2
:102430005E46A7EB0907019BD9680B79032B47D0B0
:10244000412B38D0009A3046FFF776FF0546002F23
:1024500009DD0024002301340121B06A1A4602F08C
:1024600019FCBC42F6D129463046FFF7BDF905B04C
:10247000BDE8F08F022808D15C682309B3F5D47F4A
:102480000CD040F2EA22934205D0504615F002FFEC
:10249000DBF808302BB109F10109C6E701230093ED
:1024A000F9E7024621465846FFF728F8F3E7584671
:1024B000FFF77EFAB9E78C683046009A2146FEF7AE
:1024C00041FFA2690546137E43F014031376BEE76D
:1024D000009A3046FEF736FF0546B8E7901E0660C4
:1024E0002DE9F0418D6882B0044605B3AE0712D1E4
:1024F0002B79362B2BD09D2B0DD1EB681A79A02A86
:1025000034D0AB68DBB19A0719D11B79362B16D1C1
:102510000422294616E029462046FFF749FA0622FA
:102520000121A06A02B0BDE8F04102F02BBB0322FA
:102530002946A06A02B0BDE8F04102F023BB0522A3
:102540002946204602B0BDE8F041FFF787BD0322CF
:102550000121806A02F016FB20462946FFF728FA7F
:10256000A06A02B0BDE8F04102F01EBBA12101AAA1
:1025700003F10800FEF774FAA968074621B188073D
:1025800002D10B79362B41D02046FFF711FA002FEC
:102590002ADD4FF00008002602E00136B74220DDB8
:1025A000019B204653F82630194623B19A0702D1E1
:1025B0001A79362A0CD0FFF7FBF9B8F1000FECD0EE
:1025C0001B4815F067FEA368D3B102B0BDE8F081E7
:1025D000FFF7EEF9B8F1000F0CD0A06A02F0E4FAB0
:1025E000DBE7B8F1000FF0D10622791CA06A02F0F7
:1025F000C9FAEAE70F4815F04DFEA368002BE4D1B5
:10260000024629462046FEF779FFDEE70322791CC1
:10261000A06A02F0B7FA2046A968FFF7C9F9A06AD4
:1026200002F0C2FA002FD0DD4FF00108B3E700BF7F
:10263000B01E0660D01E066001F00F03022B70B5BD
:10264000044682B008D04B6803F0F702462A18D13E
:102650000123837102B070BDA379002BFAD1E38A04
:10266000002BF7D02348019115F014FEA3680199BF
:10267000002BEFD10246204602B0BDE87040FEF7C5
:102680003DBF472AE6D0DBB28E68452B0CBF0D69F3
:10269000CD68002DE0D08379FBB1838A01339BB2F2
:1026A000012B83820DD029462046FFF781F9A06ACD
:1026B000310902F081F8A06A02B0BDE8704002F072
:1026C00073BAC18A91B10022806A02F05BFA0322D8
:1026D0000021A06A02F056FAE5E7C38A29460133D1
:1026E000C38202B0BDE87040FFF762B9806A02F0B1
:1026F00087F8ECE7F01E06602DE9F0410C4606462F
:10270000D1E90171FFF754F93F0A022F16D90225CA
:10271000DFF82C8021693046FFF74AF9E36802357B
:102720001921C3F30713B06A0834373B082B98BF4D
:1027300018F8031002F0FEF9AF42EBDCBDE8F081BF
:10274000AC1F06602DE9F0414F680D4689680646CA
:10275000A7F10D083F0AFFF72BF9012F5FFA88F860
:102760000DD908350124304655F8041F0134FFF710
:102770001FF94146B06A02F0DDF9A742F3D1BDE886
:10278000F08100BF38B50C46C9680546FFF710F95F
:10279000A368C3F30713372B08D0382BA86A14BFDC
:1027A00002210121BDE8384002F0B8B9A86A002131
:1027B000BDE8384002F0B2B910B504468968FFF7A9
:1027C000F7F80321A06ABDE8104002F0A7B900BFE6
:1027D0002DE9F8430769064691F804907B1CA9F19E
:1027E0001D0903614B68B9FA89F95FEA13284FEABA
:1027F00059190BD00D1D0024013455F8041F304623
:10280000FFF7D6F844453A46494605D13946B06AFD
:10281000BDE8F84301F026BFB06A02F0B9F8EBE773
:102820002DE9F0470D460646D1E90171FFF7C0F8E2
:102830003F0A032F4CD9D6F8109009F101033361F8
:10284000022F43D9A7F103080124DFF8C0A028F024
:10285000010808F1030813E01A79832A2FD09B6836
:102860005BBB0721B06A02F065F9BC4204DA4A4654
:102870000021B06A02F08CF8444505F1080523D028
:10288000023429693046FFF793F8BC4205DAB06A92
:1028900001F0DEFFB06A02F02DF8EB6803F00F02E2
:1028A0000E2AD9D11B093E3B0B2B94BF1AF80310FB
:1028B0000621B06A02F03EF9D7E73121F9E730216D
:1028C000B06A02F037F9D0E7032F04D8BDE8F087EB
:1028D0004FF00009B4E73469B06A631C21463361E4
:1028E00002F032F84946B06A01F0BCFE0121B06A3C
:1028F00001F0CAFDB06A01F0CBFFB06A01F0BCFF85
:102900002146B06ABDE8F04701F0ACBEC41F0660C6
:10291000F8B505690E46CF680446AB1C002203617A
:102920002B46B968FFF79EF8B1686E1C2046FFF78A
:102930003FF8A06A314602F007F82946A06A01F084
:1029400091FEA06A4FF0FF3101F09EFD2046F9682C
:10295000FFF72EF83146A06ABDE8F84001F082BECC
:102960002DE9F04F2DED028B85B0056992461F468B
:102970000222109B04460E460393AB18806A294638
:10298000236102F04DF8A28B636A691C0132204674
:1029900008EE101A92B2A283998C9142314638BF48
:1029A0009A84FFF705F8A06A02F086F818EE101A6C
:1029B000A06A01F0C9FF2946A06A01F053FEA06A8F
:1029C00002F0ACF9D4F810B0BAF1000F0BF1010627
:1029D000266140F3A38001251FE05545A94640F03C
:1029E000B880A06A01F048FF2046D8F80C10FEF726
:1029F000DFFFA06A02F088F8A06A594601F0A4FF40
:102A00003146A06A013501F02DFE0121A06A01F0D6
:102A10003BFDD14580F2828026693A46731C04371B
:102A2000D2F800802361D8F80890B9F1000FD4D013
:102A300019F0030303D199F80420752A14D0A06A71
:102A400001F006FF49462046FEF7B2FFA06A0821C2
:102A500002F070F832460021A06A01F083FFA06AFC
:102A6000A94601F009FFBFE7D9E90212A06A4FEABF
:102A700012190293019101F0EBFE01992046FEF735
:102A800097FFA06A082102F055F8029B3246A06A1F
:102A9000194601F067FFB9F1000FE0D04946204622
:102AA000FEF7A2FE23690322A06A591C019321614B
:102AB000194601F0B5FFA28B616A0132019B92B207
:102AC000A283888C904200D28A84D8F80C102046C9
:102AD0000193FEF76DFFA06A01F0EEFFA06A02F01D
:102AE00013F8A06A142101F0EBFD019BA06A1946BE
:102AF00001F0B8FDA06A142101F0E2FD494620462C
:102B0000FEF772FE49462046A946FEF75FFEA38BFC
:102B1000A06A013BA38301F09BFF6DE7A38BA06A32
:102B2000013BA38301F094FFA06A02F0FBF818EECA
:102B3000101AA06A01F096FD03992046FEF738FFAF
:102B40005946A06A05B0BDEC028BBDE8F04F01F01C
:102B500089BD0A48156815F09DFBA3683BB1A38B9E
:102B6000013BA38305B0BDEC028BBDE8F08F0246AC
:102B700029462046FEF7C2FCF1E700BF201F066091
:102B80002DE9F047066904469A4682B0731C806AB4
:102B90000F461546236103223146DDF82890DDF803
:102BA0002C8001F03DFFA08B636A013080B2A083CE
:102BB0009A8C824238BF988425BB0321A06A01F019
:102BC00063FC39462046FEF7F3FE6FF00201A06A6F
:102BD00001F05AFCA06A01F06FFFA06A142101F015
:102BE0006FFD3146A06A01F03DFD20464146FEF7EB
:102BF000DFFEA38BA06A013BA38302B0BDE8F047D0
:102C000001F026BF53462A4639462046CDF80090AB
:102C1000FFF7A6FEDEE700BF70B5CD6884B00C46B6
:102C200006462B79772B1BD0732B03AA4FF0760126
:102C30000DD004F10C000025FDF712FF0246A1683B
:102C40003046039B0095FFF78BFE04B070BD05F185
:102C50000800FDF705FF2B6902465BB9ED68EEE75A
:102C60000023AA688968CDE900321A46FFF788FF79
:102C700004B070BD9B683046A1680193EC68039B6B
:102C80000094FFF77DFF04B070BD00BFF8B5154B91
:102C900004460D46D3F8E86006B1F8BD0769012285
:102CA000BB1803613B468968FEF7DCFE71210122F7
:102CB000A06A01F011FCE96849B9A06A012102F09B
:102CC00011F83946A06ABDE8F84001F0CBBC2046B7
:102CD000FEF76EFE334632460121A06A01F0DAFFAC
:102CE000EBE700BF0004002038B58D68044675B1DD
:102CF000AB0702D12B795D2B0FD029462046FEF77A
:102D000057FEA06A0121BDE8384001F0EBBF29461B
:102D1000806ABDE8384001F0E5BFA968FEF748FECB
:102D2000E9682046FEF744FEA06A0221BDE838406B
:102D300001F0D8BF2DE9F0470C4606461546A1071D
:102D400013D004F00F03022B07D0724815F0A2FA3B
:102D5000B368002B57D0BDE8F087EA074FEA14119B
:102D60004DD5BDE8F047FEF715BE6168CBB22C2B00
:102D700050D023D8062B37D02B2BE6D1022A64D192
:102D8000E768002FE1D017F00308DED17B68B94671
:102D9000DAB28C2A62D0302A7BD0312AD5D1012DEB
:102DA00000F0A880022D00F0B180D9F808100122AF
:102DB000B06A0909BDE8F04701F074BD2D2B11D1AF
:102DC000002AC2D1A168002943D08B0703D10B7917
:102DD0000846902B23D0002330461A46BDE8F04722
:102DE00000F09AB89B2BB0D1002DAED104F10803AE
:102DF0000A0A30462946BDE8F04700F08DB8BDE824
:102E0000F047FEF7F1BC024621463046BDE8F047E8
:102E1000FEF774BBA068002897D0002A95D1C1683E
:102E200051B111F0030307D14A68D5B2932D3FD0B9
:102E3000942D44D0AB2D88D000F1080302223046F7
:102E40000021BDE8F04700F067B8A168FEF7B0FDCB
:102E500096E70B46BDE8F04700F05EB84FEA13294D
:102E6000022D09F1FF390DD0B9F1000F0ADD07F18C
:102E7000040A08F101085AF8041F3046FEF798FDCD
:102E8000C845F6D109F1020957F8299099F80420AC
:102E900081E7022D1CD0D9F808103046FEF788FDD6
:102EA000012D1ED0B06A0121BDE8F04701F02CBD14
:102EB00081681A463046BDE8F04700F02DB801F1B0
:102EC0000803120A81683046BDE8F04700F024B8D4
:102ED000B06A01F00FFDB06A0121BDE8F04701F0D2
:102EE00013BDB06A01F0BEFCB06A0021BDE8F04736
:102EF00001F00ABDB06A01F0ABFCD9F80810B06A65
:102F000000220909BDE8F04701F0CCBCB06A01F02D
:102F1000BFFC4AE7401F06602DE9F04FB1F1000801
:102F200083B08346914614BF0126002600934ED1FC
:102F3000002A00F097804FF0FF3A009B01241F1FEA
:102F4000731E019303E0631C4C451C4619D257F8CD
:102F5000045F002DF7D0AB07F5D12B79212BF2D1EF
:102F6000019BBAF1FF3FA9EB040203EB040A5146AF
:102F700069D1DBF8280001F04BFE631C4C451C4670
:102F8000E5D3BAF1FF3F53D0B8F1000F39D106EBCA
:102F90000904DDF8008008E00136D8F80010FFF7DA
:102FA000C9FE08F10408B4420ED056454FF00002A5
:102FB0005846F1D1D8F80030013608F10408996874
:102FC000FFF7B8FEB442F0D103B0BDE8F08F18F0BF
:102FD000030A03D198F80430212B21D0B9F1000F56
:102FE000A9D14FF0FF3A0121DBF8280001F004FEDF
:102FF000414600225846FFF79DFEB9F1000FC6D1A9
:10300000E2E7BAF1000FF3D14FF0000AD8F8081048
:1030100058465246FFF78EFEB9F1000FB7D1D3E7FD
:103020005146806A01F0F4FDB9F1000F85D1EBE75C
:1030300006EB0904DBF82800214601F0DDFDB8F1BC
:10304000000FA6D0D4E70A4815F024F9DBF80830C1
:10305000002BB9D102462946584603B0BDE8F04FCF
:10306000FEF74CBA806A03B0BDE8F04F01F0C4BD72
:103070005C1F06602DE9F843066905461F460C46AD
:10308000B31C06F10109806A31462B61904601F0BC
:10309000E9FA4946A86A01F0FDFCA1680022284629
:1030A000FFF748FE24692CB926E0A168FEF7DAFC98
:1030B000E4680CB394F804C0334600222846BCF1FF
:1030C000AC0FF2D0E168FEF773FC0121A86A01F0B1
:1030D000CBFC7B1C424621462846FFF7CBFFA86A63
:1030E000314601F031FCA86A494601F0BBFAA86AF2
:1030F000BDE8F84301F0DCBC41462846FEF758FC29
:103100006B6A1978062905D0BA00A86A053201F061
:1031100057FDE4E7A86A002101F0F0FDA86A01F07C
:10312000ABFBDCE72DE9F04F2DED028B8B6887B010
:103130000F46044603F00F03022B02D1CB68002B8D
:1031400046D125692046A94BD4F818A06E1C2B4304
:10315000B4F81E90668305F102082383A38BE383F2
:10316000EB1C2361F968FEF723FCA06A012101F042
:103170007BFC3146A06A01F075FA4146A06A01F075
:1031800089FC0022B9682046FFF7D4FD2046396942
:10319000FEF70EFCA06A01F071F9002800F0C7806C
:1031A0004146A06A01F05EFAA06A01F081FCC4F811
:1031B00018A0A4F81E9020467969FEF7F9FB29466D
:1031C000A06A07B0BDEC028BBDE8F04F01F04ABA2F
:1031D0009807B6D11A792B2AB3D19A6802F00F0159
:1031E0000229AED140F23E31B1EB121FA9D1DB680A
:1031F0001A792F2AA5D19B6805AAA32104A80493B4
:10320000FDF72EFC431E022B9BD8012800F0948072
:10321000022800F0978005998E68D1E9002BF1070C
:103220008FD573088DD02AB1930703D11179A539B1
:10323000022986D9BBF1000F08D01BF0030F05D17E
:103240009BF80410A53902297FF67BAFBB6825697E
:1032500008EE103A3B69A18B05F1010808EE903A9F
:10326000A369281D7F69029305F10209E38B05F12B
:10327000030A206101931BF001032583A4F81A803F
:10328000E183009300F0898011462046FEF790FB11
:103290005146A06A01F058FB4946A06A01F0E2F9E4
:1032A000A06A01F0D5FA002218EE101A2046FFF7A6
:1032B00041FD18EE901A2046FEF77AFB4146A06ABF
:1032C00001F0D0F931462046FEF772FBA06A0E21CC
:1032D00001F030FCA06A514601F0C4F9009BA06ADD
:1032E000002B53D101F0BEFAA06A01F0D1FA002EF2
:1032F000A06AACBF0021012101F01CFCA06A4A4673
:10330000012101F02FFB029BA06AA361019BE383D3
:10331000EFB9294601F0A6F9A06A01F0ADFA009BC9
:10332000002B41D007B0BDEC028BBDE8F08F3146D9
:10333000A06A01F009FB33E7059B03260246D3F898
:1033400000B077E7059B0326D3E9002B6BE701F07C
:1033500093FA009B63B339462046FEF729FB2669A2
:10336000A06A731C3146236101F0EEFAA06A0121C4
:1033700001F08AF8A06A294601F074F9A06A01F008
:103380007BFA3146A06A01F06DF9CBE701F060FAF3
:1033900059462046FEF70CFBA9E759462046039202
:1033A000FEF706FB039A6FE7A06A01F065FAB9E73A
:1033B000A06A01F061FA39462046FEF7F9FA26695B
:1033C000A06A731C3146236101F0BEFAA06A022193
:1033D00001F05AF82946A06A01F044F9A06A01F008
:1033E0004BFAA06A01F048FACBE700BF0080FFFF6C
:1033F0002DE9F043044683B016460D46002938D027
:1034000007697A1C0261D6F80080B8F1000F06D077
:1034100018F0030903D198F804207A2A2FD04146E6
:1034200020460193FEF7C4FAA06A0022394601F053
:10343000F7FAA06A01F020FA019BA08B626A0130C2
:1034400080B2A083918C814205F1FF3138BF908416
:10345000321D2046FFF7CCFFA06A394601F036FB4B
:10346000A38BA06A013BA38303B0BDE8F04301F046
:10347000EFBA194603B0BDE8F043FEF799BAD8F8A1
:1034800008100193FEF794FA4A463946A06A01F003
:10349000C7FA4A46D8F80C102046FFF74BFC019BB0
:1034A000CBE700BF30B50C4683B00546792101AAB1
:1034B00004F10800FDF7D4FAE3680146019A2846B2
:1034C000FFF796FF03B030BD2DE9F0410D46002611
:1034D00011460446456282B041712A460661806AFF
:1034E00000F0ECFE6379012B01D16E84AE84EE68AE
:1034F0000EB1B20732D02B78002B58D0072B3DD01D
:10350000022B00F08780DA1E032A55D86779D6F897
:103510000C80012F00F0B780032B00F0AD80042B4E
:1035200000F0C580052B00F0C980062B00F08D80CF
:1035300001212046FEF72EFA0121A06A01F094FA3B
:103540000023B26841462046FFF794FD2B78062BF6
:1035500057D11421A06A01F0B3F852E033793C2B23
:10356000C9D12046B168FEF723FAA06A01F0AEFB8C
:10357000A06A02B0BDE8F04100F04EBF6379012BB4
:103580005AD020467169FEF713FAA06A00F076FF60
:103590000028EDD1A06A142101F092F8A06A01F090
:1035A00095FBA06A02B0BDE8F04100F035BF31469E
:1035B0002046FEF7FDF9EDE76379012B6ED02F2150
:1035C0002046FEF7E7F92D212046FEF70DF9B168F8
:1035D000A06A090901F0F0F837212046FEF704F946
:1035E00031692046FEF7E4F90F212846FDF742FD38
:1035F0000378022BADD0428800230F21A06A00F08F
:1036000051FFA06A01F062FBA06A02B0BDE8F04180
:1036100000F002BF6379012B25D0F1682046FEF748
:10362000C7F92B7E5B07ECD5A06A01F025F91421C0
:10363000A06A01F045F8E4E70021244B432220462C
:10364000A171F168FDF77AFD9BE7A06A01F0D8F857
:1036500001212046FEF79EF9A06A01F0D1F8A06A88
:1036600001F0CEF86CE70022194B2046A2714B22E4
:10367000B168FDF763FDD0E701220021A06A01F0E7
:1036800081FA2B7851E70DF107023946606AFDF7A0
:10369000BBFC022303706F832B783DE70DF107021B
:1036A0000F212846FDF7B0FC0223037087E70322B1
:1036B0000021A06A01F066FA2B7836E70622002185
:1036C000A06A01F05FFA2B782FE700BFBD170160F9
:1036D000C51701602DE9F0410C4682B089680746A4
:1036E000FEF766F9E668A6B37568EBB28C2B7B6AC9
:1036F00032D01B7804F10C06072B69D00125002479
:1037000004E01C46FEF754F9A54222D9631CA2002E
:10371000384656F82410AB42F3D291F804C0BCF1FD
:10372000310FEED13244D2F8048098F804202F2AC9
:10373000E7D189680022B86A0234090901F06AF801
:10374000D8F80810002301223846FEF72BFDA542C9
:10375000DCD802B0BDE8F0811B782D0A0836072BB3
:1037600003D00024AC42D1D3F3E7A36803F00F02E7
:10377000022AF6D140F2D532B2EB131FF1D13368F1
:103780001A792F2AEDD19B68002BEAD10F213846F8
:10379000FEF700F97A6AD36A128D22B924E0013A61
:1037A00003F1080320D05978C907F8D5596838467D
:1037B000FEF7F0F8022D03D973681A79312A23D065
:1037C00000230221B86A01241A4601F063FAC9E70E
:1037D000A36803F00F02022A90D140F2D532B2EB77
:1037E000131F8BD10125CAE731681048019114F0ED
:1037F00051FDBB6802460199002BAAD1384602B0A0
:10380000BDE8F041FDF77ABEB46822792F2AD7D1FE
:1038100099680122B86A090900F0FCFFA168002339
:10382000012238460324FEF7BDFC9BE7781F0660A3
:1038300010B5436A82B004461B780191072B09D06A
:10384000022B07D0154814F025FDA3680199F3B1A8
:1038500002B010BD2046FDF7A1FE01992046FFF7FA
:1038600039FFA06A00220A2100F0D4FF0023A06AD9
:1038700019461A4601F01CFAA06A142100F020FF34
:103880000121A06A02B0BDE8104001F037BA02463B
:10389000204602B0BDE81040FDF730BE901F066024
:1038A0002DE9F843CE680D4604464EBB037943B973
:1038B000A9688D071BD001F00F03022B18D0BDE8BB
:1038C000F883436A1E78002EF2D13A21FEF762F89F
:1038D000A9682046FEF76CF8A06A334632460121FB
:1038E00001F0D8F9A06ABDE8F84300F0C5BFE9B916
:1038F0002046FEF75DF8A06ABDE8F84300F0BCBFC3
:1039000016F0030707D17168CBB2562B47D0572B5F
:103910005ED0062B0ED031462046FEF749F8A96846
:1039200020460022BDE8F843FFF704BA0B79392B93
:10393000DED1C4E7AF68002FEDD0B807EBD17B68CC
:10394000DAB2062AE7D1090A1A0AB1EB132FE2D13B
:10395000022AE0D1BB6823B1990702D11B79212B40
:10396000D9D0FB6823B19A0702D11B79212BD2D081
:10397000B1682046FEF71CF8F1682046FEF718F8FB
:10398000A06A00F085FFB96820460022FFF7D2F94F
:10399000F96820460022BDE8F843FFF7CBB90122C1
:1039A000A968FFF7C7F9F1682046FEF701F8B36888
:1039B0001B09563B0A2B2CD81C4AD15CA06A01F08B
:1039C000B9F8A96820460222BDE8F843FFF7B2B96A
:1039D0004FEA112808F1010308F1FF3956F82310C6
:1039E000FDF7E6FFB9F1000F99DDA06A00F030FFA6
:1039F000A9683A462046351DFFF79CF901374F4527
:103A000009D156F8281020460022BDE8F843FFF7F8
:103A100091B91421D2E7A06A00F01AFF002255F8EC
:103A2000041F2046FFF786F9E8E700BFB81F0660CD
:103A30002DE9F04F85B0044615460191002900F0AC
:103A4000B4800669321D06F1010A06F1020906F189
:103A500003080261D5F800B0BBF1000F07D01BF0DE
:103A6000030204D19BF804107A2900F0A48059467F
:103A700020460293FDF79CFF2F6820463F093946F8
:103A8000FDF7B2FE39462046FDF784FF20460521AA
:103A9000FDF770FCA06A00F0EFFE029B394620465D
:103AA0000293FDF777FFA06A0022062100F0B2FE24
:103AB0003146A06A022200F0B3FFA28B616A013294
:103AC000029B92B2A283888C9042204638BF8A849F
:103AD0002A1D01990139FFF7ABFFA06A00F0ECFF46
:103AE0004946A06A00F030FF3146A06A00F0BAFDF6
:103AF000A06A01F013F9A06A00F0AAFE00220F21CB
:103B0000A06A00F0CFFEA06A00F0C2FEA06A1421F5
:103B100000F0D6FD00230321A06A1A4601F0C8F880
:103B20002046FDF74FFB5246A06A012100F01AFF24
:103B3000A06A002101F0D6F85146A06A00F092FD7B
:103B4000A06A00F0E1FF4146A06A00F0FDFE0321FB
:103B5000A06A00F099FCA38BA06A013BA38300F04C
:103B600077FFA06A01F0DEF84946A06A00F07AFD0E
:103B70001421A06A00F0A4FDA06A00F069FEA06A0A
:103B800000F066FE00230321A06A1A4601F090F8B7
:103B90002046FDF717FBA06A00F06EFE4146A06AC2
:103BA00005B0BDE8F04F00F05DBD194605B0BDE8B9
:103BB000F04FFDF7FDBEDBF80810CDE90232FDF74E
:103BC000F7FEDBF8087020463F093946FDF70CFE8A
:103BD00039462046FDF7DEFE20460521FDF7CAFBEB
:103BE000039ADBF80C102046FFF7A4F8029B55E778
:103BF0002DE9F04F8D6887B004462B792946032BB9
:103C000000F0C380162B14D0FDF7C8FC10B907B024
:103C1000BDE8F08F05AA792105F10800FCF720FF27
:103C2000EB680146059A2046FFF702FF07B0BDE8A2
:103C3000F08FFDF7B3FC0028E9D026692046EB6839
:103C400006F1010B06F1020A4FEA1318331D236136
:103C5000E968FDF7ADFEA06A0022072100F0DAFD59
:103C60000023A06A1A46194601F022F84146204670
:103C7000FDF7BAFD2769A269A38B07F1010901923B
:103C8000BA1C4946A06A2261E28B2783E383A4F829
:103C90001A90029200F0E6FC5946A06A022200F057
:103CA000BFFEA28B616AF31C0132039392B2A2831E
:103CB000888C9042204638BF8A844146FDF76AFED0
:103CC00020460921FDF756FB0022A9682046FFF790
:103CD00031F8A06A00F0F0FE5146A06A00F034FE10
:103CE0005946A06A00F0BEFCA06A01F017F8A06A6D
:103CF00000F0AEFD0122A06A4FF49F7100F0ECFBD2
:103D0000A06A082100F016FF039B0021A06A1A4652
:103D100000F028FEA06A00F0AFFDA06A00F0F4FEFB
:103D20003146A06A00F010FE039BA06A194600F01D
:103D300099FC0121A06A00F0A7FBA38BA06A013BBC
:103D4000A38300F085FEA06A00F0ECFF5146A06A54
:103D500000F088FC20462969FDF72AFE4946A06A42
:103D600000F0F2FD019B3146A06AA361029BE38350
:103D700000F078FC20466969FDF71AFE3946A06A12
:103D800007B0BDE8F04F00F06DBCFDF73BFDAA6940
:103D9000137E43F01403137607B0BDE8F08F00BF25
:103DA0002DE9F04F8FB00D4682460021019204A804
:103DB00028221C4648F0B8FE4FF0FF32019B00213C
:103DC000099203A8DAF8002003958DF81040FDF75A
:103DD000E3F9044600F05AFA0B9F05460D90002FB8
:103DE00000F0308100260AE03946012203A8FFF7DF
:103DF0006BFB079BBF689E4238BF1E4617B1059BF1
:103E0000002BF1D00B9B002B00F0C4804FF0010E73
:103E1000A346059C002C40F0BC801A7E198DD20769
:103E200017D5481E002900F00B81DF6A07EBC10798
:103E300001E001380DD317F8072C083F12F0020FEC
:103E400040F0E280002CF4D1012A08BF3C46013842
:103E5000F1D24FF000021A8400293ED00022A84679
:103E60000BE0C15D16D9A9B900F807E06178CD076C
:103E700012D4198D01328A4216DA93F800C0D700A5
:103E8000D86ABCF1010F00EBC204EAD165680F2DBE
:103E9000F0D0C15D0229E9D1198C0132481C188487
:103EA0006180198D8A42E8DB4546B1B1002202E00B
:103EB00001328A4211DAD86A10F8324000EBC200AF
:103EC000032CF5D14478E407F2D4198C01324180F7
:103ED000481C198D18848A42EDDB5F68002F54D08E
:103EE0003A8D002A51D00024A44604E00CF1010CC4
:103EF0003A8D944528DAF86A10F83C2000EBCC089B
:103F0000033A012AF2D80029F0D00022A94602E0A3
:103F100001328A4211DAD86A10F8327000EBC2001E
:103F2000042FF5D14768D8F80450BD42F0D1448041
:103F30000132198D01348A42EDDB5F680CF1010C0E
:103F40004D463A8D9445D6DBFCB11FFA84F9A9B1F0
:103F5000002206E06188013249446180198D8A425D
:103F60000CDAD86A00EBC20410F832000428F1D150
:103F70006078C007EED401328A42F2DB5A8B198C8A
:103F80004A4489445A83A3F820909B68002B7FF40D
:103F900040AF5C463146284600F07CF90B9E059BFD
:103FA00066B123BB0222314603A80D95FFF78CFAB8
:103FB000059B002B35D0B668002EF2D1BBB9284640
:103FC00000F072F95046FCF7DFFF65692046A468EF
:103FD000FDF710F8002CF9D10598002834D12246BD
:103FE000214628460FB0BDE8F04F01F031BC0C9BD4
:103FF00003A8D968FDF778FA0C9B069A5B8A0399A7
:10400000059805F089FBDAE7002C3FF422AF97E82A
:104010000300D4E9008284E80300C7E90082198D17
:1040200017E70322314603A8FFF74EFA059B002B42
:10403000C1D10422314603A8FFF746FA059BBAE72F
:104040001C844AE73E46A5E7F8F706FA30B583B088
:1040500004460D460DF10702FCF7D6FF9DF8073028
:104060000BB903B030BD01462A462046FDF72EF8B5
:1040700003B030BD10B582B004460DF10702FCF765
:10408000C3FF9DF8073033B12378012B0CD90223ED
:10409000037002B010BD2378012BFAD90378002BEE
:1040A000F7D102230370F4E70023037002B010BDC0
:1040B00070B506460D46104619461C46FCF7DAFF59
:1040C00002786AB1012A0BD0022A2D684288214663
:1040D0003046AC460CBF00230123BDE8704060476A
:1040E0006B6821463046BDE87040184770B582B015
:1040F0000B460DF1050C664602F07F04D2093546E9
:1041000006F8014DF8D1ACEB0601984701A98E42A3
:104110000CD02B46024601E013F8014B64F07F04FB
:104120008B4202F8014BF7D19B1B18449DF80430D9
:10413000037002B070BD00BF42790346032A026AD1
:1041400002D8114419627047006B1144104419627F
:10415000704700BF10B442790346032A05D8826A2B
:10416000114499625DF8044B7047D0E90924006B53
:1041700021442244996210445DF8044B704700BF0B
:1041800030B5054683B00C4601210192FFF7E2FFEE
:10419000019A0346034928461C7003B0BDE830402D
:1041A000FFF7A4BF5541016090F805C0BCF1040FB2
:1041B00010B402D1C46B44F822305DF8044BFFF711
:1041C000DFBF00BF30B5C4681346C58E628BA48BB9
:1041D000B0F838E022442A4472440EF1010EA0F8EF
:1041E00038E0BDE83040FFF7DFBF00BF2833D9B269
:1041F000FFF7C6BF38B514460D460321FFF7AAFFE7
:104200000570230A4470837038BD00BF70B54379D0
:104210000D46032B11D9C3696FF00204032153F833
:104220002230826AA41A1C44FFF794FF0570E6B29C
:10423000C4F307244670847070BD00240321FFF787
:1042400089FF057026468470467070BD70B543794D
:104250000D46032B11D9C36947F6FD74032153F8AA
:104260002230826AA41A1C44FFF774FF0570E6B27C
:10427000C4F307244670847070BD00240321FFF747
:1042800069FF057026468470467070BD002140208D
:10429000F8F724B90B46002110B504469800A36135
:1042A000F8F700F9E06110BD10B50446C069F8F7F1
:1042B00025F92046BDE81040F8F720B92DE9F04176
:1042C00000230124154641714461064683600F4670
:1042D0008371836203624F49C0E903236B8C128CA4
:1042E0001A44A24238BF2246FFF700FFAA8C494970
:1042F0003046FFF7FBFEF3682146304693F81880FE
:10430000FFF71AFF214680F800803046F36893F8E3
:104310001A80FFF711FF214680F800803046F368CD
:1043200093F81C80FFF708FF214680F80080304694
:10433000F3689C7FFFF700FF042F04703AD002213E
:104340003046FFF7F9FE6C8A02213046FFF7F4FE93
:104350000470240A0221447030462C8AFFF7ECFED8
:104360000470240A4470288DB0B1002401E0A042FA
:1043700012DDEB6A13F8342003EBC4030134032A83
:10438000F5D193F8028001213046FFF7E3FE80F873
:104390000080288DA042ECDC01213046FFF7DAFED8
:1043A000FF23042F03704FF00000B086308709D040
:1043B000BDE8F081D6E9083216493046D21AFFF737
:1043C00095FEC0E76B8BAA8BD342F1D02C8D74B1D4
:1043D000EB6A002193F801C001311CF0010F02D0FB
:1043E0005A88824210D0A14203F10803F2D140F270
:1043F0008623F26B42F8203001306B8BAA8B13447A
:104400008342E3DCBDE8F0815B68DB0043F0060338
:10441000EFE700BF3941016070B543790446012BD5
:104420000BD000250121FFF787FE05706379A28E6E
:10443000032BE2860BD0042B00D070BDE068E26B4A
:10444000216B037E4069BDE8704001F0F1B9A36AB9
:104450002946206AE36260621844F8F73FF8E3688F
:1044600020632946588B9B8BA28E1844238F1044BF
:1044700018448000F8F732F8E06370BD80790038A6
:1044800018BF0120704700BF4379012B09D0D0E944
:104490000223114481605A8C9142C8BF5984002381
:1044A0008371704770B51D46012106461446FFF71B
:1044B000EBFF3DB90F2C05D8503C0121FFF74AFE18
:1044C000047070BD05F1190122463046C9B2BDE83D
:1044D0007040FFF755BE00BF10B5144682B00B46C2
:1044E00001211B340193FFF7CFFF019AE1B202B023
:1044F000BDE81040FFF77EBE70B51D464FF0FF319E
:1045000006461446FFF7C0FF3DB90F2C05D8403CC6
:104510000121FFF71FFE047070BD05F12201224644
:104520003046C9B2BDE87040FFF72ABE10B5144648
:1045300082B00B464FF0FF3124340193FFF7A4FF04
:10454000019AE1B202B0BDE81040FFF753BE00BFD0
:1045500010B5144682B00B4600212A340193FFF7B0
:1045600093FF019AE1B202B0BDE81040FFF742BEEE
:1045700070B51D46049E059B1446491BA1EB4601E0
:1045800053B10239FFF780FF611C45EA0622C9B228
:10459000BDE87040FFF7F4BDFFF776FF45EA06225D
:1045A000E1B2BDE87040FFF7EBBD00BF2C4B2DE939
:1045B000F047D3F8E83081460F46022B02D8446911
:1045C0008C4201D3BDE8F087856A0C1B036940F279
:1045D000FF78ED1A062C24D9444526464FF00201F7
:1045E000484628BF46460F2D94BF4FF0000A4FF0B3
:1045F000010ABAF1000F14D1FFF79EFDA41B46700B
:104600003609234606F070062E43554666F07F06AF
:104610000670002BDED1D9F82830C9E90437BDE88F
:10462000F0871F2DAA464FF0000628BF4FF01F0A43
:10463000AA4506D3032C264628BF0326A41B7601D1
:10464000F6B2A5EB0A050121484646EA0A06FFF73D
:1046500073FD44EA05030670002BBBD1DBE700BF06
:104660000004002038B50D460021FFF70DFF437907
:10467000032B05D8012B03D0826AC36943F8252098
:1046800038BD00BF012A70B5144605460E460BD052
:104690004FF0FF31FFF7F8FE022C08D10121FFF7A0
:1046A00059FD6A23037070BD1146FFF7EDFE6834B3
:1046B00032462846E1B2BDE87040FFF79BBD00BF1F
:1046C00070B50C460121FFF7DFFE142C11D0152C1C
:1046D0001BD0132C13D0C2681721538B928B134419
:1046E000828E541C1A440C4B8486BDE87040FFF740
:1046F0005BBD0121FFF72EFD1123037070BD012169
:10470000FFF728FD1023037070BD0121FFF722FD84
:104710001223037070BD00BF9045066070B50C4653
:1047200082B001210646FFF7AFFE04F1100301211C
:104730003F2B05D8803CFFF70DFD047002B070BD23
:10474000FFF708FD0DF1050114230D46037004F079
:104750007F03E2B2E411AC4605F8013D631C012B76
:10476000F5D8013419D053061FD401AC491B30468B
:10477000FFF7F0FCA5420BD001462A4612F8013B98
:1047800063F07F03A24201F8013BF7D1521B1044B2
:104790009DF80430037002B070BD5206E5D47F234B
:1047A00005F8013CACF10205DFE7002305F8013C08
:1047B000ACF10205D9E700BF00B50A4683B001217C
:1047C0000192FFF761FE019A162103B05DF804EB38
:1047D000FFF710BD10B50B4682B001210193FFF722
:1047E00053FEC168019B4A8B898B0A44818E0A441F
:1047F00001318186172102B0BDE81040FFF7D4BC1B
:1048000008B50121FFF740FE0121FFF7A3FC1823A3
:10481000037008BD10B582B0144601915100C1F17A
:104820000101FFF731FE002C019A14BF1F211E2148
:1048300002B0BDE81040FFF7DDBC00BF08B50121A4
:10484000FFF722FE0121FFF785FC2023037008BD3E
:1048500008B50121FFF718FE0121FFF77BFC30238B
:10486000037008BD08B50221FFF70EFE0121FFF716
:1048700071FC3123037008BD08B54FF0FF31FFF71D
:1048800003FE0121FFF766FC3223037008BD00BF61
:1048900008B50021FFF7F8FD0121FFF75BFC33238A
:1048A000037008BD13460A4610B5044682B073B1C2
:1048B000022B17D06FF0010120460192FFF7E4FDB3
:1048C000019A262102B0BDE81040FFF793BC019188
:1048D0001946FFF7D9FD019A1D2102B0BDE810402D
:1048E000FFF788BC0191FFF78BFF2046FFF7D0FF51
:1048F000019ADFE708B50021FFF7C6FD0121FFF7A8
:1049000029FC3423037008BD10B5044661B10229A7
:1049100014D06FF002012046FFF7B6FD0121FFF72A
:1049200019FC2723037010BD4FF0FF31FFF7ACFDDA
:104930000121FFF70FFC2123037010BDFFF760FF7B
:104940002046FFF7D7FFE4E700B50A4683B0002111
:104950000192FFF799FD019A352103B05DF804EB50
:10496000FFF774BC10B50C4682B04FF0FF310192D6
:10497000FFF78AFD019A2CB1362102B0BDE8104044
:10498000FFF764BC372102B0BDE81040FFF75EBC02
:1049900010B50C4682B04FF0FF310192FFF774FD65
:1049A000019A2CB1382102B0BDE81040FFF74EBC8F
:1049B000392102B0BDE81040FFF748BCF8B5064603
:1049C0000C46154662B91146FFF75EFD230418D464
:1049D00024F4004230463521BDE8F840FFF736BCEC
:1049E00021F400424621FFF731FC0121230A304621
:1049F00023F07F0343EA0502D4B2FFF7ABFB047058
:104A0000F8BD322703250121FFF7A4FB0770012120
:104A10003046FFF79FFB013D0770F8D1D8E700BF94
:104A200030B583B01446054601915AB90221FFF70B
:104A30002BFD019A3D342846E1B203B0BDE8304079
:104A4000FFF7E4BB0021FFF71FFD019AF2E700BF6B
:104A500008B54FF0FF31FFF717FD0121FFF77AFB93
:104A60004123037008BD00BF38B5044649B1032196
:104A70004725FFF709FD01212046FFF76BFB057075
:104A800038BD4225FFF700FD01212046FFF762FBFC
:104A9000057038BD00B50A4683B001210192FFF7C9
:104AA000F3FC019A432103B05DF804EBFFF7AEBBC2
:104AB0006FF00301FFF7E8BC08B50021FFF7E4FC45
:104AC0000121FFF747FB4423037008BD38B50446B6
:104AD0000D46FFF7F1FF14212046FFF7F1FD2046B8
:104AE0002946FFF7BFFD0221FFF7CEFC0121FFF7AA
:104AF00031FB3E2203466FF0030120461A70BDE8E9
:104B00003840FFF7C1BC00BF08B50021FFF7BCFC6F
:104B10000121FFF71FFB4523037008BD10B50C46AC
:104B20000021FFF7B1FC0121303CFFF713FB0470BB
:104B300010BD00BF302938B50C46054620D03129BC
:104B400009D04FF0FF31293CFFF79EFC0121FFF710
:104B500001FB047038BDDE244FF0FF312846FFF71B
:104B600093FC0121FFF7F6FA0346002128461C704A
:104B7000FFF78AFC0121FFF7EDFAD323037038BD5C
:104B8000DD24E9E770B514460D46032A04F150040C
:104B900014BFC5F101010121FFF776FC2A46E1B2FD
:104BA000BDE87040FFF7ECBA08B56FF00101FFF700
:104BB0006BFC0121FFF7CEFA5423037008BD00BF40
:104BC000032938B5144612D004290BD002254FF022
:104BD000FF31FFF759FC572145EA8402BDE8384010
:104BE000FFF7CEBA013401256FF00101F1E700258E
:104BF0004FF0FF31EDE700BF10B50C460139FFF76C
:104C000043FC59212246BDE81040FFF7B9BA00BF66
:104C100038B515460C461144FFF736FC5A2144EAD4
:104C20000522BDE83840FFF7ABBA00BF134310B50B
:104C30000C4608D10121FFF727FC62696021BDE81D
:104C40001040FFF7BFBA4FF0FF31FFF71DFC62695C
:104C50006121BDE81040FFF7B5BA00BF70B514463A
:104C6000049A05460E4613430DD1C4F10101FFF726
:104C70000BFC72696221FFF7A5FA01212846FFF7B4
:104C800069FA047070BDE143FFF7FEFB72696321AE
:104C9000F1E700BF30B5154683B01C4664220B46D1
:104CA0000021CDE90054FFF763FC03B030BD00BF25
:104CB00030B5154683B01C4666220B464FF0FF31D7
:104CC000CDE90054FFF754FC03B030BD4FF0FF3185
:104CD00010B5FFF7D9FB01218171FFF73BFA5B2388
:104CE000037010BD10B50C464942FFF7CDFB022101
:104CF000FFF730FA5C234470037010BD38B50C46E2
:104D00004942FFF7C1FBC2685D340121137E43F0C5
:104D100004031376FFF71EFA047038BD0421FFF771
:104D2000B3BB00BF6FF00201FFF7AEBB2DE9F04F40
:104D3000062985B09DF8384040F2A780B4EE400ABD
:104D4000F1EE10FA80F19A8010EE105A002D80F2E8
:104D50009580B1EE400A84462D2401390CF8014BB0
:104D6000F0EEC07A9FEDC57A02F02006F4EE477AA5
:104D7000F1EE10FA00F3E481B4EE400AF1EE10FA1D
:104D800080F18882002B01F1FF3542F0200EC0F245
:104D90008B80AEF1670A46F04502BAFA8AFA0392AE
:104DA0004FEA5A1A002B14BF4FF0000B0AF0010B08
:104DB000BBF1000F00F0828010EE103A1A1E40F096
:104DC0001881062D00F3DA81CB1F4FF0670E002407
:104DD000DA4623EAE3724FF0010B27462646019498
:104DE000BEF1670F00F0C481002AD4BF4FF0000A63
:104DF0000AF0010AB44280F25581BBF1000F40F085
:104E00005181BAF1000F0ED01CF8012C302A06D1C6
:104E10000CF1FF339C4613F8012D302AFAD02E2ACC
:104E200008BF0CF1FF3C019B03B3039A0CF1040C87
:104E30000CF8033CF3170CF8042C914A82FB064152
:104E4000C3EBA10382FB0321DA17C2EBA10202EB41
:104E50008202A3EB420203EB8303A6EB430602F1BB
:104E6000300330360CF8023C0CF8016C0023ACEB3C
:104E700000008CF8003005B0BDE8F08F002C6FD03A
:104E8000844601390CF8014B6AE7012940F254814C
:104E90003F2300F8013B00230370012994BF002049
:104EA000012005B0BDE8F08FAEF1670A46F045037A
:104EB000BAFA8AFA039306234FEA5A1A10EE102A16
:104EC000002A4FD0BEF1660B18BF4FF0010BB2F1B4
:104ED0007E5FC0F097806B4A2024DFED6B7A00265E
:104EE0006A4F02F1140801E0F2EC017AF4EEC07AA4
:104EF000F1EE10FA04D8D7ED007A264420EE270A06
:104F000090454FEA640407F10407EDD1FDEEC07A45
:104F100017EE902A092A04DDDFED5D7A013620EED6
:104F2000270ABEF1660F00F08781BEF1650F00F021
:104F3000EA80BEF1670F40F0E3811A1DAA4200DB50
:104F40008B1F9E4280F2D681721C9B1A23EAE37269
:104F5000F4180023013437464FF0660E019311E038
:104F60008446FDE6BEF1660F40F085815C1CAC42D4
:104F700080F23F814FF0000B23EAE3725F465E460A
:104F8000CDF804B0002C7FF72FAF002AD4BF4FF02C
:104F900000084FF001080AEA080A0246B2EE047A55
:104FA000404600234FF02E09904602960BE00CF885
:104FB000019BF8EEE77A0133A34230EE670A20EE58
:104FC000070A80F2B680FDEEC07A30210CF10102B2
:104FD00017EE905A17EE906A0D44002EA8BFE9B262
:104FE000BB428CF80010944601D10028DFD19446D2
:104FF000DFE7B2F17E5FDA464FF0670E4FF0010354
:10500000BFF469AF9FED237A2024234A0026B4EE33
:10501000C70ADFED227A224F02F11408F1EE10FAEE
:10502000ACBF4FF031094FF0300901E0F2EC017AEA
:10503000F4EEC07AF1EE10FA04DDD7ED007A2644E2
:1050400020EE270A90454FEA640407F10407EDD1EA
:1050500010EE102AB2F17E5F80F09480DFED0D7AC1
:10506000B4EEE70AF1EE10FAC0F2C680002EB7EEF9
:10507000000A14BF2D222B22019285E0FFFF7F7FC3
:1050800067666666EC200660AEC59D74D02006603B
:10509000CDCCCC3DF8FF7F3FD42006601FB14F0A36
:1050A000E8200660F1EE047AB4EEE70AF1EE10FAB9
:1050B000FFF6A7AE0CF1FF323025114612F8013988
:1050C0002E2BA3F13004F8D0092C00F2AF80392B3D
:1050D00040F0C58081425570EFD101464B782E2BB0
:1050E00003D1BEF1660F40F0EA800CF1010C8C4553
:1050F00006D9634613F8012C03F801298B42F9D134
:1051000031230B707DE68A1F9A427DDD23EAE3722C
:105110002B230193002A02F101044FF000074FF006
:10512000650ED4BF4FF000084FF0010808EA0A0AE4
:1051300033E7029E40465DE600293FF4AEAEAAE6A4
:1051400086F0490386F04E0286F046048CF8003063
:105150000CF103038CF802408CF801200022181A8D
:105160001A7005B0BDE8F08F24EAE47223460027E8
:10517000002B38DD14464FF0670E03E74FF0670E43
:10518000012324E62D220192BEF1660F63D0042E86
:105190003CDCBAF1000F39D06446BEF1670F04F869
:1051A000019B01D1721E13445A1CAA425ADBCB1E2A
:1051B0002E22013E0CF1020C0CF8012C00F0918023
:1051C0001C46302201E0002C71D0013E04F1FF3476
:1051D0000CF8012BF7D123EAE3724FF0FF374FF0C1
:1051E000660E0196CEE64FF001084FF0670E44467A
:1051F000D3E6CB1E8C1EBDE6F2EE047A2D220136DC
:10520000019220EE270ABFE7CB1F7FE78C1F9C424D
:1052100003DCBEF1670FA7D0CB1FBEF1650F23EAF9
:10522000E3723FF477AF00242746D9E54B78302B63
:105230007FF4E7AD013151E7AE42BFF664AFF41839
:10524000621CAA4239DBAD1B012DA5F1020340D03F
:105250001A46F4187DE6644604F8019BA4E701337E
:105260000B70CEE5002BA3D1A4461A464FF0660E74
:105270001C460193B8E55A1D9542D8BFCB1FBEF11D
:10528000650F24D123EAE3722B234FF0010B002694
:1052900001933FE746F04E0286F041040CF1030310
:1052A0008CF800208CF801408CF8022056E723EAA5
:1052B000E3724FF0660E019496E51A4649E60B70CC
:1052C00030234B70019B2D2B06D001360FE7D346C0
:1052D0007DE5002234463CE6013E08BF2B230193C6
:1052E00005E723EAE3721C464FF0FF374FF0660EE6
:1052F000019647E62B2123EAE3720027019137E765
:1053000000242B211A462746019169E501291368DB
:1053100009D933F0100190F800C009D1BCF1300F69
:1053200015D0082B19D0C3B90A2300201360704789
:10533000082B14D0022B10D1BCF1300F0DD14378C3
:1053400043F02003622B14BF0020022070474078F6
:1053500040F02000782815D063B100207047BCF1E0
:10536000300FFAD1437843F020036F2B14BF002095
:10537000022070476F2809D06228D5D10223184631
:105380001360704710230220136070470823022027
:1053900013607047044608B531B1054A0023026026
:1053A0004A6C096804F0B8F92046F7F755F800BFD1
:1053B000E43506602DE9F04FB2F1000A85B00646EB
:1053C000984618BF4FF0010A012A00EB010701922D
:1053D000C8BF4FF0000A242AC8BF4AF0010ABAF138
:1053E000000F79D1B84212D2044602E0A742264605
:1053F0000DD0264614F8010BF8F7CAFE0028F5D1A7
:10540000B74204D933782B2B61D02D2B53D0B91B45
:10541000304601AAFFF77AFF0644B74261D9344605
:105420000025A14614F8013BA3F1300BBBF1090F95
:1054300009D95F2B14D043F02003A3F16102192A8C
:1054400011D8A3F1570B019959450CD928460EF0F4
:1054500021FA019B28BB05FB03B595EA450220D440
:10546000A742A146DDD8BAF1000F00D06D426D0011
:1054700045F00105B14534D0B9450CD24C4602E0A7
:10548000BC42A14607D0A146013499F80000F8F7C4
:105490007FFE0028F4D14F4523D1284605B0BDE852
:1054A000F08F5246B91B03A8039605F0A5FBDDF863
:1054B0000C900546DEE7013601AAB91B3046FFF71E
:1054C00025FF0644BE4204D24FF0010AA7E7264654
:1054D0009DE7B1460125CDE7074812F0DBFE00F05D
:1054E0008FFC064812F0D6FE019A0146044804F0EB
:1054F000BBF84146FFF74EFF0021066024210660FD
:10550000103706602DE9F04F04469146984666181C
:105510002DED028B83B0B4420E98019080F02D8166
:10552000A24603E05645544600F0BB8057460AF1B8
:10553000010A3878F8F72CFE0028F3D1BE4240F279
:1055400053813B782B2B00F0D2802D2B00F0128161
:1055500005463B7843F02002692A00F0DA806E2A83
:1055600000F0F2804FF0000EF2EE046A9FEDA28A86
:105570003C469FEDA27A7046F446724619E0022A34
:1055800000F08380B4EEC78AF1EE10FA40F1858016
:1055900007EE90AA012AF8EEE77AE8EE267AB0EE56
:1055A000678A00F0948000228E4240F220810B78BE
:1055B0000C46A3F1300A611CBAF1090FDFD9002AA9
:1055C00008BF2E2B0CBF4FF0010A4FF0000A5AD033
:1055D000022A04D043F0200BBBF1650F48D0B9F18B
:1055E000000F05D043F0200BBBF16A0F00F0D7800D
:1055F0005F2BD9D0BEF1000F00F0ED80A0EB0C00C6
:1056000010F1250F53DA2530DFED7D7A07EE100A11
:1056100028EE278AF8EEC70AB2EE040A34F06CFED0
:1056200028EE008A002D54D1BC4268D0B4420AD280
:10563000254601E0B54208D02C4601352078F8F720
:10564000A7FD0028F6D1B44259D1BAF1000F43D1D9
:10565000B8F1000F30D118EE103A23F0030040F0FB
:105660000200A0F1FF4003B0BDEC028BBDE8F08F5B
:105670008E4243D963782B2B00F08F802D2B00F0C6
:105680008580022293E701228EE75E4B9C458BDCEE
:105690000CEB8C0C0AEB4C0C86E7002AF3D10130A2
:1056A00082E7002537469FED548A2846AA4607EE32
:1056B000900AF8EEE70AAFE7B0EE480ADFED4E0ACF
:1056C00003B0BDEC028BBDE8F04F03F079B90138AF
:1056D0006AE7B1EE488AA7E7F0EE480A9FED460A6E
:1056E00003B0BDEC028BBDE8F04F03F069B905468D
:1056F0005746B245FFF42DAF54463FE072D14248C1
:1057000012F0C8FD0146414803F0BCFF0199FFF7C4
:1057100041FEBB1C9E42F2D97B7843F020036E2BE6
:10572000EDD1BB7843F02003662BE8D1FB1DFC1CB8
:105730009E4204D9FB7843F02003692B32D09FEDC1
:10574000348A4FF0000A6DE7BB1C9E42D7D97B78A4
:1057500043F02003612BD2D1BB7843F020036E2BA2
:10576000CDD12C48FC1C47F0F3F94FF0000AB0EE05
:10577000408A57E757460125BBE70025DFED1E0AA3
:1057800027464FF0000AB0EE608A45E7A11C4FF0B3
:10579000010EB142B3D0022206E7A11CF9E7CA46C6
:1057A0000C4627E73B7943F020036E2BC7D17B796A
:1057B00043F02003692BC2D1BB7943F02003742B43
:1057C000BDD1FB799FED128A43F02003792B04D0E1
:1057D0004FF0000A26E7604412E707F108044FF093
:1057E000000A1FE70C4605E705463C46C6E70C469F
:1057F0004FF0000AFEE600BF00000000EC78AD604C
:10580000EA1C0802646666064C21066010370660D2
:105810000000807F387007600021102008B5F6F77F
:105820005DFE0121027861F30202027008BD00BF33
:10583000B0F800C003F07F03C0E90112DB002CF4D4
:105840007F7243F0020322F0030213430380704788
:1058500010B5044608461146237803F00703022BCF
:105860000FD1D4E9012304F023FB2388C3F3C6013D
:105870009B0600D410BDC1F30011BDE8104004F038
:10588000E9BB024812F006FD00F09EFA68210660AE
:1058900038B5154611F480720C460CBF1146D5E997
:1058A0000012FFF7D5FF6209E1B202F008022A44B4
:1058B000BDE8384002F008BF08B5024812F0EAFC23
:1058C00000F082FA7C21066070B505460C464AB1AC
:1058D0008E18D5E900039847431C04D004F8010B47
:1058E000B442F6D170BDFFF7E7FF00BF38B5002521
:1058F0000446D4E900039847421C07D000F07F0318
:1059000043EAC5150306F4D4284638BDFFF7D4FF93
:10591000B0B500AF0546FFF7E9FF04462846E31D92
:10592000224623F00703ADEB030D6946FFF7CCFFDA
:1059300021466846F7F756FDBD46B0BD2DE9F04F4C
:105940008DB00546FFF7D2FF80460021F6F7AAFD8D
:105950004246014682462846FFF7B6FF06A8CDF824
:1059600018A00DF009FB06A80DF006FB069B5A1CBB
:10597000191DDC1C06921A4612F8020BCDE905022D
:1059800007A85E7806949F78CDE906110DF0F4FA29
:10599000069908440130069010F8013CFF2BF9D11C
:1059A0002846D044FFF7B4FF04462846FFF7B0FF6F
:1059B000079B020A1C70240A079B5C70079B987067
:1059C000079BDA70069C444516D20DF1200903E0CE
:1059D000089B1C44A0450FD9494620460DF0DCFC2D
:1059E0000128F5D12846FFF793FF6070000AA070E8
:1059F000089B1C44A045EFD828463E44FFF776FF9D
:105A000080462846FFF772FF81464044002130441B
:105A10008000F6F747FD0490002E75D0049C04EB3F
:105A200086062846FFF774FFC00040F0060044F8E1
:105A3000040BB442F5D1B8F1000F3ED000272EE0A0
:105A40000DF1200B2846FFF751FF01460390584601
:105A5000F7F74AFE039A0A992846FFF735FF732C99
:105A600043D0A4F16203B3FA83F35B09002B3CD16A
:105A7000692C43D0A4F16302662CB2FA82F24FEA99
:105A8000521201D0002A41D00023DDE90910009311
:105A9000FFF738FD013746F8040BB8450DD0D5E9BE
:105AA00000039847431C31D0C4B2652CC8D10137DC
:105AB0001748B84546F8040BF1D1B9F1000F08D0EA
:105AC000002401342846FFF739FF46F8040BA145AE
:105AD000F7D1FFF7A1FE04465146DDE90423FFF7A5
:105AE000A7FE20460DB0BDE8F08F0A4B59460A4884
:105AF000732C18BF184607F013FACBE70A22DDE92A
:105B00000910FFF757FCC5E7064694E7FFF7D4FEF8
:105B100090450660044B0660984D066010B504225F
:105B200082B004460DEB0201FFF7CEFE9DF8043073
:105B30004D2B16D19DF80530032B12D19DF8063060
:105B4000022B0ED19DF807301F2B0AD82046FFF7F5
:105B5000F5FE0346A26820681C469047204602B026
:105B600010BD024812F096FB01F030F8902106605B
:105B700000B585B0014601A80FF0D0FE01A8FFF7DF
:105B8000CDFF05B05DF804FB70B5144CF7F7D0FB02
:105B900000251349134B04F16806134A04F154001D
:105BA000236562646566C4F8E850C4E90D150321F5
:105BB000C4E90F53C4E9125503F074FA01213046C9
:105BC00003F070FA4FF4AF724FF4BF71304647F0F4
:105BD0001BF8C4F89850C4E9056670BD00040020A5
:105BE000143306601C500660F4340660704700BF32
:105BF00070B50546134E0022EC00B06944F006046F
:105C00000430214646F0F8FF08B1406870BDD6F870
:105C1000983033B102462146181D46F0EDFF0028AA
:105C2000F3D100222146084846F0E6FF0028ECD1D7
:105C3000064812F02FFB2A460146054803F014FDE2
:105C4000F6F70AFC0004002024590660F8210660DB
:105C50000434066038B50A4B0446D3E905539D4227
:105C600009D0C1000022281D41F0060146F0C4FF02
:105C700008B1406838BD2046BDE83840FFF7B8BFDE
:105C80000004002008B5074BD3F8980038B1002273
:105C90006621043046F0B0FF08B1406808BD0248F4
:105CA00008BD00BF00040020E4570660C100034B9C
:105CB00041F00601586903F0ADBA00BF00040020AE
:105CC000C100034B41F00601986903F0A3BA00BF7D
:105CD0000004002010B5084B86B0C0000C4601A996
:105CE00005920494CDE9023340F0060305200193A8
:105CF0000CF056F806B010BDE8410660F8B505F0A6
:105D0000E5FE03F095FA42680546CAB10024AB6887
:105D1000E70053F8343083B1DE08042B30460CD052
:105D2000F7F71CFC034630461B785F2B04D0AB68AA
:105D30003B44596846F064FF6A680134A242E6D8E1
:105D4000F8BD00BF08B503F017FCF6F785FB00BFF0
:105D500008B519B103F096FCF6F77EFB03F002FCE0
:105D6000F6F77AFB08B503F019FCF6F775FB00BFF0
:105D70000EB400B582B003AA52F8041B0192FFF7DB
:105D8000F1FF00BF08B50446F6F73EFD30B1074805
:105D900012F080FA01460648FFF7DAFF054812F0D4
:105DA00079FA224601460248FFF7E2FF1422066014
:105DB0008C330660402206600146024808B5FFF7B2
:105DC000C7FF00BF803006600146024808B5FFF7F4
:105DD000BFFF00BF303506600146024808B5FFF737
:105DE000B7FF00BF9C3206600FB400B583B0034814
:105DF00004AA52F8041B0192FFF7B4FF9C3206601C
:105E00000146024808B5FFF7A3FF00BF1037066040
:105E10000FB400B583B0034804AA52F8041B0192E2
:105E2000FFF7A0FF103706600146024808B5FFF7EC
:105E30008FFF00BF983606600FB400B583B00348EB
:105E400004AA52F8041B0192FFF78CFF98360660F3
:105E5000032830B5054685B00C4639D0CA0719D499
:105E600006280AD1334B0B40062B3ED08B0704D1BA
:105E70000A68314B92699A4231D0204601F086F986
:105E80004369002B45D0214628469847002840D03A
:105E900005B030BD4810072D0AD8DFE805F0060E22
:105EA000090916090604002807DB204605B030BDA5
:105EB000C043400040F00100EAE7B0F1404F21D07C
:105EC0004042400040F00100E2E730B11B48DFE70C
:105ED000084646F08DFE0028F8D01948D8E74868F3
:105EE00040B1400040F00100D2E7C80846F0A8FEEB
:105EF0000028F6D103A9204607F0A8F80399F7F780
:105F000003FAEEE74FF0804005B0BDE8304004F002
:105F1000CBBD0C4812F0BEF90B4A03462046515D3A
:105F20001C46019101F032F9034601992046DA88B6
:105F3000FFF782FF070080FFF5E40160882B066011
:105F4000802B066070220660D05306602DE9F04178
:105F500004460D4616461F4601F018F9D0F810E029
:105F6000BEF1000F07D03B46324629462046F44694
:105F7000BDE8F0416047064812F08CF90346204620
:105F80001C4601F003F903462046D988FFF754FF69
:105F90009022066000231A461946FFF7D7BF00BFBC
:105FA000F0B5184C9BB00E460546A16907A8A26142
:105FB0006269039163610492F6F736FA0190D0B9F1
:105FC0003246294605A82F68FAF766FD019B394637
:105FD00005A81A46FDF7E4FE019B1A461946FFF78D
:105FE000B5FF0190F6F718FA039A0198049BC4E9EB
:105FF00005321BB0F0BD039A049B0898C4E9053232
:10600000F6F72AFA0004002000B583B000220191BF
:1060100001AB0121FFF79AFF03B05DF804FB00BF5D
:1060200010B5144682B000226B46CDE9001402215F
:10603000FFF78CFF02B010BD13460A4659680039BD
:1060400018BF0121C1F1020C0144186803EB8C0355
:10605000FFF77CBFF0B51C4683B0930717460D468B
:10606000019032D1136833498B4231D032498B428F
:1060700052D032498B4228D0D98840F24F2C61450A
:106080001DD040F2BF1C614519D040F2532C614530
:1060900015D02B498B4218D12A4BE968994214D06C
:1060A00098B1104605F0E2FD274B006898423CD0BD
:1060B00001AB00220121FFF749FF206006E00199B2
:1060C00051B1C4E9007103B0F0BD276003B0F0BD69
:1060D0005368236003B0F0BD1C481D4EB34218BF87
:1060E00083421C4E0CBF01200020B34208BF40F089
:1060F0000100194EB34208BF40F0010010B9174823
:106100008342DED100210C20F6F7CCF9144B8760D6
:10611000C0E900352060D9E710B101F037F8054635
:106120007B68C4E9003503B0F0BD0E4812F0B2F848
:10613000FFF742FE1C530660E0520660945306606F
:1061400064410660CD030260E84106609038066055
:1061500054380660CC380660083906604439066059
:1061600064240660AC22066000232DE9F0410D4650
:1061700014460746C2E9003301F008F80F2D064621
:1061800011D0322D07D0F36983B122462946384613
:10619000BDE8F0411847836A002BF4D00D4BC4E9E9
:1061A0000037BDE8F0812060BDE8F081B06B0028C9
:1061B000FAD0E9001A46043041F0060146F01CFD11
:1061C0000028F1D02346426831463846BDE8F04108
:1061D000FFF740BFB458066070B5144682B006465B
:1061E0000D46FFF7C1FF23680BB102B070BD084830
:1061F00012F050F801463046019100F0C7FF024608
:106200002B460199D288034803F02EFAF6F724F9B9
:10621000C42206608030066000B583B06A46FFF78E
:10622000DBFFDDE9000109B102F0E4F903B05DF83C
:1062300004FB00BFF0B595B005460E46174601A811
:106240001C46F6F7F1F860B10CB115B0F0BD029B39
:10625000084918680AF0D6FA0028F6D10298F6F72D
:10626000FBF83A4631462846FFF77EFFF6F7D4F8AA
:1062700015B0F0BD80300660F0B58BB004460E4618
:1062800003AAFFF771FF049B002B4BD1039808B1C1
:106290000BB0F0BD20460BF081FF002842D003AACE
:1062A00020462F21FFF760FF02A9039807F070FD39
:1062B000014630460191F7F73FF9029B01331D1863
:1062C0002846F7F70BF80199029A044646F004FCB9
:1062D000029B2E223046E254029B0133E718F7F767
:1062E0003DF9014630460191F7F726F9019902463A
:1062F000384646F0F1FB294620460E4DF7F772F876
:106300000D4AC0000D4B146105A940F006000122A2
:106310000895059005200992CDE906330BF040FD64
:106320000BB0F0BD064811F0B5FF324601460548F6
:10633000FFF71EFD882B066000040020E841066080
:10634000E8220660243206602DE9F04105460C463D
:1063500017461E4629B1186800F018FF6B68834283
:1063600007D133463A462146A868BDE8F041FFF719
:10637000EDBD024811F08EFFFFF756FD00230660C9
:10638000F0B585B005460E46144600F0FFFEC36921
:1063900053B1042102AA284603940291314698473A
:1063A000029B73BB05B0F0BD806B50B3F1001A4681
:1063B000043041F0060146F01FFC10B3406810F0B5
:1063C00003071ED10168174B99421AD1CDB105F0D0
:1063D0004DFCCDE9025454B14068134B984210D0A3
:1063E00002AB3A460221FFF7B1FD05B0F0BD80686F
:1063F0000D4B984205D002AB22460121FFF7A6FDC6
:10640000D0E70A4811F046FF01462846019100F006
:10641000BDFE024633460199D288054803F024F9AF
:10642000F6F71AF864410660E84106601823066032
:106430008030066010B5044603F026F970B9204696
:1064400003F038F908B1204610BD084811F022FFCA
:1064500001460748BDE8104003F014B90023204668
:106460001A461946BDE81040FFF770BD4423066088
:1064700098360660F0B599B00C46054617461E469C
:1064800000F084FE3F4988426CD0836A7BB33E4A69
:10649000944244D08CB102AA284640F28531019240
:1064A000FFF79AFE019A002101200494FFF7C4FD32
:1064B00003460120336019B0F0BD384600F066FE97
:1064C00032490AF09FF9002832D028464FF4DF7194
:1064D00002AAFFF749FE029B002B3BD002AA2146ED
:1064E0002046FFF7A9FD034620463360E3E7264B2D
:1064F0009C42CFD102AA322128460192FFF734FEF6
:10650000DDE90123002BC7D005A80192F5F78CFF28
:10651000019A014678B3069B02203360CBE72846F8
:10652000984703460038336018BF012019B0F0BD0A
:10653000284640F2E53102AAFFF716FE029B4BB156
:1065400002AA214601200497FFF776FD03460120A9
:106550003360B0E73846FFF76DFF03460220336033
:1065600019B0F0BD33463A462146284619B0BDE879
:10657000F04003F07DBDFFF75FFD3060F5F74CFFA5
:10658000012098E7243B0660E8410660E831066098
:1065900070B582B005460C4600F0F8FD174A064675
:1065A000436A93421BD09CB12BB1214628469847A1
:1065B00008B102B070BD1E2128466A46FFF7D4FD1F
:1065C000009B7BB12146684603F074FE02B070BDAB
:1065D00021461020F5F766FF736A0446E4E7284673
:1065E00002B070BD064811F055FE0446284600F082
:1065F000CDFD03462046D988FFF71EFCA97801602F
:106600007023066030B583B0044600F0BFFD856A94
:106610002DB120462B4603B0BDE83040184732214B
:1066200020466A46FFF7A0FD009B33B16A46294623
:106630002846FFF701FD03B030BD064811F02AFEE1
:10664000034620461C4600F0A1FD03462046D9889B
:10665000FFF7F2FB8C23066030B5044699B000F0DA
:10666000FBFA204600F092FD856A2DB120462B46AC
:1066700019B0BDE8304018473221204603AAFFF781
:1066800073FD039BC3B105A8F5F7CEFE014640B1EB
:10669000069B104918680AF0B5F850B1284619B0A1
:1066A00030BD03AAFFF7C8FC0190F5F7B5FE0198CD
:1066B000F5E70698F5F7D0FE074811F0EBFD034625
:1066C00020461C4600F062FD03462046D988FFF7AD
:1066D000B3FB00BFA83506608C2306602DE9F04FA0
:1066E0002DED028B13688BB008EE103A002840F0B5
:1066F000F48002F1040B8146C1F307235FFA81FAAB
:1067000002930AEB43045B0000930BEB8403D3F882
:1067100004805BF82430B8F1000F08D018F0030FA4
:1067200005D1994AD8F80010914200F0E080009D10
:10673000002B00F0E7809A0706D11A6893498A4235
:1067400038D093498A4235D00AF1040201931544A6
:10675000A800F6F7C3FD019B0646B9F1000F00F053
:10676000C1800AF1010740F8049B4FEA8A090393AC
:10677000884B59464A46AA46019346F0ADF9039B19
:1067800006A91846FFF704FF044602E046F8275022
:1067900001372046FFF760FF0546002835D0BA458F
:1067A000F4D8019B4FEACA004FEA4A0A1E61F6F785
:1067B00095FDEBE7184606AA05A900F063FF059BC7
:1067C000013353441D44A800F6F788FD0646B9F18D
:1067D000000F00F089800AF10104012740F8049BB2
:1067E0004FEA8A096B4B59464A46019346F074F9C1
:1067F000059A06EB84000699920046F06DF9059B18
:1068000053441F44009BDC1902E0009B5546DC19F1
:10681000029B0BEB090106EB8700DA0046F05CF9FE
:10682000B8F1000F4AD018F0030904D1564BD8F83C
:1068300000209A427DD04FF42A71404606AADFF824
:1068400058A1FFF7C9FC002106AA0846FFF7F4FB90
:106850000021FFF79DFEDDF804B08146009718E0A7
:1068600007EA0A023846062A02D007F035FE074634
:1068700006AA1E214046FFF7AFFC06AA0021012010
:106880000897FFF7D9FB46F82470331F023443F80A
:1068900024004846FFF7E0FE621C074658B19542C7
:1068A000DED86D00CBF81060042D38BF0425A80099
:1068B000F6F714FDD4E7009FE31B0093009B3946D5
:1068C00018EE100A5A083346FFF740FB019B1E6181
:1068D0000BB0BDEC028BBDE8F08F02F1080BD2F8D3
:1068E000049009E7574640E74F46544678E740464C
:1068F000019302F067FC029B1D18019B6D00002BA9
:106900007FF419AF0AF101073D44A800F6F7E6FC51
:106910000646B9F1000F35D0009B40F8049BDC1906
:106920004FEA8A091B4B59464A46019346F0D4F870
:106930006EE7404602F07CFC42688046002ABDD0EB
:106940004D46DFF85490D8F808304FEAC50A53F89E
:106950003500013500EA090388B104280FD0062B61
:1069600001D007F0B9FD46F82400D8F808305344A8
:106970005A68A300023433445A60D8F80420954280
:10698000E1D399E75746CBE71C2F066024500660F9
:106990001C3E066000040020070080FF830770B5DE
:1069A0000C4686B0154606D10368214A93421DD095
:1069B000204A93421AD002A9FFF7EAFD00230646B7
:1069C00001936CB13046FFF747FE28B3019B6FEA95
:1069D000030C0133A444A342019345F82C00F1D3E6
:1069E0003046FFF739FEE8B906B070BD02AA01A92A
:1069F00000F048FE019BA3420ED313D8002CF3D025
:106A0000029A043D02EB840454F8043DA24245F886
:106A1000043FF9D106B070BD074811F03BFC019965
:106A2000FFF7F6F9054811F035FC2146FFF7F0F9BC
:106A3000245006601C3E0660AC230660D02306602E
:106A40008307F0B5154683B0CFB2C1F3072406D152
:106A500003683B4A934240D03A4A93423DD00021DA
:106A6000FFF796FD0023064600936FB13046FFF70F
:106A7000F3FD00285ED0009BFA1A01332244BB428A
:106A8000009345F82200F1D30021084604F0E8FD08
:106A9000074602E0384604F0A5FA3046FFF7DCFD71
:106AA00001460028F6D1BB68A34243D305EB84021C
:106AB00045F8247054B1D7E902311B1B034401305F
:106AC00051F82330844242F8043DF4D1B968384685
:106AD000091B04F0F3FD03B0F0BD694601AA00F004
:106AE000D1FD00993B198B4224D8DDF804C054B184
:106AF0000CEB81032A1FA3EB840653F8040D9E427E
:106B000042F8040FF9D1C81B0CEB8701001B04F0FD
:106B1000A7FD45F82400BB00002FDCD0019905EB50
:106B200084040B4453F8042D8B4244F8042FF9D10C
:106B300003B0F0BD044811F0ADFB0099FFF768F910
:106B4000245006601C3E0660AC23066001460348E4
:106B5000490008B541F00101FFF7F4F87C34066004
:106B60000146024808B5FFF7F3F800BF7C34066021
:106B700043000C460648022143F0010300B583B0F0
:106B80006A460093019402F001FDF5F765FC00BF31
:106B90007C3406600146024808B5FFF7D9F800BF0B
:106BA000343106600146024808B5FFF7D1F800BF4E
:106BB000403406600FB400B583B0034804AA52F80D
:106BC000041B0192FFF7CEF8B83406600146024874
:106BD00008B5FFF7BDF800BFC833066008B5024826
:106BE00011F058FBFFF7F0F83824066030B595B087
:106BF00004460D4601A8F5F717FC48B9294620467A
:106C0000FFF702FA0446F5F707FC204615B030BD41
:106C100000240299024800F0F5FA204615B030BD74
:106C20000414066008B5044B5A6E02B908BD002270
:106C3000586E5A66F5F710FC0004002082B0024B33
:106C400001AA1A6002B0704700040020014B58608E
:106C5000704700BF0004002000B583B0054A01A9B9
:106C6000D2E900325B1A9A4202D903B05DF804FB04
:106C7000FFF7B4FF0004002030B583B0144605468A
:106C80009DF8182009B1012A10D19C4205D0AC42D0
:106C90001AD8AB420FD303B030BDAC42FBD00D4885
:106CA00011F0F8FA2A462146FFF7C6F80A4811F013
:106CB000F1FAFFF7B9F80948019311F0EBFA019BDB
:106CC0002A461946FFF7B8F8054811F0E3FA611BA8
:106CD000FFF7B2F8CC240660A02406603C250660CD
:106CE0000825066010B49DF8044011B10968C1F38D
:106CF0001B1101945DF8044BFFF7BEBF2DE9F04F67
:106D0000804683B0894693461F46002B48D0002416
:106D10000C9D0D9EA246019411E06A88910542D413
:106D2000D2B20AF1010A59F82400012A1AD0022A23
:106D30002CD03060013408350436A7421BD0A04562
:106D4000EBD8298800225846C90041F0060145F0D9
:106D500053FFF8B16A88019BD2B240680133012A1F
:106D60000193E4D1013445F043FF08353070A74268
:106D700006F10406E3D1D04515D8DBF80030019ABE
:106D8000B2EB131F14D303B0BDE8F08F00F04CFB3F
:106D90003060CFE76A88D3050FD46A683260C9E7EC
:106DA0009A460193E7E7084811F074FAFFF73CF8B8
:106DB000064811F06FFAFFF737F8054811F06AFA44
:106DC0002988FFF739F800BF6C250660A825066002
:106DD0009025066008B5024811F05CFAFFF7E2FE64
:106DE000C8250660094A0023014602F1420C03E06F
:106DF000624505D032F8023F8B42F9D318467047FE
:106E000001EB510141F00103184670470C26066062
:106E100010B50B46044641B9C0E90111236803F0DF
:106E2000080343F00103236010BD0021D800636014
:106E3000F5F754FBA060F1E70B01C0E9011202680D
:106E400043F0070302F0080213430360704700BFDA
:106E500010B5037804469B0706D50022236862F329
:106E60001F13C4E9003210BD8068F5F747FBF4E753
:106E700010B5037804469B0709D52368002203F068
:106E80000C0343F00103C4E90122236010BD8068B4
:106E9000F5F734FBF1E700BF2DE9F04147680646FE
:106EA000781CFFF79FFF00210446C000D6F8088039
:106EB000F5F714FB3368746003F00E03B06043F021
:106EC000010333609FB108F10404002554F8041C49
:106ED000013541B104294FF00102304603D045F09D
:106EE0008BFE23684360AF4204F10804EED14046B4
:106EF000BDE8F041F5F702BB0B46002210B5044691
:106F000011469800C4E90032F5F7E8FAA06010BD18
:106F10002DE9F04F83B0134606468B460092026877
:106F20001AB9D90752D500F075F859460620FEF770
:106F30008FFF009A33684FEA600A02F00102019263
:106F4000BAFBF3F203FB12A94C4600270BE000F05A
:106F500005FA00283FD133680134B4FBF3F103FB99
:106F60001144A14515D0B06859464FEA840850F83D
:106F7000245000EB840E2846C5B1042DE7D101341E
:106F8000002F08BF7746B4FBF3F103FB1144A14582
:106F9000E9D1019BD3B1002F34D1304600F03AF84B
:106FA0003368BAFBF3F203FB12A9CDE7009BDA07C3
:106FB0000CD57268002F08BF77465D4601327260BB
:106FC000C7F800B0284603B0BDE8F08F002528467A
:106FD00003B0BDE8F08F009B9B07F3D573680134C5
:106FE000B268013B73603368B4FBF3F103FB1144F7
:106FF00052F8243003B10423284642F8083003B085
:10700000BDE8F08F72685D4601327260C7F800B06B
:10701000D8E700BF2DE9F041076806460024D0F804
:107020000880781CFFF7DEFE2146C6E900048000D8
:10703000F5F754FAB06077B1A8F1040555F8041FCC
:10704000013431B104294FF00102304601D0FFF77D
:107050005FFFA742F2D14046BDE8F041F5F74EBAD6
:1070600010B501688646F9B184680023224601E024
:107070008B4217D0944652F8040B01330028F7D006
:107080000428F5D0DEF80420013ACEF80420B3FB42
:10709000F1F201FB123354F8233003B10423CCF88E
:1070A000003010BD002010BD084610BD10B50446CC
:1070B0008068F5F723FA0023C4E90033A36010BD0C
:1070C00000B5826B53685FEA131C0FD0D2680023AF
:1070D00002F1040E01E09C4508D05EF83300013354
:1070E000B0F904208A42F6D15DF804FB01485DF84E
:1070F00004FB00BFE841066013460246084610B58F
:1071000082B01C68B3F90610E38800910249F6F7D3
:10711000DDFF02B010BD00BF5C260660704700BFF7
:10712000064B0340062B07D000F00303022B01D0CF
:10713000006870470248704702487047070080FFA8
:10714000C4370660984D066038B581680446CB07A1
:1071500015D40846FFF7E4FF05466B6905209847FC
:10716000E168B1EB600F0CDA49002B6A0422A068D9
:1071700041F001019847E3680133E36038BD024DF7
:10718000EBE7002038BD00BF703C0660C30701D4A8
:10719000FFF7C6BF00487047703C06602DE9F0411C
:1071A00006460C461546FFF757FD45F045FD1CF019
:1071B000BFFCC0B9E3070BD42046FFF7B1FF8768D7
:1071C00057B12A46214630463B46BDE8F0411847B4
:1071D00006488768002FF4D1C28830460449BDE8CC
:1071E000F041F6F773BFBDE8F08100BF703C066068
:1071F0006826066003460A4601481946FFF7CEBFD7
:10720000C45E06602DE9F04F2DED028B83B004467D
:1072100008460D4600AF02F04DFA70B929462046E7
:107220000222FFF7BBFF3B492046F6F78FFB0C37E6
:10723000BD46BDEC028BBDE8F08F10F051FE00287A
:10724000ECD03A1D3946284602F0A0FA3B68002BE4
:10725000E4D06B46304808EE103A11F01BF80646B1
:1072600010F0AEFF03463046073323F00703ADEBC3
:10727000030D69466E4610F0A7FF284811F00AF882
:10728000804610F09DFF03464046073323F0070376
:10729000ADEB030D6946E94610F096FF204810F06B
:1072A000F9FF804610F08CFF03464046073323F079
:1072B0000703ADEB030D6946EB4610F085FF314641
:1072C0002046F6F743FB3E68033E1FD4DFF844A098
:1072D00004E02046F6F73AFB033E17D47B684946A4
:1072E00020464FEA860803EB860C53F82620DCF88C
:1072F0000430F6F7EBFE7B68514643449A68002A57
:10730000E7D059462046F6F7E1FEE5E718EE103AD9
:107310009D4683E700650760702606609426066038
:10732000AC26066008B5C307024609D4FFF7F8FE8D
:10733000084B0069984208D0003818BF012008BDEA
:107340000548044B00699842F6D11046BDE8084054
:1073500009F018B925030260703C0660884210B538
:1073600004462CD02A4B994227D09C4225D0E007D6
:1073700021D4284B2340062B30D0A3072AD0254BFD
:107380000B40062B19D08A0703D1234B0A689A4277
:1073900013D0E3073AD42046FFF7C2FE836963B1F6
:1073A0000A4602202146984738B11C4BC01AB0FA51
:1073B00080F0400910BDCA071FD5002010BD00F0A5
:1073C0000303022B1DD01BB9154B22689A42C9D06A
:1073D000012010BD104B22689A42D0D10D4B0B40BA
:1073E000062B05D08807E8D10B4B0A689A42E4D1F6
:1073F0002046BDE8104006F071BC23460C461946F5
:10740000B7E7044B0340062BACD1E1E70548C5E7DD
:10741000E8410660070080FF984D0660882B0660F3
:10742000F82C0660703C0660134B984210B5044679
:1074300010D0124B98420FD0C20709D483070DD148
:107440000F4B02689A4209D1BDE8104003F0F4BB2B
:10745000401010BD002010BD012010BD094810F0E3
:1074600019FF0146204640F28522FFF759FE0346E8
:107470000846D988FEF7E0FC802B0660882B066062
:10748000703C0660B8260660C20707D4830703D1A4
:10749000034B02689A4201D0FFF7C6BF03F0C4BB9A
:1074A000703C0660144A904210B582B010D0134A66
:1074B000904207D010F0010210D043100B6010462C
:1074C00002B010BD01231A460B60104602B010BD79
:1074D0000122002310460B6002B010BD8407EED1DC
:1074E000074C0368A342EAD1019103F0A5FB01997F
:1074F00001220860E3E700BF802B0660882B06604E
:10750000703C06601B4A0346904210B582B013D00F
:10751000194A90420DD010F0010210D0431000EE35
:10752000103AB8EEC00A012281ED000A104602B0FE
:1075300010BDB7EE000AF6E79FED100AF3E710F072
:10754000030C08D10E4C0368A342EFD1019103F064
:10755000E1FC0199E7E7BCF1020FE7D109481840C7
:107560000628E3D003F1FF4323F0030300EE103AB3
:10757000D9E700BF802B0660882B06600000000062
:10758000703C0660070080FF30B583B0044601A957
:10759000FFF7B8FF18B19DED010A03B030BD0848F0
:1075A00010F078FEE307054608D42046FFF7B8FD43
:1075B000C18840F23E222846FEF73EFC0148F7E72C
:1075C000B8260660703C0660F8B5284B04460D46A8
:1075D0001646984214D0264B98420BD0C30713D5B9
:1075E0004410002307EE904AF8EEE77AC1ED007AE6
:1075F0001360F8BD4FF07E5200230A603360F8BD7F
:1076000000230B601360F8BD10F003030AD1036878
:10761000184FBB4214D0184DAB4218D1BDE8F8400A
:1076200001F0E4B9022B12D1144B0340062B0ED00B
:1076300004F1FF44002324F003042C603360F8BD00
:1076400003F068FC002385ED000A3360F8BD0C48A8
:1076500010F020FE014620464FF4E672FFF760FD71
:1076600003460846D988FEF7E7FB00BF802B06607B
:10767000882B0660703C0660F82C0660070080FFCF
:10768000B826066038B5850704460CD00E4810F0C1
:1076900001FEE307024615D42046FFF741FDC188ED
:1076A0001046FEF7C9FB0368084DAB4206D0084DF3
:1076B000AB42EBD1BDE8384003F0F2BFBDE8384043
:1076C00008F03AB90348EAE7D0260660245006607D
:1076D0001C3E0660703C066010B582B00C4601A9E5
:1076E000FFF7D0FF019BA34201D102B010BD0348B8
:1076F00010F0D0FD019A2146FEF78AFBF4260660C1
:10770000F0B51E46D30783B0144607460D4615D57F
:1077100050100190002809DB1EB9A84217D203B00F
:10772000F0BDA8421BD9284603B0F0BD2844019003
:107730005EB10028F5DA002003B0F0BD01A91046C3
:10774000FFF7B0FE70B10198E4E70028E5DA0C48D5
:1077500010F0A0FDFA8801460A48FEF709FB0198DF
:1077600003B0F0BD084810F095FD02462046FFF733
:10777000D7FC0346F9881046DA88FEF75DFB00BFA8
:10778000482706609C32066024270660820707D1DE
:10779000002803DB400040F00100704703F022BAEC
:1077A00003F082B98207014610B503D1104B02687D
:1077B0009A4210D0CB0708D40846FFF7B1FC4369C2
:1077C0003BB10520BDE8104018470A484369002B2B
:1077D000F7D1184610BD084B0340062B04D0806833
:1077E000400040F0010010BDC008F5F7A5FEF7E726
:1077F000044B0660703C0660070080FF10B504462D
:10780000FFF7D0FF00B110BD074810F043FDE307BC
:10781000024606D42046FFF783FCC1881046FEF7D7
:107820000BFB0248F9E700BF60270660703C06606A
:10783000F8B510F00107044615461BD1FFF770FCA0
:10784000036A43B12A4620469847064610F058FB83
:107850000EB13046F8BDBDB1042D0DD00E4810F06C
:1078600019FD024677B92046FFF75AFCC188104639
:10787000FEF7E2FA0948E3E7094810F00BFD02467B
:10788000002FF0D00548F1E7064810F003FD02464E
:10789000002FE8D0F6E700BFD4270660703C0660F2
:1078A000B027066084270660704700BF10B4054A01
:1078B0000023054CC1E90203C1E9004208465DF816
:1078C000044B70474971016008410660C30710B559
:1078D000044609D4FFF724FCC36A4BB120469847FD
:1078E000B0FA80F0400910BD0248C36A002BF5D100
:1078F000184610BD703C066008B5FFF7E7FF00B101
:1079000008BD024810F0C6FCFEF78EFA0428066097
:10791000062803D1490041F001007047002070475C
:10792000042808D0052804D18868400040F00100F0
:107930007047002070478A68024B0348002A08BF3E
:1079400018467047802B0660882B066000230B4A80
:1079500010B40B4CC1E90233C1E900400368934203
:1079600003D008465DF8044B7047436808465DF84D
:10797000044BC3F317238B60704700BF002B0660D6
:1079800094290660F8B50D4601790446164601F0C3
:107990007F010022402009F0D3FDE7680F4A03462B
:1079A0002F60A16800FB01F16960217901F07F017E
:1079B000A9602168914201D00020F8BD94F904200B
:1079C000002A03DBB20701D50120F8BD6268002060
:1079D000C2F3172203FB02732B60F8BD002B066075
:1079E0002DE9F04F0C4689B0054608681F469146C0
:1079F000FFF7CCFB012202A980462068FFF77CFF3D
:107A0000012205A96068FFF777FF00229DF81C108E
:107A1000402009F095FD012837D1022DDDE90261F2
:107A200006EB010A16D9A268DFF87CB05A4504D0EB
:107A300003464046FFF764FE0644032D0AD0E26881
:107A40005A4507D040460123DDE90241FFF758FEC1
:107A500004EB000AB24505D2E7B94FF0FF3009B098
:107A6000BDE8F08F069BAAEB06013046059ACDF8DB
:107A7000009005F00DFA0028EED0029BC01A4000DD
:107A800040F0010009B0BDE8F08F054810F002FC9D
:107A9000FEF7CAF9034810F0FDFBFEF7B1F900BF8D
:107AA0003428066054280660E8410660002301225D
:107AB000FFF796BF00234FF0FF32FFF791BF00BFE3
:107AC00001231A46FFF78CBF01234FF0FF32FFF767
:107AD00087BF00BF7828F8B505460E461FD00022A4
:107AE0000146402009F02CFD002107461020F4F744
:107AF000D9FC04460C4B06FB07F025710021626897
:107B0000A6606FF31F226260084A012D18BF13465A
:107B10002360F4F7C7FC03462046E360F8BD044841
:107B200010F0B8FBFEF76CF9C42A0660882A0660DC
:107B30006828066001280A4600B583B006D10968A6
:107B400040F20E336A460220CDE9001301460023BD
:107B5000024805F089FA03B05DF804FB984D066011
:107B600070B50B4684B004460122184601A9FFF700
:107B7000C3FE00222179402009F0E2FC029D6368E7
:107B80000646B5FBF0F5B5EB132FC3F3172212D859
:107B9000521BE06862F31F236360A36805FB06F2D3
:107BA000019903FB060044F097FFA36808482B44A3
:107BB000A36004B070BDD4E90210294406FB01F1B2
:107BC000F4F78EFC6368E0606FF31F236360E4E703
:107BD000E841066070B5426882B004460B4632F058
:107BE000FF050ED02079D4E9022109F0ABFF164839
:107BF000D4E901320132A3F58073C4E9013202B045
:107C000070BD2A4601910179402009F099FCA168D4
:107C100062680646083100FB01F1082060F31F226C
:107C2000E0686260F4F75CFC62682946A568C2F30C
:107C30001722E060013A06FB02F205FB06663044BB
:107C400044F072FF019BCDE7E841066010B4426842
:107C50000346C46891688C420BD21079D1689A6847
:107C600000F07F0022440134DC605DF8044B09F031
:107C70007FBD00205DF8044B704700BF2DE9F04345
:107C80008C4687B004461546002A34D011F003060E
:107C900003D1844B0A689A4232D000236246A1681D
:107CA0002068FFF72DFD804B2168024699420ED0D7
:107CB000042D11D094F804C02B46E1680CF07F002D
:107CC0007A4E09F03FFF304607B0BDE8F0836368A5
:107CD000042D00EB132208D12079E16800F07F0029
:107CE00007B0BDE8F04309F043BD94F9043094F8BF
:107CF00004C0002BE0DB0026304607B0BDE8F0836F
:107D00006A46806808F00AFF002800F0C5802179E3
:107D1000042D32464FF0400001F07F0165D009F09C
:107D20000FFC15F0030206463AD12B686049186A29
:107D3000884200F084805F4A934231D1012E40F0A6
:107D4000A680324603A92846FFF7D6FD564ADDE94C
:107D50000398DDE900012368451AE768934245442A
:107D600023D0002D2CDD6368B5EB132F57D8A36803
:107D7000404401FB06712B441A1A06FB007006FBF7
:107D800002F244F0B7FE009806FB08F2494600FBF9
:107D9000067044F0AFFEA368444E2B44A36092E704
:107DA000454810F077FAFEF7FDFE94F90430002BF9
:107DB000A1DA002D6BD16368C3F3172306FB0377A9
:107DC000494606FB08F206FB007044F085FE019967
:107DD000A2680098521A06FB0171404406FB02F2A9
:107DE00006FB007044F086FED5E709F0A9FB2E4B98
:107DF000226805469A4237D02079DDE90031C91A58
:107E0000FFF768FEE1680646C068DDE900239B1ABB
:107E100005FB021105FB03F244F05EFE53E7A16887
:107E20003846294406FB01F1F4F75AFB636807461C
:107E3000E0606FF31F236360DDE9000197E72979B4
:107E4000402001F07F0109F07BFBB0421FD1164AB0
:107E50002B689342D5E902897FF47BAF6B68C3F34B
:107E6000172306FB039974E731461020F4F71AFB39
:107E7000064694E80F0086E80F00009A02EB1120F6
:107E800060F31F217160019B9B1AB3601BE70B48D5
:107E900010F000FAFDF7B4FF094810F0FBF9FEF707
:107EA00081FE00BF44460660002B0660E841066084
:107EB0007D7C0160044B0660D0280660AC2806601B
:107EC00078280660831E2DE9F041064688B00D46ED
:107ED00014462C2B23D8DFE803F05322222222223F
:107EE000222222222222752217222222222222222A
:107EF0002222272217222222222222222222222268
:107F0000222222222222820014F0010040F08480EA
:107F100014F0030303D16B4A216891427CD0002402
:107F2000204608B0BDE8F08102A901222846FFF7EB
:107F300029FD05A920460122FFF7DEFC00229DF85D
:107F40001010402009F0FCFA069EA96805469DF82D
:107F50001000B6FBF5F63144FFF7BCFD0446C068DF
:107F6000DDE9021244F0B8FDE068039B06FB05F270
:107F70000599184444F0B0FD204608B0BDE8F081F2
:107F8000012202A92846FFF7FDFC012205A920468F
:107F9000FFF79CFC88B10220DDE90534DDE902121F
:107FA000009408F0A1FE40B1474CB9E7E3075FD465
:107FB00014F0030358D0022B5DD0444C204608B087
:107FC000BDE8F081424B0A689A42A8D021462C466F
:107FD0002846FFF7C5FD204608B0BDE8F081012224
:107FE00005A92046FFF772FC0028DFD0AA07E4D1DC
:107FF000384B2A689A42E0D10124012202A928467E
:10800000FFF7C0FC0094DDE90523DDE9020104F07F
:108010003FFF0028C8D1D0E72046FFF705FA01222C
:1080200005A907462846FFF7ADFC102EDDF818809D
:1080300026D0A9689DF81C0007FB01F1FFF74AFD57
:108040000446C668B8F1000F3FF46AAF7D1E002FEA
:108050003FF466AF013D30460599424644F03CFD91
:10806000691C4644F6D15BE7164B22689A42A4D1BC
:108070000020FEF797FD184B2340062BF8D19CE714
:1080800000222979402009F05BFAAB6807FB03F373
:1080900000FB03F1E868F4F723FAAB68064607FB38
:1080A00003F3C5E902306B686FF31F236B603FB1C8
:1080B000013F46442C46B8F1000F3FF431AFC5E70D
:1080C0002C462DE7703C0660882B0660802B0660EE
:1080D000002B0660C42A0660070080FF01282DE9F6
:1080E000F041804684B00D4635D08B072CD0284611
:1080F000FFF758FB00284ED0441021464046FFF7BA
:10810000E9FC002106462846FEF742FA002507460C
:108110003846FEF7A1FA48B164B901463046FFF788
:1081200059FD3846FEF798FA0028F5D1304604B0DC
:10813000BDE8F08105F1010C2A460346F16840468E
:10814000654609F0FFFCE3E70B68164A934202D04C
:10815000154A9342CBD1012201A92846FFF7B6FB6D
:108160000028C4D041460022402009F0E9F9029BD2
:10817000B3FBF0F100FB01F4A3420ED14046FFF740
:10818000A9FC064622460199C06844F0A5FC304689
:1081900004B0BDE8F0810446AFE7044810F07AF877
:1081A000FDF72EFE044B0660C42A0660F428066024
:1081B00070B50C4682B000261546194601220223EE
:1081C00020460096FEF78EFD286805F0C7FD012CBD
:1081D00006D06968007802B0BDE87040FFF77EBF46
:1081E0003146007802B0BDE87040FFF773BC00BFB5
:1081F00030B510460C46002585B0194601232A46A5
:10820000009505462046FEF76DFD04B32968CA07B0
:108210000BD48B0703D1114B0A689A4205D0012079
:1082200005B0BDE83040FFF759BF0846FFF7FCF83E
:108230000246012011460392FFF74CFC0446039AC4
:108240000021C06844F070FC204605B030BD2146D6
:10825000012005B0BDE83040FFF73CBC703C066033
:10826000F8B50D790C460646012D32D02A46204934
:10827000F5F72CFFA3682BB930461E49BDE8F8403E
:10828000F5F764BB1C493046F5F760FBA368B3B152
:1082900000251A4F2A46E1682079013509F068FA6D
:1082A000012201463046FEF779FFA368AB4206D9AA
:1082B000002DEFD039463046F5F748FBEAE7104984
:1082C0003046F5F743FB30460A49BDE8F840F5F77C
:1082D0003DBB0C49F5F73AFB30462B46D4E9022169
:1082E00004F0F2FC30460349BDE8F840F5F72EBB38
:1082F0002C2906607C430660382906604029066008
:108300003C2906602029066070B506460D461020FF
:1083100000211446F4F7C6F8067142686FF31F2275
:108320004260024AC0E90254026070BD002B066040
:10833000F8B50546084605F011FD07460022402025
:10834000397809F0FDF82979AC68064601F07F011B
:108350000022402009F0F4F800FB04F3B3FBF6F12F
:1083600006FB11336BB9EA683878FFF7CDFF95F952
:108370000430002B00DBF8BD037963F07F03037149
:10838000F8BD02480FF086FFFDF74EFD4429066058
:1083900070B5084686B0194600260123154600969A
:1083A0001A46FEF79FFC012203A92868FFF7A4FAEA
:1083B0009DF814403246049E2146402009F0C0F842
:1083C000039AB6FBF0F12046FFF79EFF0322044616
:1083D00003A92868FFF77AFA18B1237963F07F03BD
:1083E0002371204606B070BD0246012010B50C4630
:1083F00082B011460192FFF76DFB21460446019AB7
:10840000C06844F069FB204602B010BD024601205E
:1084100010B582B011460192FFF75CFB0446019A49
:108420000021C06844F080FB204602B010BD00BFB0
:1084300038B505460C4610200021F4F733F8034AFE
:1084400002600122C0E90254426038BDC42A0660BD
:10845000136830B40BB130BC70474568AC1C50F8A1
:108460002440002DF7D0A4F1040C02E001339D421A
:10847000F1D05CF8044FA142F8D1023350F8233018
:1084800030BC1360704700BF2DE9F04790460E46A0
:1084900015490446F5F75AFAD8F80430EBB1043E12
:1084A00008F104070025DFF848A0DFF8489001E054
:1084B000F5F74CFA56F8042F514620460135F5F7EA
:1084C00005FE57F8041F20460122FEF767FED8F884
:1084D000043049462046AB42EAD820460349BDE86D
:1084E000F047F5F733BA00BF3C2B06607C430660CB
:1084F000402B0660402906604B680A46023351F85B
:108500002310FFF7C1BF00BF0979490041F0010105
:1085100044F066BB052805D00979490041F0010106
:10852000FDF796BC00207047032A0B7906D013B1E3
:108530000649F5F70BBA0649F5F708BA13B105492C
:10854000F5F704BA0449F5F701BA00BF2C15066027
:10855000B4140660F4130660FC13066030B51046D0
:108560000C46002583B0194601232A46009505468E
:108570002046FEF7B7FB14B9054803B030BD2868A4
:1085800044F036FB0028F7D0024803B030BD00BFEE
:10859000802B0660882B06602DE9F04102EB430436
:1085A000884607461E4601341546A4002046F4F7C7
:1085B00095FE221F0446069940F8048B44F08CFA7D
:1085C00023463246691C3846FDF7C0FC014B1C614E
:1085D000BDE8F0810004002010B5944682B01C462E
:1085E0000A4663460094D0E90101FFF7D5FF02B0C7
:1085F00010BD00BF38B505460C460C200021F3F72E
:1086000051FF024A8460C0E9002538BDCC2B0660CA
:10861000406870474160704710B50021044608204B
:10862000F3F740FF014AC0E9002410BD082C0660A2
:108630002DE9F04315468268044687B001EB4509F1
:108640000E461F4602EB090005281AD804F10C015A
:10865000920001A844F040FA01ABA0684FEA8902F9
:10866000394603EB800044F037FAA16801AB2A4693
:1086700031446068FDF76AFC0446204607B0BDE857
:10868000F08300218000F3F70DFFA26804F10C01D4
:108690008046920044F020FAA0684FEA89023946E9
:1086A00008EB800044F018FAA1682A46434631449A
:1086B0006068FDF74BFC04464046F3F71FFF204679
:1086C00007B0BDE8F08300BFF8B50D4606460021AF
:1086D0001746EC1CA4002046F3F7E4FEA4F10C02BC
:1086E000054B044646603946A5600C30236044F0D3
:1086F000F3F92046F8BD00BF442C066030B591ED7B
:10870000010A87B00C460546B5EE400AF1EE10FAB4
:1087100010D191ED020A002106236722009102A8E0
:108720001021FCF703FB02AA1A492846F5F7CEFCF4
:1087300007B030BD00220623102102A80092672254
:10874000FCF7F4FA02AA14492846F5F7BFFC94EDA9
:10875000020AB5EEC00AF1EE10FA13DAB4EE400ADE
:10876000F1EE10FA0ED600220623102102A8009284
:108770006722FCF7DBFA02AA08492846F5F7A6FCAF
:1087800007B030BD06492846F5F7E0F894ED020A37
:10879000E9E700BF802C0660842C06608C2C066004
:1087A000882C066008B52DED028B072805D8DFE878
:1087B00000F0571D0404320444080020BDEC028B75
:1087C00008BD91ED020AD1ED017A20EE000AA7EE74
:1087D000A70A32F07FFD10EE103A23F00300BDEC43
:1087E000028B40F00200A0F1FF4008BDD1ED018AEC
:1087F0000C2091ED028A0021F1EE688AF3F752FE17
:10880000B1EE488A194B0360C0ED018A80ED028AFF
:10881000BDEC028B08BDD1ED017AF5EE407AF1EEA8
:1088200010FA21D1D1ED027A1149F5EE407A1148C2
:10883000F1EE10FA08BF0846C0E7D1ED017A91EDDC
:10884000027AFDEEE77ABDEEC77A17EE900A17EED0
:10885000103A5840BDEC028B400040F0010008BDCA
:10886000BDEC028B084608BD0248A7E7F82C06605D
:10887000802B0660882B066030B510460C4600251C
:10888000194602232A462DED028B85B00095054638
:108890002046FEF727FA2CB3012C30D02868354C3F
:1088A000820702D10368A34253D0FEF76DFEF0EEBB
:1088B000408A9FED318A6868830702D10368A3422A
:1088C0003ED0FEF761FE30EE088A00210C20F3F75F
:1088D000E9FD0460C0ED018A80ED028A05B0BDECBF
:1088E000028B30BD21460C20F3F7DCFD0023214A2A
:1088F00043600260836005B0BDEC028B30BD286828
:108900001E4B0340062B29D0810707D103681C4A60
:10891000934223D0174CA34201D1DFE7154CFEF759
:1089200033FE0021B0EE408A0C20F3F7BBFD00239C
:10893000046080ED018A836005B0BDEC028B30BD20
:10894000D0ED027A90ED010A78EEE78A38EE008ADF
:10895000BBE7D0ED018A90ED028AACE703A90024C1
:1089600005F016FA012303991A460094FCF7CAFD94
:10897000B4E700BFF82C066000000000070080FF8D
:10898000984D0660136803B1704740F24A3399422C
:108990000CD040F276239942F6D1836823F003038A
:1089A00043F00203A3F1FF4313607047436823F0D1
:1089B000030343F00203A3F1FF431360704700BFBA
:1089C00008B500210C202DED028BF0EE408AB0EEB0
:1089D000608AF3F767FD044AC0ED018A026080ED0A
:1089E000028ABDEC028B08BDF82C066043680B6060
:1089F00083681360704700BF10B52DED048B82B003
:108A000004460846B0EE409A01AA6946B0EE608A74
:108A1000FEF7DAFDA01E1E2811D8DFE800F07B105B
:108A20001010101010101010101049525B9D68109B
:108A300015101010101049525B9D68101500002091
:108A400002B0BDEC048B10BD28EE080AA9EE090A9D
:108A500032F040FCB5EE400AF1EE10FA40F09080A2
:108A6000DDED017AF5EE407AF1EE10FA40F0B180DA
:108A7000DDED007AF5EEC07AF1EE10FAC0F2A980D1
:108A8000F5EE407ADFED5A7AF7EE008AF1EE10FA51
:108A900048FEA78A00210C20F3F704FD554BC0EDDA
:108AA000018A036080ED028A02B0BDEC048B10BD28
:108AB000DDED008ADDED017A79EE288A38EE278A2D
:108AC000E8E7DDED008ADDED017A79EE688A38EEBF
:108AD000678ADFE79DED007ADDED017A67EEC88AEF
:108AE00028EE078AE9EE078AA9EE278AD2E7DDEDAC
:108AF000017AF5EE407AF1EE10FA1DD1DDED007A43
:108B0000F5EE407AF1EE10FA6AD0C9EE278A88EEC7
:108B1000278ABFE7DDED007AF4EE497AF1EE10FA2C
:108B200018D1DDED017A344BF4EE487A3348F1EE9A
:108B300010FA08BF184683E79DED006AB5EE406A5B
:108B4000F1EE10FA0DD1B1EE490AC8EE278A80EE97
:108B5000278A9FE7294873E729480FF09BFBFDF719
:108B600063F967EEA75AF1EE676AE6EE065A86EEFB
:108B7000257AC6EEA57A8DED007ACDED017AADE7C6
:108B800032F0A4F8F0EE490AF0EE408AB0EE480A5E
:108B900033F058FD9DED007ADDED016A27EE008A85
:108BA00020EE660AA6EEA88AA7EE280A31F0A8FEF3
:108BB000B0EE409AB0EE480A33F046FAF0EE408A42
:108BC000B0EE480A33F0F6F920EE098A68EE898A99
:108BD00060E70C480FF05EFB01460B48FDF7B8F864
:108BE0000A480FF057FB01460748FDF7B1F800BFF0
:108BF00000000000F82C0660882B0660802B0660C1
:108C0000942C0660E02C06604C370660C42C06608D
:108C10000B461146D3ED020A93ED010AFFF7ECBEB5
:108C20000B6830B484689C4211D9C56801E09C424D
:108C30000DD055F833204FEAC30C0133002AF6D08B
:108C4000042AF4D00B60C06830BC60447047002038
:108C500030BC704710B4074C034600220C6090F8FB
:108C600008C008465DF8044B81F804C05B68C1E9A0
:108C700002327047982E066010B40122044C002383
:108C80000C600A715DF8044BC1E9020308467047A5
:108C9000982E066010B5002104460C20F3F702FC64
:108CA00002490222C0E90014027210BDD42E0660EF
:108CB00010B5002104460C20F3F7F4FB0249012211
:108CC000C0E90014027210BDD42E066010B5002158
:108CD00004460C20F3F7E6FB02490022C0E9001429
:108CE000027210BDD42E066010B500F10C0182B0E6
:108CF00004468068FFF794FF60B12379012B0ED002
:108D0000022B09D06946D0E900230220CDE90023D7
:108D100006F00AFE02B010BD406802B010BD006847
:108D200002B010BDF0B5184B06460A7A85B00C4665
:108D3000012553F82210F4F709FE14493046144F68
:108D4000F4F704FE237A134962688DF80430002397
:108D50000091CDE9022305E001222146304600259D
:108D6000FEF71CFA6846FFF7BFFF044630B1002D3E
:108D7000F2D139463046F4F7E9FDEDE706493046D1
:108D8000F4F7E4FD05B0F0BD102F0660342D066049
:108D900040290660982E0660382D066008B50379D4
:108DA0009B0700D408BD0020FDF73EF8F8B50D463E
:108DB000064614460F6892B92246381D696843F08A
:108DC0001BFF034620B1406810B1022C0FD0F8BD44
:108DD000022E08D0A868012CF9D15860F8BD384699
:108DE000FFF7DCFFE8E7022C04D00448F3E7002299
:108DF0005A60F8BD69680248FCF7A4FFE8410660C4
:108E0000D83206600122FFF7D1BF00BF0222FFF770
:108E1000CDBF00BF0022FFF7C9BF00BF70B5044639
:108E200084B00025FFF7BAFF01A920460195FFF79E
:108E3000F7FE034678B162680426103A6260D0E912
:108E400000120220CDE9021202A9C3E9006506F072
:108E50006BFD04B070BD04480FF01CFA40F2F5122F
:108E600001460248FCF784FF882D0660D832066070
:108E700010B50446FFF792FF201DFDF7F9FF0148EA
:108E800010BD00BFE84106602DE9F04F032A0B68D2
:108E9000DFF898B016460CBF164601265B4583B036
:108EA0008846054603D0DA881C49F5F70FF91C49B6
:108EB0002846F4F74BFD00230127DFF874A0DFF804
:108EC000749001930EE03246284621680027FEF791
:108ED00065F949462846F4F739FD32466168284667
:108EE000FEF75CF901A94046FFF79AFE044630B14F
:108EF000002FE8D151462846F4F728FDE3E7094959
:108F00002846F4F723FDD8F800305B4503D0064926
:108F10002846F4F71BFD03B0BDE8F08F9C2D0660DA
:108F2000A02D0660D48A06607C4306601C2F066074
:108F300040290660A4D1076004280AD0052806D17C
:108F40004868C0F31B10400040F00100704700204B
:108F500070474A68034B32F00F02034808BF1846B7
:108F6000704700BF802B0660882B066002282DE921
:108F7000F0410E4682B014460FD02E2809D10022AF
:108F80002146301D43F038FE78B1354802B0BDE8C7
:108F9000F081002002B0BDE8F0818A0728D0A30745
:108FA00003D123682F4A934203D02F4802B0BDE873
:108FB000F08173686268534033F00F03F5D101AF5D
:108FC000043401930AE0296843F016FE0028ECD02F
:108FD00041686868FEF7C2F90028E6D03946304695
:108FE000FFF71EFE054600222046002DEBD1CCE700
:108FF0001E4B0A689A42D2D114F00301D5D12368DE
:109000009342CFD101AF3046CDE900116946FFF759
:1090100007FE394680462046FFF702FE0546B8F1B6
:10902000000F19D0C5B12968D8F80000FEF796F9ED
:109030000028BAD06968D8F80400FEF78FF96946AD
:109040000028B2D03046FFF7EBFD39468046204677
:10905000FFF7E6FD0546E2E758EA050395D0A4E7E9
:10906000882B06601C2F0660802B0660582F066038
:109070000B7A012B04D12E2802D14968FFF776BF65
:109080000020704710B5002204300C4643F0B4FDB8
:1090900008B1406810BD21460148FCF753FE00BFEF
:1090A000D8320660024B40F8043BFDF7B1BE00BF6A
:1090B0001C2F066010B5002104461020F3F7F2F9CA
:1090C000044B2146044640F8043BFDF7A1FE204630
:1090D00010BD00BF1C2F0660F8B50D4606460021E6
:1090E0006868FDF755FA022E044668688CBFAE68C2
:1090F0000B4EFEF757FB00B14010FFF7DBFF0746B2
:10910000051D02E043F078FD46602046FDF7A4FA15
:109110000146012228460029F4D13846F8BD00BF97
:10912000E841066038B505468068FFF7C3FF04468E
:109130002B6803606A684368C2F31B1262F31F1353
:10914000436003F0FC032A79C06802F00102134374
:1091500023712B792279C3F3800363F38202227196
:10916000D5E90221D20043F0B7FC204638BD00BF4C
:109170002DE9F041054682B000201E460F4690467C
:10918000FFF798FF0E4B044605609D4213D056EA48
:10919000070308D00023CDE9004347B932466946AA
:1091A000781C43F035FD204602B0BDE8F081D8F8C8
:1091B00000300193F2E7037943F004030371E6E71B
:1091C000582F066040680009704700BF30B50D4653
:1091D00083B072B1042A04D043F016FD0B4803B0EB
:1091E00030BD0022043043F007FD58B1406803B0A1
:1091F00030BD02226946CDE900051046FFF7D6FDD5
:109200000248ECE729460248FCF79CFDE84106606D
:10921000D832066010B5022282B00B460446694679
:109220001046CDE90043FFF7C1FD204602B010BD56
:109230000430704710B5044682B04068FDF70CFA60
:10924000034660B1A26869460193022053000132CF
:1092500043F00103A260009306F066FB0346184644
:1092600002B010BD30B585B08C4611461A4602AC2E
:109270000C4B05466046019400930223FDF73EFD2A
:1092800000210C20F3F70EF9056004460021029836
:10929000FDF77EF9034620466360039BA36005B09B
:1092A00030BD00BF942F0660F0B50D4611068FB09B
:1092B0001446074602F07F0602D4731E012B12D912
:1092C000022E29D0CEB9E968F9B14B68EBB18A68B2
:1092D000D20726D4012B37D0224638460FB0BDE83E
:1092E000F04006F045B92B68D888F4F737F9014605
:1092F0003846F4F72BFB022E0ED0E968224638469A
:109300000FB0BDE8F04006F033B91F4938460FB042
:10931000BDE8F040F4F71ABB1C493846F4F716FBD9
:10932000D1E71B49286807F06DFAE9684B68002807
:10933000D0D0022BD0D88868322201A909F0B4FD20
:1093400050B9E9684B68C5E70022896838460FB014
:10935000BDE8F040FDF722BFEA6803460D493846F4
:1093600092685210F4F7B2FEEB685A68022A01D0F4
:109370000FB0F0BDD86804F0F1FC0749024638464A
:10938000F4F7A4FEF4E700BF38700760A4D10760CB
:109390007C340660E02F0660F02F06602DE9F04176
:1093A000002482B00D460646194600944FF6FF731E
:1093B000284617462246FDF795FC21461020F3F774
:1093C0007DF8144B002804464FF0000114BF0446FA
:1093D0001C462660A1602DB90F4E2046E66002B003
:1093E000BDE8F08105F102084FEA88084046F3F72E
:1093F00065F806460028EFD0084BA8F10802456042
:1094000039463360083043F067FB2046E66002B01F
:10941000BDE8F081240400201C5006602450066042
:10942000F8B50E4615460446D0E901139A188A424B
:1094300009D2C0682A461844314643F04DFBA26861
:109440002A44A260F8BD02781AB90139C068CD1A61
:10945000F0E705F110070122C0680F443946F3F721
:109460004BF818B1A3686760E060E3E7D4E9015303
:109470002070013DE068ED1ADCE700BF70B51368AD
:109480008EB0144606460D461BB14C2926D00EB0B0
:1094900070BDB1F5BC7F30D000682A4B984203D133
:1094A00040F22143994221D0274907F0ABF9002827
:1094B000EDD040F223239D4218D040F2CE339D429E
:1094C00027D040F233239D421DD0B5F50D7FDED16C
:1094D000F3685A68042A0CD99B690BE01B4B52684D
:1094E0009A42D4D10023C3802360D0E7F3685A683E
:1094F0003AB9164B23600EB070BDC36813600EB04E
:1095000070BD9B68F6E7F3685A68022AF1D91B69B7
:10951000F0E7F3685A68012A02D9DB682360B6E7EE
:10952000002AE6D0322201A9986809F0BDFC054660
:109530000028DED043F029FB0146284603F026FD33
:109540002060A4E7A83506607C340660E841066028
:10955000C3685A680AB1986870470148704700BFED
:10956000E8410660002310B4C4681A461946A446B0
:109570005DF8044B604700BF10B582B00023C4689B
:10958000019101AA0121A04702B010BD10B4C46826
:109590000023A4465DF8044B604700BF2DE9F04767
:1095A00086B00D4606460021102000AF9046F2F727
:1095B00085FF044628460EF003FE00218146F2F79F
:1095C0007DFF002C44D000283CD001234FF0000A3E
:1095D000C7F80C9007F108093B72214B78612846C7
:1095E0007B60C7F810A0C7F800900EF0E9FD0346B5
:1095F00028466D46073323F00703ADEB030D69469C
:109600000EF0E2FD694642463846F4F723FCD7E9FE
:10961000043202F803A03B69A3607B69E360AD46B6
:10962000D4E902100F4B2360F3F76EFE0023606055
:109630004A4601213046BC60FFF7B0FE1837BD46F0
:10964000BDE8F087014607F10809C4E90200E9E72F
:109650002346224621463046FFF7A0FEEEE700BF34
:1096600021940160984D06600EB400B582B003AA43
:1096700052F8041B0192FFF791FF02B05DF804EB72
:1096800003B07047FFF7F0BF830703D1064B0268B2
:109690009A4202D0054907F0B5B8054BC2689A4214
:1096A000F8D10120704700BF94530660BC300660BB
:1096B0009D93016008B5FDF769FDBDE80840FFF71F
:1096C000E3BF00BF10B582B004460191FFF7F2FF7F
:1096D000019928B9204602B0BDE8104007F092B8C1
:1096E0002046FDF753FD04460199204602B0BDE82F
:1096F000104007F087B800BF10B50446FDF746FDDF
:10970000044BC2689A424FF0000318BF2469A3605B
:1097100010BD00BF9D930160F8B5044616461D4676
:109720000F46FDF733FD184BC2689A4218BF2469F3
:10973000A068F0B1E388A1889A1C8A4208DA00EB9D
:10974000830003339BB2E3808560C0E90076F8BDF7
:10975000033101228900F2F7CFFE0028F7D0E38819
:10976000A288A06000EB830003320333A2809BB287
:10977000E9E701460C20F2F7A1FEA0600028E6D040
:109780000323A380DFE700BF9D93016070B504460B
:1097900015460E46FDF7FAFC074BC2689A4218BF01
:1097A0002469A36823B1E3883360A3682B6070BD8C
:1097B00033602B6070BD00BF9D93016070B50F4E8C
:1097C00082B0054609E06868B04202D0FCF7BEFBF3
:1097D0000446204643F00CFA60B9A868FCF73CFF49
:1097E00001AB00220121044601900028EBD1204664
:1097F00002B070BD019C204602B070BDE841066019
:1098000070B5002482B00646084619460223154664
:1098100000941A46FDF766FA21460C20F2F742FE44
:1098200006602B682146044643606868FCF7B0FE7A
:1098300003462046A36002B070BD00BF01F1FF43A4
:1098400023F00303072805D8DFE800F00D0F040418
:10985000180423060020704707EE903AF5EEC07A10
:10986000F1EE10FA01D40846704783F0004323F06C
:10987000030141F00201A1F1FF40704707EE903A69
:1098800009490A48F5EE407AF1EE10FA18BF084689
:10989000704707EE903AFDEEE77A17EE903A5900DE
:1098A00041F00100704700BF882B0660802B0660E6
:1098B00001F1FF41672230B521F0030387B0002595
:1098C000044600EE103A1021062302A80095FBF78B
:1098D0002DFA02A92046F4F739F82E2102A843F008
:1098E0003DF908B107B030BD652102A843F036F953
:1098F0000028F7D16E2102A843F030F90028F1D1F9
:1099000002492046F4F722F8ECE700BFF43807607C
:1099100038B5D1ED000A054690ED000A0C462DED54
:10992000028B31F02DFCB5EE400AD5ED007AB0EE99
:10993000408AD4ED000A77EEC07AF1EE10FAC7EE55
:10994000A08A43D0B5EEC00AF1EE10FAF5EEC00AD7
:109950004CBF01220022F1EE10FA4CBF012300237C
:109960009A4205D0F7EE007A30EE208A78EEE78A48
:10997000F5EE408AF1EE10FA10D1D5ED000AD4EDE3
:10998000007A9FED160AC0EEA70A43F0D5F885EDE0
:10999000000A84ED008ABDEC028B38BDB0EE680A87
:1099A00031F03EFBF6EE007A78EEC08AF4EEE78AFC
:1099B000F1EE10FAEBDDF7EE007A30EE270A85EDD6
:1099C000000A84ED008ABDEC028B38BD9FED030ACE
:1099D00043F0B2F8B0EE408ACAE700BF00000000D2
:1099E00070B50C4686B0002619461546012332464E
:1099F00020460096FDF776F914B9134806B070BDFD
:109A0000012203A92868FDF761FFA0B9286800F0CA
:109A10000303022B0AD0FDF7B7FD10EE103A23F036
:109A2000030040F00200A0F1FF40E7E7074B0340CE
:109A3000062BE3D1EFE7334632460096DDE903011A
:109A4000FBF760FDDAE700BF02008080070080FFBF
:109A500030B50D4687B0044603A928468DED010AAE
:109A6000FDF750FD00283FD02D2C3FD8DFE814F043
:109A7000ED00FA0007011401C2003E003E003E0066
:109A80003E003E003E003E003E003E002E00AF0085
:109A90005F0068007500830041003E003E003E000C
:109AA0003E003E002E00AF005F006800750083009E
:109AB00041003E003E003E003E003E003E003E00B3
:109AC0003E003E003E003E003E00CF009DED010AFC
:109AD000DDED037A70EE277A17EE900A20F003008E
:109AE00040F00200A0F1FF4007B030BD002007B0F9
:109AF00030BD9DED010ADDED030AB5EE400AF1EE41
:109B000010FA6DD1F5EEC00AF1EE10FA68D5F0EE5C
:109B1000E07A9FED787AF4EE477AF1EE10FA5FDCA6
:109B200075480EF0B7FB01467448FCF711F99DED3E
:109B3000010ADDED037A60EE277A17EE900ACDE791
:109B4000DDED037AF5EE407AF1EE10FAE8D001A8E7
:109B500003A9FFF7DDFE0198C0E7DDED037AF5EE1E
:109B6000407AF1EE10FADBD09DED017AC7EE277A4C
:109B700017EE900AB2E7DDED030AF5EE400AF1EECA
:109B800010FACDD09DED010A31F0FAFAB5EE400A97
:109B900010EE100A8DED010AF1EE10FA00F0978038
:109BA000B5EEC00ADDED037AF1EE10FAF5EEC07AFB
:109BB0004CBF01220022F1EE10FA4CBF012300231A
:109BC0009A428BD070EE277A17EE900A86E79DEDC9
:109BD000010ADDED037A70EE677A17EE900A7DE7F1
:109BE000B5EEC00AF1EE10FA63D430F085FB10EE4A
:109BF000100A73E79DED017ADDED037A404BB4EE78
:109C0000E77A4048F1EE10FAB8BF18466CE7DDED90
:109C1000037AF5EE407AF1EE10FA81D003A901A89B
:109C2000FFF776FE019A039B022022F0030204A9AB
:109C300023F0030302430343A2F1FF42A3F1FF43D6
:109C4000CDE9042305F070FE4EE79DED017ADDEDD0
:109C5000037A2B4BB4EEE77A2A48F1EE10FA58BF9C
:109C6000184641E79DED017ADDED037A244BB4EE11
:109C7000E77A2448F1EE10FAD8BF184634E79DED94
:109C8000017ADDED037A1F4BB4EE677A1C48F1EEE2
:109C900010FA08BF184627E79DED017ADDED037A3B
:109CA000174BB4EEE77A1748F1EE10FA88BF184662
:109CB0001AE7B0EE600A31F0B3F9DDED030AB4EE55
:109CC000600AF1EE10FA0BD19DED010A8DE7DDED92
:109CD000030A9FED0D0A42F02FFF10EE100AFDE679
:109CE0002946DFED090A9DED010A2020FEF784FEDA
:109CF000FAE600BFFFFF7F7FCC2C06604C37066082
:109D0000802B0660882B06600000000001F1FF43F5
:109D10008446114623F0030300EE103A930703D163
:109D2000054B12689A4202D06046FFF791BEDFED04
:109D3000030AFEF761BE00BFF82C066000000000B9
:109D400007EE901A06EE900A9FED047AF8EE677A15
:109D5000B8EE660AA7EE870A704700BF0000804F82
:109D6000DFED067ABCEEC07A60EE277A17EE100AB5
:109D7000FCEEE77A17EE901A704700BF0000802FC4
:109D800010B5002382B004460846009311461A46D7
:109D9000FCF772FF636802B0BDE81040184700BFCF
:109DA00070B51C4682B00123002605460846009681
:109DB00011461A46FCF760FF6B68206802B0BDE8E8
:109DC0007040184770B51C4682B002230026054635
:109DD0000846009611461A46FCF74EFF6B68D4E918
:109DE000000102B0BDE87040184700BF70B51C46C6
:109DF00082B00323002605460846009611461A46FF
:109E0000FCF73AFF6B682068D4E9011202B0BDE8A4
:109E10007040184770B51E46037988B00D4603F0B0
:109E200001031146828804460093C2F34E02C388A0
:109E300028460391FCF720FF2379039913F0010FC3
:109E400006D1A3683146284608B0BDE870401847DF
:109E500006EB850205A8FCF7EFFFA36805AA3146CB
:109E60002846984708B070BD08B509F09FF80088EB
:109E700008BD00BF08B5806809F098F809F096F8A9
:109E80000430BDE80840FFF7EFBF00BF10B504463F
:109E900082B008460191FFF7EDFF019B024603499E
:109EA000204602B0BDE81040F4F710B90038066053
:109EB0002DE9F8430E46914698460546D0B14768CD
:109EC00041B3781D00218000F2F7ECFA224B0446E2
:109ED00005F108010360BA00204B9B69C0E90298B4
:109EE0004360103042F0F8FD043744F82760204604
:109EF000BDE8F88321B329461420F2F7D3FA164BB4
:109F00002F4604460360154B9B69C0F80C80C0E9DE
:109F10000139E9E7381D8000F2F7C4FA0E4B044618
:109F2000BA00036005F108010C4B9B69C0E90139D7
:109F3000C4F80C80103042F0CFFD2046BDE8F88315
:109F40001020F2F7AFFA044A044B044602609B6902
:109F5000C0E902984360CAE7183806600004002090
:109F60002DE9F041456882B006460F46A868019287
:109F7000009309F00FF88046A86809F017F809F077
:109F800009F808F1080800EB400400214444A0004F
:109F9000F2F788FA04460A4839462060307A0026EB
:109FA00020726868DDE90032606004F10C00C4E9E9
:109FB000035609F001F8204602B0BDE8F08100BF69
:109FC000243B06601C3008B550F8083C834202D0A0
:109FD0001868196008BD02480EF05CF9FBF724FF11
:109FE0008039066008B5037A03B108BD04480EF055
:109FF00051F901460348FFF737FBF2F72DFA00BF8E
:10A00000AC3906608030066070B50B7A05460C46A8
:10A01000C8684BB9FFF72EFF23460246074928467A
:10A02000BDE87040F4F752B8FFF724FF234602461C
:10A0300003492846BDE87040F4F748B8043A066082
:10A04000E439066008B50248FFF78CFAF2F704FA23
:10A05000A835066038B505460C460C200021F2F7FD
:10A0600021FA024A0472C0E9002538BD603B06604F
:10A070002DE9F84304461F460E461546FCF7ECFD55
:10A080002369002B4ED0636904F11C0293423ED039
:10A090001A68DFF8B080424542D0154600221A60A7
:10A0A0006368002B43D0244E4FF00009294604F189
:10A0B0000C00B269B361E261C4F8049042F0ACFDF7
:10A0C000B369012805466360E369B36116D00228CD
:10A0D00007D063692846C4F810901B683B60BDE850
:10A0E000F883E368986808F055FFC4F8109004EB13
:10A0F00080042846E3693B60BDE8F883636928462D
:10A100001B683B606369C3F80080BDE8F883DFF833
:10A1100034804645C4D009480EF0BCF8FBF784FEF5
:10A120001E60BDE71D463B602846BDE8F883044835
:10A130000EF0B0F8FBF764FE00040020243A06603D
:10A140005C3A0660E841066000B583B001ABFFF7FA
:10A150008FFF01280AD002280CD0019B13B1114AAD
:10A16000934217D1002003B05DF804FB019803B0BF
:10A170005DF804FB0198FDF709F80B4906F042FB76
:10A1800028B10198FFF7E4F9064B8342EAD0019821
:10A19000F2F762F901AA01210348FFF7F7F9F2F794
:10A1A0005BF900BFE8410660A835066008B50228E3
:10A1B0000B460CBF4A688A6818680349FFF7C4FF5A
:10A1C00000B108BDFFF73EFFE841066008B5002278
:10A1D000FFF7BAFF00B108BDFFF734FF08B5027AF8
:10A1E00022B90549BDE80840FFF7AEBF03480EF0AD
:10A1F00051F8FBF719FE00BFE8410660783A0660A7
:10A2000000B583B0114A124901ABFFF731FF0128B5
:10A2100017D0022806D10198FCF7B8FF0D4906F0C7
:10A22000F1FA18B10A4803B05DF804FB0198FCF795
:10A23000ADFF094906F0E6FA0028F3D10198F2F7DC
:10A240000BF906480EF026F8FBF7BEFDF82F066066
:10A25000E8410660E8310660A8350660A03A06606D
:10A2600010B596B0044603A8F2F7DEF850B1049892
:10A270000E4A0368934202D00D4A934214D1002043
:10A2800016B010BD0146221D0120FBF7D5FEE36884
:10A29000019023F00103023343F00103E360F2F77E
:10A2A000BBF8019816B010BDF2F7D6F89C320660E4
:10A2B000A835066010B40346054C012208460C6020
:10A2C0001C684C605B685DF8044BC1E90232704762
:10A2D0009C3B0660C2070DD5401009D0B0F1404F3D
:10A2E0000AD00028B8BF4042B0FA80F0C0F1200088
:10A2F00000F078BC00F03ABB202000F073BC00BF37
:10A3000030B50C4685B0012201A96068FDF7F4FA6A
:10A31000A56841F2A6539D42DDE9012120D0944673
:10A3200001244B1E11B3013B002002E0B0F5800F69
:10A330000DD29CF800E0B3F1FF3FA44403F1FF33DA
:10A340004EEA0020F2D100F04DFC05B030BD41F2E4
:10A35000A650281A18BF012000F018FB05B030BD28
:10A360004B1E4FF0FF3402EB030CDBE70846EAE735
:10A37000002800B583B000DA92B1032905D83AB9B4
:10A38000CA000123934098420ADA03B05DF804FB47
:10A39000CB000122013B02FA03F35A429042F2DA67
:10A3A000034801910DF076FF0199FCF703FC00BF13
:10A3B000D83B0660F0EEC07A10B5F4EE677A2DED6A
:10A3C000028BF1EE10FAB0EE408A2CD69FED1E7A89
:10A3D000F4EE477AF1EE10FA2DDC10EE103A1A1E68
:10A3E0001BDB1A4B1340B3F19C4F0BD900F07CFAE6
:10A3F000B0EE480A04460430F4F708F92046BDECF4
:10A40000028B10BDFDEEC87ABDEC028B17EE900AF0
:10A41000400040F00104204610BD32F00043F1D06E
:10A4200002F1FF43DFE70A480DF034FF40F28522D6
:10A43000FE21FBF7EDFC06480DF02CFF40F28522D3
:10A440004FF42071FCF7B6FBFFFF7F7F000080FF19
:10A45000B826066070B50C4686B00026194615462B
:10A460000223324620460096FCF73CFCECB1012C5E
:10A470001ED12868C30716D410F003022AD102683F
:10A48000204B9A420FD0204B0340062B03D01F4B8A
:10A4900092699A4224D105A903F07AFC0023059918
:10A4A0001A46FAF787FF06B070BD012006B070BDEE
:10A4B00005A9286803F06CFC0599044668680391B7
:10A4C000FCF7B2FF3346024603992046FAF772FFC3
:10A4D00006B070BD0C4B0340062BDCD0022A05D021
:10A4E000FCF7A2FF400040F00100DCE700F1FF4074
:10A4F00020F0030300EE103A06B0BDE87040FFF70D
:10A5000059BF00BF703C0660070080FFF5E40160A2
:10A5100038B50B4C214411F8014CB0FBF4F463B195
:10A52000084D631CA5FB03135D0810460AB142F0F9
:10A530002CFB03342C44204438BD1D46F5E700BFF6
:10A54000603C0660ABAAAAAA2DE9F04F85B0804610
:10A550008B469DF840409DF84490029413F001040E
:10A5600001920094DDE90E6700F09E805D1040D4FA
:10A570004B463A4631462020FFF7CAFFDBF8003051
:10A58000824683424FF0000300930393C0F0838020
:10A59000D8F800B000230BEB0A0000F8013C002DB6
:10A5A00040F08B803023841E00F8023C7FB1384697
:10A5B00042F0EBFA201A584509D93B7833B10246EC
:10A5C00002F8013B17F8013F002BF9D104465C4526
:10A5D00004D9009B13B1039B013C2370D8F80030D1
:10A5E0002046019A53441B1B013B136005B0BDE894
:10A5F000F08F4B463A4631462020FFF789FFDBF8C3
:10A6000000306D428246834243D3D8F800B0002325
:10A610002D225844039200F8013C0138029BB9F105
:10A62000000CCDF808900146A3F10A0318BF4FF0C3
:10A63000010C9946B5FBF6F306FB13541D46092C95
:10A6400004F1300288BF09EB0402003B01F1FF3442
:10A6500018BF012301F8012C5C4594BF00220122A0
:10A6600013EA0C0F02D0A0EB040E2AB9002B9DD0E8
:10A67000002A9BD02146DDE7BEF1030FFAD18C1EE4
:10A68000029A5C4501F8022C204694BF0022012268
:10A69000ECE72D23039300215046F1F703FFC8F8A0
:10A6A0000000CBF800A073E7029CCDF84490109412
:10A6B00005B0BDE8F04F00F027B90138AEE700BFA4
:10A6C00070B58CB00B4600250A22102108AE044656
:10A6D0000092069107AA06A905A801950596CDE95D
:10A6E0000255FFF731FF01462046F3F72FF9059891
:10A6F000B04201D0F1F702FF0CB070BDF0B50546D5
:10A7000083B00E4614463AB3012000F0CDF9019013
:10A71000F300581E00F0C8F9019902460C2042F0DF
:10A720005FFA0746294600203A4642F059FA184B8C
:10A73000044698420AD139460120FBF789FB294695
:10A740000246042042F04CFA84421ED011480DF01B
:10A75000A1FD3146FCF72EFA00F03EF90028F5DBAA
:10A76000012000F0A1F90146F000019100F09CF9F0
:10A77000019902460C2042F033FA2946024620464F
:10A7800042F02EFA024B8342E0D103B0F0BD00BF8D
:10A79000882B0660D83B06602DE9F0438DB0304B26
:10A7A0000D46013805AC0431CDE900340323FCF734
:10A7B000A5FA059C002C4FDBDDF8188041F2A6516C
:10A7C00008A82D68B8EB010721469DF81C9018BF1A
:10A7D0000127F2F789FF0A9E22460021304642F007
:10A7E000A3F9EB072CD56B1014D018464A46214626
:10A7F0000393FFF7BDFD042C039B254628BF0425CA
:10A80000002B0BDA22464FF0FF31304642F08CF934
:10A81000039B03E0042C254628BF042541F2A652E1
:10A82000904501D0641B264432463946284607F03D
:10A8300087F808A90B4802F073FB0DB0BDE8F08360
:10A840004A4621462846FFF759FF334622463946F5
:10A85000284600F0ADF8ECE70020FBF7D1FA00BF86
:10A86000F83B0660044B066008B1FFF781BD7047F6
:10A8700013460A4610B4164CA3421FD0154CA342EF
:10A8800021D01C2810D114491940062910D099074D
:10A890000AD1196811488C69844209D01048814254
:10A8A00006D01048814203D000205DF8044B704769
:10A8B00019461C205DF8044B42F092B901225DF864
:10A8C000044B42F08DB903225DF8044B42F088B985
:10A8D000802B0660882B0660070080FFF5E401608E
:10A8E000245006601C3E066010B500211020F1F7D0
:10A8F000D9FD044B044640F8043BF3F723FE204601
:10A9000010BD00BF703C06602DE9F04F85B00546D4
:10A9100098680E46DDF838801C46DDF83C901746F6
:10A920009DF844A000014A46414653469DF840B078
:10A93000FFF7EEFD336883420FD3CDF800A05B46EE
:10A940002D684A464146201D0195F4F757FE0346FF
:10A9500028463B6005B0BDE8F08F00210390F1F779
:10A96000A1FD039A28603260E7E700BFD0E9023119
:10A970006FF000421A44013331F81200B0FA80F04F
:10A98000C0EB0310400040F00100704710B50C46CA
:10A9900082B001920090FFF7A7FF22460446019B78
:10A9A00004300099F3F7F2FE204602B010BD00BF5C
:10A9B00070B5044682B00D46164600211846019334
:10A9C00042F0B2F8019B32462946201D02B0BDE894
:10A9D0007040F4F7B3BD00BFC30706D54010002890
:10A9E0000FDB14BF01200020704783683BB103795F
:10A9F00013F0010F14BF4FF0FF30012070471846CD
:10AA000070474FF0FF30704720B50D46072805D836
:10AA1000DFE800F005121B0424042C07002528465B
:10AA200020BD0B79DB07FAD5FFF75EFF291D054630
:10AA30000430F3F729FFF2E7FFF756FF291D05461B
:10AA40000430F3F72DFF284620BDFFF74DFF291DE9
:10AA500005460430F3F734FF284620BD8B680748CD
:10AA6000074D002B18BF0546284620BD081DF4F7EA
:10AA700031FD400040F00105284620BD882B0660CE
:10AA8000802B066010B584B003910290FFF72CFF75
:10AA900001210446029A0430039B0091F3F788FDDC
:10AAA000204604B010BD00BF90EA40024FEA4003C8
:10AAB00002D443F001007047C117FFF7E3BF00BFA6
:10AAC00010B584B003910290FFF70EFF00210446F9
:10AAD000029A0430039B0091F3F76AFD204604B00C
:10AAE00010BD00BF2DE9F04710F001088AB00646FE
:10AAF0000C46154605D181073CD1364B02689A4277
:10AB000038D114F0010A2FD015F0010905D1AB0797
:10AB100030D1304B2A689A422CD100200021FFF717
:10AB2000CFFF0746B8F1000F35D10436BAF1000F58
:10AB30002BD10434B9F1000F21D104356B68002BFF
:10AB400040D02B4622463146381DF4F75DFC01AB60
:10AB50009E422DD004AB9C4230D007AB9D4220D00A
:10AB600038460AB0BDE8F087A20703D1194B226826
:10AB70009A42C9D018480DF08DFBFBF755F96910C2
:10AB800007A807ADF3F7E4FCD8E7611004A804AC0C
:10AB9000F3F7DEFCCEE7711001A801AEF3F7D8FCA5
:10ABA000C4E72846F3F7E8FC38460AB0BDE8F0876A
:10ABB0003046F3F7E1FC04AB9C42CED12046F3F7DC
:10ABC000DBFCCAE705480DF065FB01460448FBF7CE
:10ABD000BFF800BF703C0660AC3C0660D83C066025
:10ABE0001037066010F0404F03D1400040F00100E4
:10ABF00070470021FFF764BF70B5044684B01E465D
:10AC00000D460392FFF770FE039B2A460096054609
:10AC100021680430F3F766FD236802462846134492
:10AC2000236004B070BD00BFC30701D5401070475A
:10AC30000430F4F74FBC00BFC30700B583B003D5A1
:10AC4000401003B05DF804FB01A90430F4F756FC92
:10AC500018B1019803B05DF804FB03480DF01AFB2E
:10AC600001460248FBF774F8F83C0660B834066009
:10AC70002DE9F0430D4607461446E9072DED028BFA
:10AC800089B054D405F10408E2072AD414F0030370
:10AC900013D12368964A934200F08580954A9342E7
:10ACA00076D0294622463846FFF7E2FD054628467B
:10ACB00009B0BDEC028BBDE8F083022BF1D18E4BC5
:10ACC0002340062BEDD04046F4F778FC2146384669
:10ACD000FEF7BEFE0546284609B0BDEC028BBDE876
:10ACE000F08302AE6310022201A902A8F3F738FC38
:10ACF0001E2F25D0122F23D0A7F109095FFA89F35F
:10AD0000242B39D8FFF7F0FD0546B9F1170F00F2F3
:10AD1000CB80DFE809F0C3BDB76A6AA5B1AB95C9BE
:10AD20008579C3BDB76A6AA5B1AB95C985796B1042
:10AD3000022201A902A80DF10808F3F711FCA3E70C
:10AD40007368002B00F0C6804046F4F737FCB0EE85
:10AD5000408A3046F4F732FCC8EE007A17EE900ACB
:10AD600020F0030040F00200A0F1FF45284609B0A2
:10AD7000BDEC028BBDE8F08331464046F3F762FD3F
:10AD8000042F00F2B380DFE807F029231D1710001D
:10AD90004046F4F713FC2146DFED580A3846FDF72C
:10ADA0002BFE054683E7261DA2E7554D554B15EAB8
:10ADB000200538BF1D467AE7514D524B0028D8BFB9
:10ADC0001D4674E74E4D4F4B002808BF1D466EE7E9
:10ADD0004B4D4C4B0028C8BF1D4668E7484D494BBA
:10ADE00035EA200528BF1D4661E72046FFF724FF0E
:10ADF000021E76DB182F414605F1040067D00C2FA8
:10AE000065D0F3F7FFFD52E773681BB13378DB07BA
:10AE10003FF559AF32464146281DF4F747F946E75A
:10AE20007368002B56D005A8F3F78CFB05A83346B2
:10AE30004246291DF4F77EF905A8F3F79DFB36E796
:10AE40007368002B46D005A8F3F77CFB281D33461A
:10AE5000424605A9F4F76EF905A8F3F78DFB26E73E
:10AE6000324641460430F3F739FE20E73246414688
:10AE70000430F4F78BF81AE7324641460430F3F712
:10AE80006DFE14E7324641460430F3F7B7FE0EE795
:10AE9000324641460430F3F7F3FF08E732464146B5
:10AEA0000430F3F751FF02E773689BB1FFF71CFD15
:10AEB000291D3346044642460430F4F73BF905A900
:10AEC0000220CDE9054504F02FFD0546EFE6F3F736
:10AED00037FDECE60C480DF0DDF901460B48FAF7BA
:10AEE00037FF0B480DF0D6F9FAF78AFF0025DEE6AA
:10AEF000703C0660F82C0660070080FF0000000030
:10AF0000802B0660882B0660CC2C06604C370660D0
:10AF1000F82306600430F4F751BB00BF10B4054AB3
:10AF20000023054CC1E90203C1E9004208465DF86F
:10AF3000044B70473DAF016008410660D0E9021242
:10AF400003468868824205D2C868511C50F8220026
:10AF5000D960704700207047104938B505F0F4FCFF
:10AF6000816800298C46B8BF01F1010C01294FEA24
:10AF70006C0C11DD6FF0404200230A449200C1685E
:10AF80008D5851F8234041F823500133C16863457F
:10AF90008C50A2F10402F2DB014838BD1C3E066071
:10AFA000E84106600B460C4910B50446184605F00A
:10AFB000CBFC042C08D0052C04D18068400040F064
:10AFC000010010BD002010BD8268044B0448002A17
:10AFD00008BF184610BD00BF1C3E0660802B0660EF
:10AFE000882B066038B50D46114905F0ADFC0446C6
:10AFF000D0E901138B4206D2E268591C0D48A160CA
:10B0000042F8235038BDC900C068F1F769FA002141
:10B01000E060D4E9012352006260D21A0133013AA0
:10B0200000EB8300920041F07FFDA368E4E700BFDE
:10B030001C3E0660E841066038B50B460446002118
:10B040001846FBF7A5FA054601E0FFF7CBFF2846B7
:10B05000FBF702FB014620460029F6D138BD00BFB0
:10B0600038B50949002505F06FFC04461021C06879
:10B07000A560F1F735FA042329461022E0606360E9
:10B0800041F052FD014838BD1C3E0660E8410660B3
:10B090002DE9F84F83468A4615469846FBF7DCFDB6
:10B0A000D34551D2ABF10409002D58D0DAF8001085
:10B0B0002846FAF7A9FF0746544609F10406B442A8
:10B0C00016D931681DB12846FAF79EFF01463A4667
:10B0D000002041F085FD80450AD11AE02168FAF789
:10B0E00093FF39460246002041F07AFD80450CD19D
:10B0F000043C2846A6420ED2002DEFD122683946E4
:10B10000002041F06DFD8045F2D033682268326046
:10B110002360B146D1E7AAEB0603A4EB0B0230682B
:10B120009B10DAF80010013B3160CAF80000B3EB65
:10B13000A20F0BDD584643462A46214609F1080B6B
:10B14000FFF7A6FFDA45ADD8BDE8F88F5146434674
:10B150002A4609F10800A246FFF79AFFF2E7DAF85B
:10B160000070A9E730B585B0134B0C46013802AD2D
:10B170000431CDE900350223FBF7C0FD0F492068FB
:10B1800005F0E2FB8368012B13D90D4C6FF04041B1
:10B19000029A1944C068A24208BF00229DF80C50D0
:10B1A000084B00EB8101084C002D08BF2346FFF738
:10B1B0006FFF034805B030BD403D06601C3E066091
:10B1C000E8410660802B0660882B066010B50C46AF
:10B1D00082B007490190206805F0B6FB2346019A2A
:10B1E000D0E9021002B0BDE8104005F00FBE00BF6C
:10B1F0001C3E066000B50A4683B00649019205F080
:10B20000A3FB019AD0E9021003B05DF804EB05F04E
:10B210003FBE00BF1C3E06602DE9F041032A0D46EB
:10B220001249174606460CBF17460127F2F78EFB58
:10B23000AB68A3B10024DFF83C80EB683A463046A7
:10B2400053F824100134FBF7A9FFAB68A34206D9D9
:10B25000002CF2D041463046F2F778FBEDE730465D
:10B260000349BDE8F041F2F771BB00BF3C3D066009
:10B270003C2906604029066070B511F003060C46B3
:10B28000034603D11E4A0D68954205D02146184653
:10B29000FFF7D2FE1B4870BD294605F055FB03465B
:10B2A000204629461C4605F04FFB82680546A368E8
:10B2B0006068991881420CD8E0689200E96800EB58
:10B2C000830041F009FCA368AA680E481344A360F8
:10B2D00070BD0431E0688900F1F702F9A368E0600D
:10B2E0003146AA681A4404326260AE683344D21A06
:10B2F00000EB8300920041F017FCA368AA68DBE72B
:10B300001C3E0660E841066070B50C4613491546C0
:10B3100005F01AFB631082680646114948BF9B1866
:10B3200023EAE374944228BF1446FFF75BFEB26839
:10B33000531EA3420DD90B4911444FEA810CF16809
:10B3400051F80C20ACF1040C41F82320013BA3423E
:10B35000F5D1F368024843F8245070BD1C3E0660E6
:10B36000E8410660FEFFFF3F70B50D4606461F49E7
:10B37000286805F0E9FA012E04464FF0000314BFD7
:10B380006A684FF0FF320068A168FCF7B9F9A2685B
:10B390002AB3E368013A53F8205003EB8001A2601E
:10B3A000121A08460431920041F0A4FB0021D4E9AE
:10B3B000022343F822106168042903D9A368B1EB82
:10B3C000430F01D8284670BD4908E0688900F1F7AD
:10B3D00087F86368E06028465B08636070BD0448D6
:10B3E0000CF058FF40F2B221FAF7FEFC1C3E06605A
:10B3F000882D066000B583B002460B4602206946E0
:10B40000CDE90023FFF7E2FE0346694602200193DF
:10B41000FFF7AAFF014803B05DF804FBE8410660AE
:10B4200038B5826804462AB3C068013A50F8215002
:10B4300000EB8103A260521A1846191D920041F0D8
:10B4400059FB0021D4E9022343F822106168042942
:10B4500003D9A368B1EB430F01D8284638BD49088A
:10B46000E0688900F1F73CF86368E06028465B0813
:10B47000636038BD03480CF00DFF40F2B221FAF7CB
:10B48000B3FC00BF882D06602DE9F04107460E464B
:10B490000D499046FFF7A6FDBA68531EB3420DD979
:10B4A0000A4C14444FEA840CFC6854F80C50ACF17C
:10B4B000040C44F82350013B9E42F5D1FB6843F84D
:10B4C0002680BDE8F08100BFE8410660FEFFFF3F37
:10B4D00038B50D4604460C4A0021042D2B46026067
:10B4E00038BF0423856063609800F0F7DBFF626873
:10B4F00003460021521B00EB8500E3609200BDE88B
:10B50000384041F011BB00BF1C3E066010B5044638
:10B5100000211020F0F7C6FF21460446FFF7D8FFB0
:10B52000204610BDF0B50E46044685B03B49304676
:10B53000154605F009FA07461C2C15D8DFE804F07B
:10B5400018181818181414141414141414143D147E
:10B550001414141414141414141420140F0003A934
:10B560002846FBF79FFF80BB0024204605B0F0BDB6
:10B57000AB0742D0022CF7D1294C204605B0F0BDD4
:10B5800015F00304F0D1254B2A689A42EDD1AB683F
:10B5900080681844FFF7BAFF0446C068D7E9022163
:10B5A000920041F099FAAA68B868E3689200E968E5
:10B5B00003EB800041F090FAD7E734462946304645
:10B5C000FFF75AFE204605B0F0BD0399002902DAC4
:10B5D000002319460393B86805F07CFAFFF796FF3D
:10B5E0000446D7E90223E1681846039B0091042131
:10B5F00005F080FA204605B0F0BD084B2A689A4253
:10B60000B8D1D0E902212046D5E90243009405F0E3
:10B61000A5FB0028B0D0034CA7E700BF1C3E066086
:10B62000802B0660882B066070B50C4682B0002621
:10B63000194615460123324620460096FBF752FB79
:10B640002CB9204602B0BDE87040FFF75FBF30461E
:10B65000FFF75CFF296802B0BDE87040FFF7ECBC63
:10B6600038B50C460546FFF751FF64B15DB1231FA5
:10B67000C4F1040103EB850CCA1853F8045FC468D5
:10B680006345A550F8D138BD044908B505F05CF90B
:10B69000BDE80840D0E90201FFF7E2BF1C3E0660AA
:10B6A00038B50D460449144605F04EF983682B6001
:10B6B000C368236038BD00BF1C3E066081607047D0
:10B6C00030B5154683B00A460749019205F03CF9AA
:10B6D000044681680023019A0068FCF711F8E368CA
:10B6E00043F8205003B030BD1C3E0660F0B515464F
:10B6F00089B00C46724905F027F907461DB3042DA1
:10B700000FD014F0030603D16E4B22689A4257D033
:10B710002A46214638466C4EFFF7D2FF304609B024
:10B72000F0BDA30703D1674B22689A4279D000236A
:10B730002246B9683868FBF7E3FFFB6853F82060DE
:10B74000304609B0F0BD14F0030503D15D4B22680B
:10B750009A4209D005A90220CDE90574FFF704FE3D
:10B76000594E304609B0F0BD02AA2146806805F066
:10B77000D5F9002800F0A18002982A46F968039CB8
:10B78000041B01EB800041F0A7F903990298D7E967
:10B790000223521A03EB800003EB8101920041F077
:10B7A000A9F92946C4EB8472D7E9023092002344F8
:10B7B00000EB830041F0B8F9BB682344BB60CFE7DE
:10B7C00001AA28466946FBF75DFF05AA2146B8682D
:10B7D00005F0A4F9002870D00598009A06998318FE
:10B7E0005C1A002C2BDDBA6878682244824247D864
:10B7F000F868D21A00EB810100EB8300920041F05F
:10B8000079F9009A0598FB689200019903EB800092
:10B8100041F070F9BB682C4E23443046BB6009B040
:10B82000F0BD2146806805AA05F078F9002834D1DA
:10B8300005AAD7E9020105F02DFA06466EE7FB6876
:10B840009200019903EB800041F046F90699059BAF
:10B85000009DD7E902202B44521A00EB810100EB36
:10B860008300920041F046F9B868C4EB8472FB682B
:10B8700020443146920003EB800041F055F9C9E7BE
:10B880009100F868F0F72CFEBA68F860224400993D
:10B890007A60059B0B440699ABE7DDE90530C01AD9
:10B8A000FFF734FE0599FB680646D0E9022003EB5A
:10B8B0008101920041F010F930E70020FBF772F9A6
:10B8C0001C3E066044460660E84106602DE9F047EC
:10B8D0008046406800218000F0F7E4FDD8F80410AD
:10B8E0008146C1B108F10806071F002505E047F8A9
:10B8F000040FD8F80410A9420DD956F8040F0135E9
:10B90000FAF7AAFE04460028F1D14846F0F7F6FD02
:10B910002046BDE8F0874B46D8F808000022BDE875
:10B92000F047FAF713BB00BF2DE9F0410E4682B095
:10B930000024194607464FF6FF733046154600941B
:10B940000222FBF7CFF9B01C013E21468000F0F740
:10B95000A9FD8046C0E900762B6883605EB100F1E6
:10B9600008070134002155F8040FFAF711FEA6422A
:10B9700047F8040FF5D1404602B0BDE8F08100BFA2
:10B9800070B51446126882B0002A36D04568C900E6
:10B990002B799B070FD441F00601606848B30191F1
:10B9A000F1F728FA01990246284641F02DF90023C3
:10B9B000236002B070BD41F006010022281D0191F4
:10B9C00041F01AF9019918B1426863689A42EED0C1
:10B9D000104B9D42EDD1104ED6F89850002DDCD181
:10B9E00001200191FDF766FB01990546C6F8980014
:10B9F000D3E72846FDF70EFCD9E7C900406841F0BF
:10BA00000601043041F0F8F80028D2D043682360E2
:10BA100002B070BD205906600004002070B50C46CD
:10BA2000054600224FF4BF716068043041F0E4F82D
:10BA3000A8B1406802F092F9064660680022CE2163
:10BA4000043041F0D9F860B1406802F087F932461D
:10BA5000034607492846BDE87040F2F737BB054E5C
:10BA6000EBE7324628460449BDE87040F2F72EBBAA
:10BA7000943E066038700760AC3E066070B50446C0
:10BA800001221048E40044F00604214641F0B4F8D5
:10BA9000456806460DB1284670BD01210820F0F723
:10BAA00001FD094B054601202B60FDF703FBF1F773
:10BAB000A1F922464FF4BF71686041F0A5F828460D
:10BAC000756070BD580400203840066040687047BB
:10BAD00041607047034601220448DB0010B50C4664
:10BAE00043F0060141F088F8446010BD580400207E
:10BAF00030B50C4683B0232105466A462046FAF746
:10BB000033FB009B43B100216A460846FAF794FADA
:10BB100021462846FFF7DEFF03B030BD30B50546AD
:10BB200083B000220C48E90041F00601019141F088
:10BB300063F80199044618B16468204603B030BD2B
:10BB40000246064841F058F804460028F5D04168FE
:10BB50002846FFF7CDFFEFE758040020BC3E066003
:10BB600000487047E841066030B51A4683B00024AB
:10BB7000054608461146234622460094FBF7B2F8D4
:10BB800021460420F0F78EFC056003B030BD00BFF5
:10BB9000820700B583B00DD1094A0168914209D1ED
:10BBA000084AC368934205D101A904F0F7FB03B02A
:10BBB0005DF804FB04480CF06DFBFAF735F900BFA3
:10BBC00094530660CD0302607440066043681847D2
:10BBD00038B504460D4610200021F0F763FC84467A
:10BBE00094E80F008CE80F006046CCF80C5038BD8C
:10BBF00038B504460D4610200021F0F753FC84466A
:10BC000094E80F008CE80F006046CCF8085038BD6F
:10BC100038B504460D4610200021F0F743FC844659
:10BC200094E80F008CE80F006046CCF8045038BD53
:10BC300030B587B08C4611461A4602AD0A4B044611
:10BC40006046009304230195FBF758F8002110206B
:10BC5000F0F728FC0460029A4260039A8260049A1A
:10BC6000C26007B030BD00BF444106600430704779
:10BC7000032A02D00249F1F769BE0249F1F766BE14
:10BC800024150660E041066038B50C4606490546B5
:10BC90002368DA88F2F71AFA2168224628464031EA
:10BCA000BDE83840FCF7F0BBCC2606602DE9F04734
:10BCB00005460C461646C76B9946002B49D01B68B3
:10BCC00001EB1310C3F31B18B84267D18C0000219D
:10BCD00003F02AFE074622460834314640F8085B46
:10BCE00040F0FAFE38194FEA8802002140F01CFFAC
:10BCF000B8F1000F24D04FF0000AD9F808304FEA0D
:10BD0000CA0653F83A0001F087F9E96B0446D1B14D
:10BD100005F13C0C002202E001328A4213D05CF8AB
:10BD2000043F9C42F8D107EB8202936883BBD9F8A9
:10BD300008300AF1010A3344D0455B689360DCD1D6
:10BD40003846BDE8F08716480CF0A4FA2146FAF709
:10BD500073F88F4206D013480CF09CFA22463946FD
:10BD6000FAF76AF84FEA870A4946384603F0DCFDDD
:10BD7000524607460AF1080A314640F8085B40F08F
:10BD8000ABFE4A46494607EB0A0040F0CDFED7E736
:10BD900005480CF07FFA2146FAF74EF80446DAE738
:10BDA00028420660CC2406604C42066038B5136811
:10BDB0008BB90468E56B6DB104F13C0C02E0013312
:10BDC000AB4207D05CF8044FA142F8D1023350F8DF
:10BDD0002330136038BD02480CF05CFAF9F7ECFF31
:10BDE0007C4206602DE9F041074610300D460021E7
:10BDF0008000F0F757FB80463C22002140F094FE83
:10BE0000C8F83C7067B1043D08F13C0600240134D9
:10BE100055F8040F01F000F946F8040FA742F6D1D7
:10BE20004046BDE8F08100BF30B585B0019101F01A
:10BE3000F3F8019B0446174A1A40062A23D09A07B2
:10BE400003D1154A196891421DD003AA184602A9C8
:10BE5000124DFBF717FCDDE90201FFF7C3FF104AA3
:10BE600010490260104AC480104CC0E90252104AC6
:10BE7000C0E905120F4A1049C0E907420F4A416262
:10BE8000426305B030BD01A9012002F045FE034622
:10BE90000190DAE7070080FF984D066089BC0160D9
:10BEA0009453066031F60160ADBC0160ADBD016028
:10BEB000C9F60160E9F7016051F5016024500660A0
:10BEC000C368002B06DDD0E901218A4207DB00218F
:10BED00008467047FBD0D0E901218A42F7DD5100C6
:10BEE000134441F0010143600846704710B4D1E9A2
:10BEF0000143CA681B1B002A1344CCBF03F1FF3364
:10BF00000133042893FBF2F30DD0052807D123EA6F
:10BF1000E3735DF8044B5B0043F0010070470020C1
:10BF20005DF8044B70470448044A5DF8044B002B4D
:10BF3000D8BF1046704700BF882B0660802B066074
:10BF400010B4C368D0E90142CB600846034BC1E995
:10BF500001420B605DF8044B704700BFF842066079
:10BF60002DE9F041002782B00D468046194616465D
:10BF70000323012228460097FAF7B4FE3946102021
:10BF8000F0F790FA01230446C0F800809D42476014
:10BF9000C36030680CD0FBF747FA60607068FBF74D
:10BFA00043FA032DA0600AD0204602B0BDE8F0811C
:10BFB000FBF73AFAA060204602B0BDE8F081B06815
:10BFC000FBF732FAE0600028EED102480CF062F98B
:10BFD000F9F716FF9842066038B50C460546D1E9D8
:10BFE00001230949F2F772F8E268012A05D02846D0
:10BFF0000649BDE83840F2F769B828460449BDE86B
:10C000003840F1F7A3BC00BFA4420660B44206600A
:10C010007C430660136810B5144603B110BD40F2AE
:10C02000BB3399420BD0B1F5727F0DD040F2C733CC
:10C030009942F3D1C068FEF737FD206010BD40681B
:10C04000FEF732FD206010BD8068FEF72DFD2060F8
:10C0500010BD00BF042A30B5044685B025D1D0E913
:10C060000123C068A3EB020C00288444CCBF0CF170
:10C07000FF3C0CF1010C11F003059CFBF0FC2CEAD9
:10C08000EC7003D11A4B0A689A4211D00A46002379
:10C0900001462068FBF734FBE268636802FB00306E
:10C0A000400040F0010005B030BD002005B030BDBB
:10C0B00001AA04F033FD29461020F0F7F3F90D4BE7
:10C0C0000360019AE168636801FB02334360029AEE
:10C0D000E168636801FB023383600399E268002929
:10C0E00001FB02F2C260DEDAE2689B1A8360DAE7E3
:10C0F00044460660BC420660034610B4806850B1F6
:10C10000441E0422586861009C605DF8044B41F0B5
:10C110000101FBF78DBB5DF8044B7047F0B50E468F
:10C1200085B019460027012315460446009730467E
:10C130001A46FAF7D7FD3C2102AA2868FAF714F844
:10C140000299264641B102AA39463846F9F774FFEA
:10C150000446204605B0F0BD0C20F0F7A3F90446D4
:10C16000066028686060FBF749FBFBF75DF9A0609B
:10C17000204605B0F0BD00BF830709D10068064B1B
:10C18000984207D0054BC01AB0FA80F040097047BA
:10C19000002070470120704720440660E443066099
:10C1A00030B4D0E902536C689C4217D96FF040421A
:10C1B000E9681A4401EB820101E09C420ED051F87B
:10C1C000042F4FEA830C0133002AF6D0042AF4D05E
:10C1D000C360EB6830BC53F80C007047002030BCE3
:10C1E000704700BF10B4054A0023054CC1E90203A3
:10C1F000C1E9004208465DF8044B7047A1C10160E7
:10C20000084106600122043008B5FAF781FE0148B2
:10C2100008BD00BFE84106600222043008B5FAF705
:10C2200077FE014808BD00BFE841066038B50B46FF
:10C230000446002118460434FAF7AAF9054601E03D
:10C24000FAF766FE2846FAF707FA01460122204669
:10C250000029F5D138BD00BF0128F8B506460F46C4
:10C2600009D90D460124013455F8041F3868FFF739
:10C27000DDFFA642F7D10148F8BD00BFE8410660E6
:10C2800038B50B460446002118460434FAF780F905
:10C29000054601E0FAF73CFE2846FAF7DDF90146CB
:10C2A000032220460029F5D1004838BDE841066048
:10C2B00030B50B4685B0044669461846FAF768F96A
:10C2C0000434054602E0FAF723FE50B92846FAF78F
:10C2D000C3F90146002220460029F4D1024805B0E6
:10C2E00030BD024805B030BD882B0660802B06604B
:10C2F00038B5044600211020F0F7D4F8236805462D
:10C3000040F8043B6168FAF7F7FDA368E868AB60A2
:10C310006268E168920040F0DFFB284638BD00BF4C
:10C3200010B582B00191FFF7E3FF04460199FFF7D2
:10C330007DFF204602B010BD10B582B00191FFF71D
:10C34000D7FF04460199FFF79BFF204602B010BDBE
:10C3500010B5022204300C46FAF7DAFD08B10348A2
:10C3600010BD21460248F9F7EDFC00BFE841066028
:10C37000D8320660043008B5FAF798FE004808BDC8
:10C38000E84106602DE9F84380460F463AB3D1F8FC
:10C390000090B8F1010F1FD9012609F1040505E04D
:10C3A00001362846FAF782FEB04515D057F8040F3B
:10C3B0008145F5D00021FAF7EBF8044601E0FAF7E1
:10C3C000A7FD2046FAF748F901460222284600292F
:10C3D000F5D10136B045E9D14846BDE8F883086893
:10C3E000FFF786FF8146D4E7012208B5FFF7CAFFB1
:10C3F000004808BDE84106600022FFF7C3BF00BF48
:10C400002DE9F8438B070D46064603D1304B0A68E9
:10C410009A4246D0AB685BB32E493046F1F796FAA4
:10C420006A68002A4DD04FF00008002401202A4FEE
:10C4300007E001223046FAF7B1FE6A680020A24206
:10C440001CD9EB684FEA840953F824100134002901
:10C45000F5D00429F3D00028EBD139463046F1F766
:10C4600075FAEB6853F80910E3E71C49F1F76EFA27
:10C4700030461B49BDE8F843F1F768BA1949304620
:10C48000F1F764FAB8F1000F05D1BDE8F88315495A
:10C490003046F1F75BFA30461349BDE8F843F1F74F
:10C4A00055BA8B68002BE0D01049F1F74FFA0949D3
:10C4B0003046F1F74BFA6A68002AE8D04FF00108DD
:10C4C000B3E730460749BDE8F843F1F73FBA00BF8C
:10C4D000E4430660A02D06604029066070430660B4
:10C4E00078430660D48A06607C4306608043066019
:10C4F00008B50430FAF7B4FD00B108BD04480BF0EC
:10C50000C9FE40F28D3201460248F9F731FC00BF06
:10C51000882D0660D83206600528F8B50D4605D08E
:10C5200006280FD0042806D00020F8BD88684000F7
:10C5300040F00100F8BD8A68104B1148002A08BF7E
:10C540001846F8BD11F00300EED10E4B0E689E4266
:10C55000EBD14F6877B10446EB6853F824100134EF
:10C5600031B1042904D00620F9F772FC06EB60060D
:10C57000A742F1D1700040F00100F8BD802B0660A9
:10C58000882B0660E44306602DE9F04106460D461F
:10C5900010200021EFF786FF0B4B074680463146FF
:10C5A00047F8043B3846FAF7A7FC56B1043D00248F
:10C5B0000134012255F8041F3846FAF7A9FCA642B7
:10C5C000F6D14046BDE8F081204406602DE9F843ED
:10C5D0000C460021804691460846FFF7D5FF002112
:10C5E00007462046F9F7D4FF08F10406054603E0A4
:10C5F0002146FAF78DFC68B92846FAF72DF804466B
:10C6000000223046002CF3D1B9F1000F08D1384692
:10C61000BDE8F88301222146381DFAF779FCEBE7E3
:10C62000D8F80C00EFF76AFF7B68C8F80430BB68E5
:10C63000C8F80830FB68034FC8F80C303846BDE82E
:10C64000F88300BFE8410660814201D0FFF7BEBF1A
:10C650000AB102487047FFF74BBE00BFE8410660D1
:10C660000022FFF7F1BF00BF814202D00122FFF795
:10C67000ADBF0148704700BFE84106602DE9F041B9
:10C680000C4682B0002719460646904601233A46DA
:10C6900020460097FAF726FB4CB921462046FFF7C3
:10C6A00073FF05460660284602B0BDE8F0813946B2
:10C6B0003846FFF769FF05463946D8F80000F9F714
:10C6C00067FF2F1D044601E0FAF722FC2046F9F728
:10C6D000C3FF0146012238460029F5D128462E60C5
:10C6E00002B0BDE8F08100BF2DE9F04186B01446EC
:10C6F0000546CDE90010FFF73FFD002844D0002794
:10C70000009E3046FFF738FD002833D04FF0000878
:10C710001CB1AA68B3689A421CD0204B341D049502
:10C7200002931F4B03930023059302E0FAF7F0FBFB
:10C7300080B102A8FFF734FD0146002220460029FF
:10C74000F4D1184C4FB9B8F1000F0CD1204606B007
:10C75000BDE8F081144C002FF5D0281DFAF7A6FC97
:10C76000B8F1000FF2D0301DFAF7A0FC204606B059
:10C77000BDE8F08103466A4601210C48FFF77EFFC1
:10C780004FF001080646C3E7034601AA0121074806
:10C79000FFF774FF01270546B2E700BF08410660B6
:10C7A000A1C10160882B0660802B066020440660D2
:10C7B0000B46002201461846FFF796BF0022FFF7FE
:10C7C00093BF00BFF0B511F0030783B00C461646C7
:10C7D0000546CDE900120FD1464B0A689A4229D08E
:10C7E0002E2D3A460CD100223146201DFAF790FB3F
:10C7F000002856D0404C1AE0002217462E2DF2D0C9
:10C800003046FFF7B9FC88B11B2D0FD8DFE805F0E3
:10C810003B42292D340E0E0E0E151F4B0E0E0E53DD
:10C820000E0E0E0E0E1721590E0E0E60002420461D
:10C8300003B0F0BD01221746E0E7002F54D1204697
:10C84000FFF756FD31460446FFF7F0FCEFE7002FF7
:10C8500045D12046FFF74CFD31460446FFF710FD59
:10C86000E5E7A268B3689A421BD120460022314610
:10C87000FFF73AFF0446DAE7214600223046FFF789
:10C8800033FF0446D3E7204601223146FFF72CFF51
:10C890000446CCE7214601223046FFF725FF044637
:10C8A000C5E7164CC3E720463146FFF7CDFE002F03
:10C8B00008BF0446BBE769460220FFF763FD044654
:10C8C000B5E7204600223146FFF7BEFE0446AEE73C
:10C8D000002269460220FFF755FD0446A7E73146CE
:10C8E0002046FFF7CDFCA2E769460220FFF7B4FC23
:10C8F0009DE700BF20440660882B0660802B066001
:10C9000001220430FAF704BB0B4602495A68F1F7DA
:10C91000DDBB00BFCC260660CB0770B584B051D517
:10C920004A104AD403230125294E0393CDE901512E
:10C93000D0E90131C068B04238D0039028410028C6
:10C940001CDB35D0B34208D05B101FD49342A8BF84
:10C9500013465B0043F001030193B14208D0491034
:10C960001CD48A42A8BF0A46520042F00102029239
:10C9700001A9032002F0D8FF04B070BD541EAC40E2
:10C980002C4301944FF0FF340294DBE79B18DDD574
:10C990000028CCBF002301235B42DAE78918E0D5E9
:10C9A0000028CCBF002201225242DDE72846C9E719
:10C9B00008480BF06FFCF9F723FA07480BF06AFC04
:10C9C000F9F71EFA05480BF065FCF9F72DFA00BFE0
:10C9D000E841066008460660EC450660D4450660FE
:10C9E00070B504460D46104E1049F0F7AFFF012216
:10C9F00069682046FAF7D2FB31462046F0F7A6FFD9
:10CA00000122A9682046FAF7C9FB31462046F0F713
:10CA10009DFFE96820460122FAF7C0FB2046044941
:10CA2000BDE87040F0F792BF4029066024460660DA
:10CA30007C4306602DE9F041144D0C4682B0164649
:10CA4000854219461DD1002301222046009303236D
:10CA5000FAF748F9012C10D0032CD6E900870CBF57
:10CA6000B4680B4C00211020EFF71CFDC0E9005802
:10CA7000C0E9027402B0BDE8F081054C3768A046F9
:10CA8000F0E704480BF006FCFAF78CF84446066021
:10CA9000E84106602C460660136803B1704740F217
:10CAA000BB33994212D0B1F5727F0CD040F2C7333C
:10CAB00099420ED040F27F239942EFD1134601688C
:10CAC000054AF9F7C7BA8368136070474368136073
:10CAD0007047C368136070478046066070B50646AD
:10CAE0000D46102000211446EFF7DCFC024AC4601A
:10CAF0000260C0E9016570BD444606602DE9F84357
:10CB0000DFF8CC908046C0680C46174648454AD0AE
:10CB1000FAF78AFC061E53D022DDD8F804004845F7
:10CB20001CD0FAF781FC051EB8BF2D1925EAE57562
:10CB3000A542A8BF2546D8F80800484509D0FAF70D
:10CB400073FC031EB8BF1B1923EAE3718C42A8BF14
:10CB50000C46BE60C7E90054BDE8F8830025EAE74B
:10CB6000D8F80400484508D0FAF75EFC051EB8BFA7
:10CB70002D1945EAE575A54200DB651ED8F80800C9
:10CB8000484516D0FAF750FC0028BE60B8BF00191F
:10CB900040EAE070A042B4BF044604F1FF34C7E9A4
:10CBA0000054BDE8F883D8F8040001264845B8D100
:10CBB000D4E74FF0FF34BE60C7E90054BDE8F88306
:10CBC00002480BF067FBF9F71BF900BF0846066047
:10CBD000E841066010B444680C6081681160C26866
:10CBE0005DF8044B1A607047830707D10368094A50
:10CBF00093420CD010F0010003D0704700F0010008
:10CC000070470548181AB0FA80F0400970470120B3
:10CC1000704700BF902B0660703C066008B5014667
:10CC2000FFF7E2FF18B901F00303022B00D008BDA3
:10CC300002480840063818BF012008BD070080FFE1
:10CC400010B4054A0023054CC1E90203C1E90042C2
:10CC500008465DF8044B7047DDDB01600841066063
:10CC600008B5FAF793FA03460648DC880BF012FB86
:10CC700040F2CD322146944208BF4FF4D572F9F705
:10CC8000DBF800BF88460660884210B503D20378FF
:10CC9000303B092B00D910BD0023864613601EF8D7
:10CCA00001CBACF1300C03EB8303714570460CEB08
:10CCB00043031360EFD01EF801CBACF1300C5FFAE8
:10CCC0008CF4092CEFD910BD2DE9F84F8D188B4647
:10CCD00006461F46A9426AD20B46002206E0BCF176
:10CCE000220418BF01249D4209D944B113F801CB95
:10CCF000BCF1270FF3D101229D421446F5D8002A3A
:10CD00004ED0002C4CD0222422222F493046F1F75D
:10CD1000DDF9DFF8C480DFF8C490DFF8C4A00EE0CE
:10CD20005C2A2ED01F2A1CD97F2A1AD00FB11306D5
:10CD300022D425493046F1F7C9F95D450AD91BF8D7
:10CD4000012BA242ECD1224620493046F1F7BEF930
:10CD50005D45F4D8224630461B49BDE8F84FF1F74F
:10CD6000B5B90A2A12D00D2A15D0092A04D149468C
:10CD70003046F0F7EBFDE0E741463046F1F7A6F923
:10CD8000DBE713493046F0F7E1FDD6E711493046BD
:10CD9000F0F7DCFDD1E751463046F0F7D7FDCCE7A0
:10CDA0002722094930462724F1F790F9B1E72722D5
:10CDB00005491446F1F78AF9304603492246BDE891
:10CDC000F84FF1F783B900BFBC460660B446066071
:10CDD000B8460660C0460660CC460660C846066097
:10CDE000C44606602DE9F8430C461546214906461F
:10CDF0002544F0F7ABFDAC4221D2013C013D1E4F72
:10CE0000DFF88480DFF884900BE00A2A27D00D2A0F
:10CE10002AD0092A1ED041463046F1F757F9A542DB
:10CE20000DD014F8012F222A0FD05C2A0DD01F2A12
:10CE3000EBD912493046F1F749F9A542F1D1304614
:10CE40000C49BDE8F843F0F781BD39463046F1F7AB
:10CE50003DF9E4E749463046F0F778FDDFE7084959
:10CE60003046F0F773FDDAE706493046F0F76EFD1D
:10CE7000D5E700BFD4460660B4460660BC460660EF
:10CE8000C0460660C4460660D8460660C8460660CE
:10CE900099422DE9F047DDF820901F4680469246E2
:10CEA0000FD3B9F1000F10DDCE1A002408EB0405F2
:10CEB0003A46514628463FF0FFFD18B1B4424C4473
:10CEC000F4D100252846BDE8F087CC1A0026EDE70E
:10CED000F8B5074615460E4610200021EFF7E2FA96
:10CEE00004460760856086B129463046F0F70CFAA3
:10CEF00000216060681CEFF7D5FA31462A46E060F1
:10CF000006463FF0E9FD002373552046F8BD00BFFB
:10CF100008B5F0F767FAC00040F0060008BD00BF92
:10CF2000194B984270B506460C461CD000211020C3
:10CF3000EFF7B8FA0660616805468160A068F0F70F
:10CF4000E3F96860A068D4E900310131994207D162
:10CF5000AA680023E8608354A3602360284670BD5C
:10CF6000EFF7BEFAF4E7D1E90110F0F7EDF9054665
:10CF70000028DBD02046ED00F0F7DCFB002345F075
:10CF800006052360EAE700BF984D066038B5044601
:10CF90000D46F0F7D9F918B1C00040F0060038BDD1
:10CFA0002A4621460248BDE83840FFF791BF00BF3E
:10CFB000984D066010B4074C0B46844204D00648D6
:10CFC0005DF8044BFFF784BF114618465DF8044B2B
:10CFD000FFF7DCBF984D0660044B066003460A4627
:10CFE00001481946FFF774BF044B066000B50246BE
:10CFF00087B0114602A80192F0F776FB019A002152
:10D0000004983FF091FD02A90248FFF789FF07B09D
:10D010005DF804FB044B066008B50A4B0340062B81
:10D020000BD083070BD1084B02689A4207D1D0E995
:10D030000210BDE80840F0F7D5B9C00808BDFFF7F9
:10D040000FFE00BF070080FF984D0660054B0340B0
:10D05000062B03D083680B60C0687047C008F0F7E8
:10D060008FBA00BF070080FFF0B50C4689B00546B7
:10D07000174619461BB11A6832F00F0362D1002619
:10D080000323204632460096F9F72CFE4CB3012CC0
:10D0900016D03868830703D12D4B02689A4223D0FB
:10D0A00004A90122FAF728FCDDE90401F1F7E8F808
:10D0B000002849D0DDE90401FFF768FF09B0F0BDA1
:10D0C000102102AA0DEB0100F0F728FB396802A835
:10D0D0003246FAF763F804A92846FFF721FF09B0A2
:10D0E000F0BD0E2009B0F0BD02A9FFF7AFFF3A680E
:10D0F000184B04461340062B1FD0566876B1029990
:10D100002046F1F7BDF8F8B102992046F0F71CF976
:10D11000014648B1C00040F00600E0E70299204611
:10D12000F0F7F2F80646EAE7029F1020EFF7BAF9A7
:10D1300005604660C0E90274D1E7D0083FF080FD89
:10D140000646DBE7F9F746FE00210348F8F700FE44
:10D15000044B0660070080FFD436066001280A46AB
:10D1600000B583B006D1096840F20E336A4602204A
:10D17000CDE90013014600230248FFF775FF03B015
:10D180005DF804FB984D06602DE9F04304468BB032
:10D190000191F9F7FBFF02A906462046FFF756FF6B
:10D1A000019B07469A075FD0364AD468002301AA3C
:10D1B00001213448A0470346019004AA03A9184658
:10D1C000FAF760FA039D2DB30024DFF8C4802546EA
:10D1D00005E00134039B8068A34205441AD9049BEF
:10D1E0004FEA840953F82400F9F7D0FF864243D16F
:10D1F0000CB1029B1D44049B53F8090000EA08028D
:10D20000062AE6D1C0080134F0F796F9039B0544DD
:10D21000A342E4D8294606A8F0F766FA039B089DC6
:10D22000DBB10024049B05A953F824000134FFF767
:10D230000DFF059A014628463FF04EFC039B059AD8
:10D24000A342154409D9002CECD02846029A39464D
:10D250003FF042FC029B1D44E4E706A93046FFF77D
:10D260005FFE0BB0BDE8F0831968064A9142A4D076
:10D270000548814299D1A0E704480BF00BF8F8F774
:10D28000D3FD00BF1C3E066024500660E0460660E9
:10D29000070080FFF0B585B0254B0C46013802AD84
:10D2A0000431CDE900350123F9F728FD2068F9F7AD
:10D2B0006DFF002107460846FEF7D2F903A906468E
:10D2C0002068FFF7C3FE039D01460544A84211D222
:10D2D0000A461378944601320A2B0ED00D2B1FD02C
:10D2E0009542F6D8521A3846FFF764FE014630469A
:10D2F000FDF778FE304605B0F0BD01249DF80830FA
:10D30000ACEB010203B1224464443846FFF752FEFD
:10D3100001463046FDF766FEA542EBD92146D7E728
:10D320009CF801300A2B14BF01240224E6E700BF59
:10D33000E04A06602DE9F04F87B00C4607460868C2
:10D3400098460392F9F722FF06466068F9F71EFF38
:10D35000864252D104A92068FFF778FE05A9054648
:10D360006068FFF773FE049A022F824605EB020BFA
:10D3700016D8A946CB452ED3039B5246ABEB0901E9
:10D3800048460093059BFFF783FD20B31F4B9E4249
:10D390002BD0401B400040F0010007B0BDE8F08FEB
:10D3A000A3681B498B421ED00121304600912946BB
:10D3B00001F0AAFE8146032FDCD0E368144A9342B1
:10D3C000D8D00122294630460092049A01F09CFEF2
:10D3D0008346CB45D0D2B8F1000F11D14FF0FF30CA
:10D3E00007B0BDE8F08FA946E5E701462846F0F70B
:10D3F000ADFE400040F00100CFE76068FFF730FC71
:10D4000004480AF047FFF8F7FBFC00BF984D0660A0
:10D41000E84106605428066000230122FFF78ABF16
:10D4200000234FF0FF32FFF785BF00BF01231A46EC
:10D43000FFF780BF01234FF0FF32FFF77BBF00BF34
:10D440002DE9F04F8BB00C461546039010680692FC
:10D45000F9F79CFE012C0646079062D06868F9F740
:10D4600095FE864270D1069B09A958680491FFF782
:10D47000EDFDDDF8248007460499069B1868FFF748
:10D48000E5FD039B0646099D012B45D04FF0010A9F
:10D49000002435B300234FF001099B460493059304
:10D4A00002E0013D544419D0012332194146384667
:10D4B000CDF80090FFF7ECFC0028F2D1BBF1000F93
:10D4C00018D1039B002B36D0039B012B37D0013D95
:10D4D0004FF0010BCDE904445444E5D1BBF1000FFA
:10D4E0000AD11B4B079A1B489A4208BF0E200BB06B
:10D4F000BDE8F08F0494D4E7049A059B0132D21A58
:10D50000099B934212D0059B079833441946FFF7B5
:10D5100051FD0BB0BDE8F08F4FF0FF3A05EB0A0468
:10D52000B7E74FF006080C4F09A9A6E7069B186855
:10D530000BB0BDE8F08F099B05941A1BE1E7621C54
:10D54000099BCDF814B0DCE7069B5868FFF788FB11
:10D55000984D0660F44A0660604D066003460A4630
:10D5600002201946FFF76CBF03460A460020194601
:10D57000FFF766BF03460A4601201946FFF760BF62
:10D5800070B586B00C46054601A9FFF75FFD06465B
:10D590002046F9F749FF019B0446834217D2014612
:10D5A00002A8F0F7A1F82246202104983FF0BCFA27
:10D5B000019A04983146A41A00EB54003FF08CFA0B
:10D5C0002846F9F7E3FD02A9FFF7AAFC054628461D
:10D5D00006B070BD2DE9F04F04282DED028B8DB003
:10D5E000039100F0A0804FF0FF3A039C2068F9F708
:10D5F000CDFD034660681D4608EE903AF9F7C6FD7A
:10D60000039BA842044640F09A809868F9F7BEFD53
:10D61000844240F09080039C05A92068FFF716FD26
:10D6200006A981466068FFF711FD07A98346A06837
:10D63000FFF70CFD08EE100ADDE90543A3426BD8A5
:10D640004FF00008002B61D1B8F1000F05D0079A08
:10D6500018EE101A40463FF03FFA0127079D574544
:10D6600058D0002C56D02346069A44464E4698463B
:10D67000134601224146304600925A46FFF708FC05
:10D680000346F8B1069A02B901338CB39A1B6019AC
:10D690003146029315443FF01FFA079A18EE101A0C
:10D6A00060193FF019FA069A029B013705999E18F6
:10D6B000079B494457451D44A1EB060802D0B8F129
:10D6C000000FD5D14346A0461C46B8F1000F12D03A
:10D6D0002246314608EB05003FF0FEF908A918EE96
:10D6E000900AFFF71DFC0DB0BDEC028BBDE8F08F7A
:10D6F0009E1B3544D9E7291977B108A8EFF7F4FF45
:10D70000DDF82880DDE90543002B9DD00027574533
:10D710003D46A6D14E46D8E7039B18680DB0BDEC38
:10D72000028BBDE8F08FC868F9F77EFE0028F3D0C1
:10D7300040EAE07A59E7039B9868FFF791FA586846
:10D74000FFF78EFA2DE9F0470D4684B08146086850
:10D75000F9F71CFD80466868F9F718FD804560D12F
:10D7600002A92868FFF772FC03A904466868FFF75E
:10D770006DFC029AB9F1020F064604EB020721D8AC
:10D78000039A002A3CD0A3189F4248D3002505E005
:10D79000039A01351444A3189F420DD33146204605
:10D7A0003FF08AF90028F3D02046F0F7C1FC039A35
:10D7B0000446A3189F42F1D2680040F0010004B073
:10D7C000BDE8F087AB68DFF860A0534523D00121A6
:10D7D00040460091214601F097FC0246B9F1030F43
:10D7E0001BD0EB68534518D0214614460122404611
:10D7F0000092029A01F088FC039A0746002AC2D1DF
:10D80000391B2046F0F7B2FC0130400040F0010027
:10D8100004B0BDE8F0872246E0E71446B0E70120F7
:10D82000CDE76868FFF71CFAE84106602DE9F04192
:10D830000F4688B014468046F9F7A8FC05463846DE
:10D84000F9F7A4FC85423AD103A94046FFF7FEFB55
:10D8500004A906463846FFF7F9FB049B02468BB342
:10D860001B49304600948D420CBF0E211949012CF2
:10D87000079118BFCDF81C80CDE90511039908BFA9
:10D88000CDF81480FFF704FB90B1841B3146284685
:10D890002246FFF78FFB0499039A03462846069712
:10D8A000521A21440593121B3144FFF783FB079062
:10D8B00005A9032002F038F808B0BDE8F081384629
:10D8C000FFF7CEF904480AF0E5FCF8F799FA00BF33
:10D8D000984D0660F44A0660284706600122FFF76B
:10D8E000A5BF00BF4FF0FF32FFF7A0BF2DE9F04109
:10D8F000884686B0074601A94046FFF7A7FB019975
:10D90000054602A8EFF7F0FE019B049E4BB10024F0
:10D9100015F8010B0134B84706F8010B019BA3422F
:10D92000F6D84046F9F732FC02A9FFF7F9FA06B03B
:10D93000BDE8F08101460148FFF7D8BF49E2006029
:10D9400001460148FFF7D2BF5DE200600B46F0B52B
:10D9500083B00746184601A9FFF778FB019B0446F0
:10D9600033B3154E1548B74218BF874214BF01267E
:10D97000002612D1354614F8010B0135F0F714FCDE
:10D9800020B114F8010CB847064688B1019BAB42A0
:10D99000F1D86EB10A4803B0F0BD002502E0019B4A
:10D9A000AB42F7D914F8010B0135B8470028F6D17E
:10D9B000044803B0F0BD00BF19E2006031E200602E
:10D9C000882B0660802B066001460148FFF7BEBF2A
:10D9D00091E1006001460148FFF7B8BFA9E100608E
:10D9E00001460148FFF7B2BFC1E1006001460148AE
:10D9F000FFF7ACBF19E2006001460148FFF7A6BF80
:10DA000031E2006070B54D4B90B00A680C46054697
:10DA10001340062B2BD0930703D1494B1168994231
:10DA200025D012F0010612D0521000F18380114669
:10DA30000CA80192EFF758FE0021019A0E983FF0D2
:10DA400073F80CA93F48FFF76BFA10B070BD012DB9
:10DA50006BD110460D2103AAF8F786FB039B13B385
:10DA600003AA31463046F8F7E7FA10B070BDA81E99
:10DA700001285AD810460CA9FFF7E8FA22682F4B64
:10DA800005461340062B3BD05468002C32D00021B1
:10DA900010200C9EEEF706FD2A4B44600360C0E99F
:10DAA000026510B070BD2A4605A92068F9F70EFF7F
:10DAB00058BB206808ADF9F775FE60B341102846E1
:10DAC000EFF700FE20680CA9F8F762FD044607E0B6
:10DAD000F9F7AAFCFF2823D8C1B22846EFF790FE39
:10DAE0002046F8F7B9FD0028F2D129461548FFF77E
:10DAF00017FAAAE70C992846EFF706FC0446C6E792
:10DB0000D0083FF09DF80446BFE7DDE905120D4857
:10DB1000FFF7DEF999E710212846EFF7D3FDD1E7AB
:10DB200009480AF0B7FBF8F76BF908480AF0B2FBAE
:10DB3000F8F77AF90020F8F763F900BF070080FFD3
:10DB4000984D0660044B06603847066054470660EF
:10DB50000846114608B51BB11B6833F00F0306D108
:10DB600018B1BDE80840FFF74DBF024808BDF9F7FE
:10DB700031F900BFF44A0660012800B583B004D033
:10DB800050B9084803B05DF804FB0A6840F20E3350
:10DB900069460220CDE90023FFF734FF03B05DF8AA
:10DBA00004FB00BFF44A0660012A10B50C4682B09F
:10DBB00008D000234FF0FF3201208A60C1E9003312
:10DBC00002B010BD01A9FFF741FA019A01464223B4
:10DBD0000020A360C4E9001202B010BD10B582B0ED
:10DBE0000446806801A9FFF731FAE368019A93427D
:10DBF00007D2C05C01334000E36040F0010002B096
:10DC000010BD002002B010BDF0B5064685B0154627
:10DC10000C46F9F7BBFA694607463046FFF716FA95
